:100000000000012089F50000B1F50000B3F5000003
:10001000B5F50000B7F50000B9F5000000000000DC
:10002000000000000000000000000000BBF5000020
:10003000BDF5000000000000BFF50000C1F50000A4
:10004000C3F50000C3F5000041FB0000C3F500004C
:1000500071A00000C3F50000C3F50000C3F5000067
:10006000C3F50000C3F50000C3F50000C3F50000B0
:10007000C3F50000C3F50000C3F50000C3F50000A0
:10008000C3F5000005FF0000C3F50000C3F5000044
:10009000C3F50000C3F50000C3F50000C3F5000080
:1000A000C3F50000C3F50000C3F50000C3F5000070
:1000B000C3F50000C3F500000000000000000000D0
:1000C000C3F50000C3F50000C3F50000C3F5000050
:1000D000C3F50000C3F50000C3F5000000000000F8
:1000E0000000000000000000000000000000000010
:1000F0000000000000000000000000000000000000
:1001000000000000000000000000000000000000EF
:1001100000000000000000000000000000000000DF
:1001200000000000000000000000000000000000CF
:1001300000000000000000000000000000000000BF
:1001400000000000000000000000000000000000AF
:10015000000000000000000000000000000000009F
:10016000000000000000000000000000000000008F
:10017000000000000000000000000000000000007F
:10018000000000000000000000000000000000006F
:10019000000000000000000000000000000000005F
:1001A000000000000000000000000000000000004F
:1001B000000000000000000000000000000000003F
:1001C000000000000000000000000000000000002F
:1001D000000000000000000000000000000000001F
:1001E000000000000000000000000000000000000F
:1001F00000000000000000000000000000000000FF
:1002000010B5054C237833B9044B13B10448AFF350
:1002100000800123237010BDA40200200000000014
:10022000F08D010008B5034B1BB103490348AFF340
:10023000008008BD00000000A8020020F08D010031
:10024000154B002B08BF134B9D46A3F5803A0021A8
:100250008B460F461348144A121A12F05EF90F4BE0
:10026000002B00D098470E4B002B00D09847002061
:10027000002104000D000D48002802D00C48AFF307
:10028000008012F093F8200029000FF051FE11F0C9
:10029000DBFE00BF0000080000000120000000009D
:1002A00000000000A40200209009002000000000CF
:1002B00000000000002070470020704700207047B9
:1002C00000207047F0B5044685B00E4668461146DA
:1002D0001F4609F023FB23686A465D6A31463B46A8
:1002E0002046A84705B0F0BDF0B5044685B00E46DF
:1002F000104669461F4609F021FA23686A465D6A7E
:1003000031463B462046A84705B0F0BD70B590B0D9
:100310000C4615461E4605F0E7F948B364B321467E
:100320004022684613F0CDF82F21684613F060F89C
:1003300028B9234603224021684609F071FA3F227A
:100340003146684613F097F80C480DF0F1FF78B18C
:100350000B4B93F90030062B0CD10A4B93F900306C
:1003600043B901232A46694604480EF03EFA0120AB
:1003700010B070BD0020FBE72046F9E7E403002041
:10038000DC030020B403002007B5002300931A46C5
:10039000194603480EF030FF03B05DF804FB00BFC0
:1003A000C002002007B5002300931A4619460348EF
:1003B0000EF022FF03B05DF804FB00BFC80200206E
:1003C0000020704700207047406808B508B101F070
:1003D00061FF012008BD13B500220446114668469E
:1003E00003F022FE606801F055FF052805D80123BF
:1003F00003FA00F010F0250F0BD161684FF4007282
:10040000684604F003FA0021684604F0CFF802B011
:1004100010BD0020FBE713B50022044611466846D4
:1004200003F002FE2046FF22694604F03AF9204616
:1004300002B010BD07B5002300931A4619460348C1
:100440000EF0DAFE03B05DF804FB00BFD00200201E
:10045000704743683BB1B0F90A00012806D002DBBF
:100460000338022801D9002070470220704700009D
:100470002DE9FF4102AC84E80600064638493948B8
:100480009DF828501F460EF0FFFE204604F01AFB90
:10049000204603F047FF40BB204604F0A9F9052899
:1004A00004D8DFE800F015221603031605462E498E
:1004B0002C480EF0E9FE0A2229462A480EF04DFF8C
:1004C00028480EF0F1FE204604F0FCFA002009E076
:1004D000012533680095DD6B94E806003B46304605
:1004E000A847012004B0BDE8F081204604F0CAF816
:1004F000012812D0022830D01C491A480EF0C4FE40
:10050000204604F0BFF80A22014616480EF03EFFCE
:1005100014480EF0C9FE0125C9E70021204603F06A
:1005200097FF13280EDC1E21204604F001F87168A5
:100530004FF40072204604F019FE4FF420617068F9
:1005400002F072FB336801250095D3F83C8094E8F3
:1005500006003B463046C047C3E700230393F1E75C
:10056000546F01006C0300206A6F01005D6F010091
:1005700008B511B9B0F9080008BDB0F90A208A42DF
:1005800003DC0089084400B2F6E7406801F026FF6A
:10059000F9E7000007B5002300931A4619460348FF
:1005A0000EF02AFE03B05DF804FB00BFD802002065
:1005B0000A460068022100F065BD000070B50368BE
:1005C0000546F3B17221FFF7F3FF28680E4E03686A
:1005D0000021DB69984700242868042C03680CD0AC
:1005E000DB689847A35D984205D0286803685B6A7A
:1005F0009847002070BD0134EEE75B6A9847012000
:10060000F8E71846F6E700BFC46F01002DE9F04196
:10061000036804461BB900263046BDE8F081FFF7A9
:10062000CDFF07460028F6D0254672212046FFF769
:10063000BFFF55F8100B03680421DB69984704F1EC
:100640001608002620680368DB689847C0B205F8E2
:10065000010B0138C0B2FD2898BF3E46A845F1D134
:10066000206803685B6A9847D6E7F8B503680446D4
:100670000F4613B900252846F8BDFFF79FFF054632
:100680000028F7D061212046FFF792FF2068036819
:100690002646DB690421984756F8100B03680622AA
:1006A0005B68394698473B682361BB88B380206804
:1006B00003685B6A9847DEE770B5036804460D4639
:1006C000164613B90025284670BDFFF777FF0028AE
:1006D000F8D072212046FFF76BFF206803684021A5
:1006E000DB699847731E2A46002120680FF0B0F896
:1006F00006B2206803685B6A9847002EE2D00023A8
:10070000AB55E0E738B5036804460D460BB9002049
:1007100038BDFFF753FF0028F9D0284612F0A3FE9A
:100720000F28F4D872212046FFF742FF20680368A3
:100730004021DB699847294620680EF0AEFD20680D
:10074000036800211B6898470546206803685B6AB8
:100750009847281C18BF0120DAE738B5036804461B
:100760000D460BB9002038BDFFF728FF0028F9D04F
:10077000284612F078FE0F28F4D872212046FFF7A1
:1007800017FF206803685021DB69984729462068D5
:100790000EF083FD2068036800211B68984705461A
:1007A000206803685B6A9847281C18BF0120DAE7B5
:1007B00070B5036804460D46164613B90025284651
:1007C00070BDFFF7FBFE0028F8D072212046FFF72E
:1007D000EFFE206803682021DB699847731E2A46D4
:1007E000002120680FF034F806B2206803685B6AC5
:1007F0009847002EE2D00023AB55E0E738B50368F8
:1008000004460D460BB9002038BDFFF7D7FE00287F
:10081000F9D0284612F027FE1F28F4D8722120466E
:10082000FFF7C6FE206803682021DB699847294648
:1008300020680EF032FD2068036800211B6898478D
:100840000546206803685B6A9847281C18BF01208A
:10085000DAE773B5036805460E461BB90024204647
:1008600002B070BDFFF7AAFE04460028F6D0722140
:100870002846FFF79DFE286803681021DB6998472A
:1008800004220DEB020128680EF0CDFF01993046DD
:100890000EF0CFFC286803685B6A98473379002B19
:1008A000DCD0FF2BDBD17379FF2BD8D1B379FF2BB1
:1008B000D5D1F479FF3C18BF0124D0E773B50368A4
:1008C00005460E461BB90024204602B070BDFFF756
:1008D00075FE04460028F6D072212846FFF768FE10
:1008E000286803681C21DB69984704220DEB02018C
:1008F00028680EF098FF019930460EF09AFC28689F
:1009000003685B6A98473379002BDCD0FF2BDBD17F
:100910007379FF2BD8D1B379FF2BD5D1F479FF3C74
:1009200018BF0124D0E773B5036805460E461BB90E
:100930000024204602B070BDFFF740FE04460028A8
:10094000F6D072212846FFF733FE28680368142189
:10095000DB69984704220DEB020128680EF063FF63
:10096000019930460EF065FC286803685B6A984779
:100970003379002BDCD0FF2BDBD17379FF2BD8D15F
:10098000B379FF2BD5D1F479FF3C18BF0124D0E710
:1009900073B5036805460E461BB90024204602B015
:1009A00070BDFFF70BFE04460028F6D072212846E2
:1009B000FFF7FEFD286803681821DB6998470422C9
:1009C0000DEB020128680EF02EFF019930460EF063
:1009D00030FC286803685B6A98473379002BDCD0C9
:1009E000FF2BDBD17379FF2BD8D1B379FF2BD5D176
:1009F000F479FF3C18BF0124D0E737B54B68019369
:100A00000368044613B9002003B030BDFFF7D6FDDC
:100A10000028F8D072212046FFF7CAFD206803683D
:100A20001021DB6998472068036804225B680DEB9E
:100A3000020198470546206803685B6A9847281CAE
:100A400018BF0120E0E737B54B68019303680446FF
:100A500013B9002003B030BDFFF7B0FD0028F8D077
:100A600072212046FFF7A4FD206803681C21DB6982
:100A700098472068036804225B680DEB02019847E1
:100A80000546206803685B6A9847281C18BF012048
:100A9000E0E737B54B6801930368044613B90020BB
:100AA00003B030BDFFF78AFD0028F8D07221204640
:100AB000FFF77EFD206803681421DB6998472068F2
:100AC000036804225B680DEB020198470546206825
:100AD00003685B6A9847281C18BF0120E0E737B518
:100AE0004B6801930368044613B9002003B030BD7E
:100AF000FFF764FD0028F8D072212046FFF758FD6B
:100B0000206803681821DB6998472068036804227D
:100B10005B680DEB020198470546206803685B6A35
:100B20009847281C18BF0120E0E713B577230093EE
:100B300003680446A3B1FFF741FD88B17221204646
:100B4000FFF736FD206803680C21DB699847042213
:100B5000694620680EF067FE206803685B6A984764
:100B6000009B0020DAB262F30700C3F3072262F3AE
:100B70000F20C3F3074262F317401B0E63F31F609D
:100B800002B010BD37B501910368044613B90020C7
:100B900003B030BDFFF712FD0028F8D072212046C7
:100BA000FFF706FD206803680C21DB699847206881
:100BB000036804225B680DEB020198470546206834
:100BC00003685B6A9847281C18BF0120E0E707B557
:100BD000FFF7ABFFC043C0F3C01003B05DF804FBE8
:100BE00037B505460C46FFF7A0FF84F001040190DD
:100BF00064F3C7108DF804000199284603B0BDE8DE
:100C00003040FFF7BFBF07B5FFF78FFF80F0080048
:100C1000C0F3C00003B05DF804FB37B505460C46D1
:100C2000FFF783FF84F00104019064F3C3008DF8A3
:100C300004000199284603B0BDE83040FFF7A2BF89
:100C400037B50D460446FFF770FF019065F30200CB
:100C50008DF804000199204603B0BDE83040FFF74D
:100C600091BF37B50D460446FFF75FFF019065F36E
:100C700006108DF804000199204603B0BDE830400D
:100C8000FFF780BF07B5FFF750FF00F0070003B084
:100C90005DF804FB07B5FFF748FFC0F3021003B08F
:100CA0005DF804FB70B51E4D0C468AB00646043450
:100CB0001C4928460EF0E8FA214607A80FF005F86F
:100CC00007A928460EF0E4FA2846174D0EF0ECFA74
:100CD00007A80EF06AFF294601A80EF0ABFF01A994
:100CE00004A80EF0F2FF214604A80FF02EF82946C2
:100CF000044607A80EF09EFF07A920460FF025F82E
:100D0000014630460EF0E1FF07A80EF04EFF04A8A2
:100D10000EF04BFF01A80EF048FF30460AB070BD40
:100D20006C030020C96F0100D46F01007FB50D4630
:100D30000446222128460FF05DF822210646284667
:100D40000FF072F8002E034604F1040422DB0028A1
:100D500020DD721C294601A80FF06AF801A920467F
:100D60000EF0BDFF01A80EF020FF0D490D480EF05A
:100D70008BFA214601A80EF0A8FF01A909480EF040
:100D800087FA08480EF090FA01A80EF00EFF012035
:100D900004B070BD294620460EF088FFE5E700BF8D
:100DA000D66F01006C0300207FB503680446002B5A
:100DB00039D07721FFF7FCFB206803680021DB694D
:100DC00098470025206802690368954204D21B6891
:100DD000002198470135F5E7DB69144E002198475B
:100DE00000252068715D036801351B689847042D54
:100DF000F7D1206803685B6A98470D4901A80EF097
:100E000019FF01A92046FFF791FF01A80EF0CDFEC2
:100E100007212046FFF714FF07212046FFF721FF97
:100E2000012004B070BD1846FBE700BFC46F01008D
:100E3000AA8801007FB50368044613B9002004B0F6
:100E400070BDFFF7BBFB0028F8D0E3681F2BF5D877
:100E5000264672212046FFF7ABFB56F8040B0368C9
:100E60006021DB699847314620680EF011FA20684E
:100E7000036800211B6898470546206803685B6A81
:100E800098478DB10A490B480EF0FEF9314601A88A
:100E90000EF01BFF01A907480EF0FAF905480EF005
:100EA00003FA01A80EF081FE281C18BF0120C6E736
:100EB000EE6F01006C03002030B5036885B0044676
:100EC00013B9002005B030BDFFF778FB0028F8D03B
:100ED000254672212046FFF76BFB55F8040B03688B
:100EE0006021DB6998470022216801A80EF0CAFC46
:100EF00001A928460EF0F3FE01A80EF056FE206868
:100F000003685B6A98470B490B480EF0BDF9294608
:100F100001A80EF0DAFE01A907480EF0B9F906485B
:100F20000EF0C2F901A80EF040FEE068003018BFD4
:100F30000120C7E7E16F01006C03002007B5002323
:100F400000931A46194603480EF056F903B05DF8AF
:100F500004FB00BFE002002007B5002300931A46FF
:100F6000194603480EF048F903B05DF804FB00BFD2
:100F7000E802002001207047C08A7047027D1AB144
:100F80000368FF211B68184770470369994228BF0F
:100F90001946816108467047037D10B5044633B990
:100FA000A069236998422CBF0020012010BD03686E
:100FB0001B699847FF28F3D10020F7E7036810B5B5
:100FC00004461B699847A3690133A36110BD7047AC
:100FD0000368DB6A1847000008B502698369934219
:100FE00005D2C169034819440CF05FFA08BD4FF0FF
:100FF000FF30FBE7F002002010B5D0E906345A1CA0
:1010000082610A460248E1180CF051FA012010BD35
:10101000F00200207FB50D4604463F2128460EF021
:10102000E9FE031E0BDB0022294601A80EF000FF9B
:1010300001A928460EF053FE01A80EF0B6FD0F4997
:1010400028460EF08EFE064650B10023A3614FF4F1
:10105000FA43236101208423E361207504B070BD4D
:10106000074928460EF07DFE0028F7D08423C4E906
:101070000666236126750120F0E700BFFA6F0100C4
:101080000770010001294FF0000303D002290AD0A4
:101090001846704783614FF4FA4303618423C361A8
:1010A0000175012070478422C0E90633026103758F
:1010B000F7E7000007B5002300931A4619460448D5
:1010C0000EF09AF8034803B05DF804EB0CF0EAB9AF
:1010D000F1020020F002002038B5002383608380F5
:1010E000036804460D46002B47D0274A1268002AA1
:1010F00043D0002908BF1D462B7C03F00F03062BAD
:1011000010D1224A224829460CF03DFE08B143691D
:101110002371204A1E4829460CF035FE00282DD0A8
:10112000436963711C4A216819480CF02CFE05467E
:1011300008BB1A491A480EF0A7F80A226179184824
:101140000EF024F9174916480EF09EF80A2221796C
:1011500013480EF01BF912480EF0A6F82B460E4A63
:1011600021680B480CF053FE0B4A216808480CF02C
:101170000AFE054608B11435A56038BD286810F090
:1011800046FF6071CEE700BF34040020E88701000D
:101190008C07002054700100BA700100BD7001007E
:1011A0006C030020537A010010B50446016011461B
:1011B000FFF792FF204610BD41790C4A002352F8F8
:1011C0002300884203D10A4A52F82300704752F89C
:1011D000230028B942F82310054A42F8230070473B
:1011E0000133052BEBD10020704700BF080300201E
:1011F0001C03002010B50A4A4079002352F823400E
:10120000844203D1074A42F8231010BD52F823400C
:1012100014B952F82320F5E70133052BEED1F4E79A
:10122000080300201C0300202DE9F0412DED028B66
:101230009AB00546FFF7C0FF04460EF021FE0023DA
:10124000014643F69822204608F094FB002800F05F
:10125000DB8006231622697905A80DF01FFC3721D3
:1012600005A80DF02BFC0022114605A80DF040FD4D
:10127000002108EE900A05A80DF0D2FD654908EEA0
:10128000100A65480EF000F80A22697962480EF0EB
:101290007DF8624960480DF0F7FF18EE900A10F0F3
:1012A000F5FA022402460B4600945B480EF02AF938
:1012B0005B4959480DF0E8FF18EE100A10F0E6FA05
:1012C00000940B46024654480EF01CF9554952480A
:1012D0000DF0DAFF50480DF0E7FF534A29685348F4
:1012E0000CF051FD524A2968804650480CF04BFDE5
:1012F0000AAC074618EE901A0026204602F0A1FE1E
:10130000CDE900664FF0FF3194E80C00404608F04C
:101310004BFB18EE101A204602F093FECDE9006652
:101320004FF0FF3194E80C00384608F03DFB414A8D
:1013300029683E480CF027FD074600285ED0037C54
:1013400003F00F03042B59D1F5EE408AF1EE10FAA9
:1013500054D0B5EE408AF1EE10FA4FD0F4EE688A20
:10136000F1EE10FA4AD1B4EE488AF1EE10FA45D106
:101370003C2231460BA80A9611F0CFF87969402239
:10138000204612F09EF82F21204612F031F828B99D
:101390007B6903224021204608F042FA2649204674
:1013A00012F017F818EE900A02A908F0C7F92348BE
:1013B0000CF0BEFF40B1224B93F9003023B902AAD2
:1013C00021461E480DF0FCF9204612F04CF81AABED
:1013D0001844482300F8413C02A918EE100A08F00E
:1013E000ADF916480CF0A4FF40B1154B93F900304D
:1013F00023B902AA214611480DF0E2F90EF040FD92
:1014000001462846FFF7F6FE1AB0BDEC028BBDE898
:10141000F08100BFB67001006C030020C2700100B3
:10142000D2700100D9700100DB7001008C07002030
:10143000E0700100E4700100E8870100E40300208F
:10144000B40300202DE9F04F0546006887B00F4631
:10145000904640B1A86830B10378FF2903F010032B
:1014600035D11BB9012007B0BDE8F08F032AF9D0B0
:1014700047789C499C480DF007FF0A2269799A48F1
:101480000DF084FF994998480DF0FEFEAB68964830
:1014900059780A2201F00F010DF078FF3F099449B5
:1014A00091480DF0F1FE0A2239468F480DF06EFF8B
:1014B0008D480DF0F9FEAB685A7802F00F02BA427F
:1014C00007D11A786FF304121A700020CBE7002BB3
:1014D000FBD100220DF108091146484602F0A4FD97
:1014E000AB685B7803F00F03BB4223D0B8F1030F66
:1014F00020D080497C480DF0C7FE0A2269797A48DD
:101500000DF044FF794978480DF0BEFEAB6876488F
:1015100059780A2201F00F010DF038FF7449724822
:101520000DF0B2FE0A2239466F480DF02FFF6E48CB
:101530000DF0BAFE29680C2F00F2AF80DFE807F04B
:10154000073A94A1A3947394A5A784A9AB00AB68B0
:101550005B7803F00F03023B082B24D8DFE803F08D
:101560000523239D230F23231900634A63480CF0AE
:101570000AFCAB681C78064604F001042DE0604AC2
:101580005E480CF000FCAB681C780646C4F34004CF
:1015900023E05C4A59480CF0F6FBAB681C78064621
:1015A000C4F3800419E0584A54480CF0ECFB06469A
:1015B000002412E0554A51480CF0E5FBAA68137864
:1015C000D94303F0010461F300031370064620B908
:1015D0000122494604A803F004F94D4A2968474806
:1015E0000CF0D1FB4B4A2968824644480CF0CBFBF7
:1015F000834638B9BAF1000F04D15246494604A8CF
:1016000003F0EFF8002E4BD1484602F08BFE002885
:1016100046D1AB685A7867F303025A701A7866F3BA
:1016200004121A701EE73C4A34480CF0ACFBA9685F
:101630000B7883F00202C2F34002C3F34004064673
:1016400062F341030B70C8E7344A2C480CF09BFB53
:10165000A9680B7883F00402C2F38002C3F380040C
:10166000064662F38203EDE7274A24480CF08BFB21
:10167000064600289CD10222494604A803F0B1F88E
:1016800096E7274A72E7274A70E7274A78E7274A0A
:1016900076E7274A7EE7274A7CE7002426469CE730
:1016A000AB68B8F1030F5A780FD067F303025A7092
:1016B0001A786FF304121A70CDE900AB214699E84D
:1016C0000C00304608F070F9CCE602F00F01B94288
:1016D0003FF4C8AE67F307125A701A7842F010024E
:1016E0009FE700BF4C7001006C030020F870010000
:1016F00056700100547001005A7001008C070020E0
:101700005970010060700100677001006C70010089
:10171000A2700100E4700100717001007770010097
:101720007D70010082700100887001008E700100E0
:10173000957001009B7001002DE9F0435C4A95B063
:101740000746884601685B480CF01DFB5A4A396819
:10175000814658480CF017FB0646B9F1000F01D13D
:10176000002879D0554A396852480CF00CFB544A8D
:10177000396805464F480CF006FB5249044652486A
:101780000DF082FD0A2279794F480DF0FFFD4F4997
:101790004D480DF079FD0A2241464B480DF0DDFD24
:1017A00049480DF081FD5EB3337C03F00F03042B39
:1017B00026D14022716904A811F083FE44480CF040
:1017C000B7FDE8B1434B93F90030CBB92F2104A802
:1017D00011F00EFE28B973690322402104A808F015
:1017E0001FF8B8F1000F40D025B12B7C03F00F0398
:1017F000042B34D0384A012304A935480CF0F5FFF6
:10180000B9F1000F28D099F8103003F00F03042B22
:1018100022D1D9F8141004A800F0CEFF04A800F0DB
:1018200009FFB0B1B8F1000F33D025B12B7C03F024
:101830000F03042B24D002AC01220021204602F029
:10184000F3FB0123009394E80600002304A801F0B1
:101850004DFA04A800F014FD15B0BDE8F0836A69E4
:101860001378002BCCD00123C6E724B1237C03F0EE
:101870000F03042B02D00123184ABDE76269EFE78A
:1018800069690B78002BE4D0002204A801F0E2FF84
:10189000DFE724B1237C03F00F03042B02D002AC5A
:1018A0000222CAE761690B78002BD2D04246ECE7EE
:1018B000A27001008C070020E47001006C70010030
:1018C00067700100AF7001006C030020D770010049
:1018D000E4030020B40300209E820100A9820100DD
:1018E00070B598B0054602AC84E8060039483A491C
:1018F0000DF0CAFC0A22697936480DF047FD3749D8
:1019000034480DF0C1FC204603F0DCF82968344A65
:1019100034480CF038FA0023CDE900334FF0FF31A2
:1019200094E80C0008F040F829682F4A2D480CF084
:101930002AFA29682D4A06462A480CF024FA054658
:1019400060B3037C03F00F03042B27D141694022CD
:1019500008A811F0B6FD2F2108A811F049FD28B9FB
:101960006B690322402108A807F05AFF00231022C8
:1019700000930DEB02014FF40073204602F09CFF30
:101980001B480CF0D5FC48B11A4B93F900302BB929
:10199000012304AA08A916480CF027FFBEB1337C26
:1019A00003F00F03042B12D1716908A800F004FFA3
:1019B00008A800F03FFE38B10123009394E8060028
:1019C000002308A801F092F908A800F059FC18B00B
:1019D00070BD00BF6C030020B6700100D77001001D
:1019E000AB7001008C070020A2700100E4700100C0
:1019F000E4030020B403002010B503788B420446B2
:101A000004D14378402B01D1408810BD4023217080
:101A1000637008460EF004FB80B26080F5E70000BA
:101A200083682DE9F04104460D46002B00F05A81F1
:101A3000AD4F3B780133DBB20A46FF213B70FFF725
:101A400001FD637926790E3B072BC6F3400830D899
:101A5000A64A2168A6480CF096F9064648B3037CCE
:101A600003F00F03052B24D16179A248FFF7C4FFCF
:101A70000022804631469E480CF07DF94369984526
:101A80001FDA0026032D60D0A3685A7802F00F02F7
:101A9000013A0B2A59D8DFE812F01F00ED0042008E
:101AA0006A00ED007200ED009100A200AA00D300D0
:101AB000E50060790EF0E4FBA8EB00035E425E41B6
:101AC000E0E7314601228A480CF055F94669B045F5
:101AD000CCBF00260126D5E7B3F802800EF0D0F97E
:101AE0004FF6FF7381B24FF47A72404607F042FF1F
:101AF00058B3814A21687E480CF045F928B12A463E
:101B000003212046FFF79EFC1FE07C4A21687848AD
:101B10000CF039F90028F2D12A460D21F1E7B3F88B
:101B200002800EF0ADF94FF6FF734FF4967281B25A
:101B3000404607F01FFF40B12A4604212046FFF728
:101B400081FC0EF09DF9A3685880A2681378C3F356
:101B5000C001B14200F0468113F0E00F00F09C801C
:101B6000C3F34211013961F347131370B6E0B3F8C0
:101B700002800EF085F94FF6FF739622D7E7B3F88F
:101B800002800EF07DF94FF6FF7381B24FF47A7246
:101B9000404607F0EFFE0028D7D0594A2168544844
:101BA0000CF0F1F810B12A460821AAE7554A21683D
:101BB0004F480CF0E8F80028F5D1ADE7B3F8028003
:101BC0000EF05EF94FF6FF734FF4967281B2404605
:101BD00007F0D0FE0028B8D02A460921AEE7B3F8B6
:101BE00002800EF04DF94FF6FF739622EEE7B3F840
:101BF00002800EF045F94FF6FF7381B24FF47A720E
:101C0000404607F0B7FE00289FD03F4A2168384879
:101C10000CF0B9F810B12A460B2172E73B4A216853
:101C200033480CF0B0F80028F5D1394A2168304823
:101C30000CF0A9F800287FF46FAF2A46062160E770
:101C4000B3F802800EF01CF94FF6FF734FF4967252
:101C500081B2404607F08EFE00283FF476AF2A4658
:101C60000C216BE7B3F802800EF00AF94FF6FF7310
:101C70009622EDE7B3F802800EF002F94FF6FF73FB
:101C800081B24FF41672404607F074FE00283FF40C
:101C90005CAF2A46002134E70EF0F2F8A3685880C2
:101CA0005B7803F00F03002E51D0072B11D8DFE82B
:101CB00003F0481004101004104B164A21680C4819
:101CC0000CF061F840B32A4606212046FFF7BAFB24
:101CD00020B1A3681A7866F3C3021A703B78013BFF
:101CE000DBB23B70BDE8F08104030020A770010067
:101CF0008C070020300300207D70010082700100FD
:101D0000887001008E700100957001009B700100C9
:101D10007770010071700100334A216833480CF07C
:101D200032F80028CFD1324A216830480CF02BF825
:101D30000028C8D12F4A21682C480CF024F800282C
:101D4000C1D12A460121C0E72A460A21BDE7013B4D
:101D50000C2BBED801A252F823F000BF911D000049
:101D6000D31C0000971D0000971D0000D31C00002D
:101D70009D1D0000D31C0000DF1D0000DF1D0000C2
:101D8000DF1D0000DF1D0000DF1D0000971D0000AB
:101D90002A46022199E72A46052196E7164A216834
:101DA00012480BF0F0FF10B12A4607218DE70E4ACA
:101DB00021680E480BF0E7FF0028F5D10C4A216896
:101DC0000A480BF0E0FF0028EED12168094A0748D5
:101DD0000BF0D9FF01460028E6D12A4675E72A46CE
:101DE000002172E70221BEE6887001008C07002006
:101DF0008E70010059700100717001002DE9F047EB
:101E0000032986B0804669D00168624A62480BF0B7
:101E1000BAFF98F8051006466048FFF7EDFD05B2D9
:101E2000002E69D0337C03F00F03052B64D13146BB
:101E300059480BF098FF032853D9002231465648E1
:101E40000BF099FF01224469534831460BF093FF90
:101E50000222D0F814A0504831460BF08CFF4369A1
:101E60004D480A270322314607FB03F90BF083FF95
:101E700043695F43214600974B46524628460DF082
:101E80008AFE0446314644480BF06DFF052830D1E8
:101E90000422314640480BF06EFFB0F914A03E48D2
:101EA000BC42C4BF3C4640F2FF3531464C45BCBF46
:101EB0004C4600250BF057FF022826D10022314660
:101EC00035480BF058FF4369AB4251DC01223146E3
:101ED00031480BF050FF4369AB4258DB06B0BDE818
:101EE000F08705EB850464004FF000094FF420579C
:101EF000C8E74FF0010AD2E705EB850464004FF014
:101F000000094FF420574FF0010AD8F80830B3F910
:101F100002002A1A002AB8BF5242524507DC1A783A
:101F20005109052907D8013161F3471202E01A78F7
:101F30006FF347121A701B789F2B03D94C4501D0C1
:101F4000BC42CBD1A842C9D00022114604AE02A89F
:101F500002F06AF8224602A9304602F0CEFB96E86B
:101F600006004046FFF7BCFCD8F808305D80B5E7B6
:101F70000024D8F80830B3F90230A342AED021468D
:101F80004046FFF7D9FBD8F808305C80A6E701246B
:101F9000EFE700BFA77001008C070020300300208E
:101FA00008B583680246F3B1012916D00ADB03297C
:101FB00008DC0379402B0CD006D8032B02D810463E
:101FC000FFF72EFD002010E0422B02D0FAD3803B19
:101FD000F3E71046FFF712FFF4E70379042BF1D182
:101FE000FFF722F9EEE74FF0FF3008BD7FB5037C25
:101FF00003F00F03062B054623D10146124A13486E
:102000000BF0C1FE90B1037C03F00F03052B0DD143
:10201000C4680026ACB1294601A80194FFF75CF81A
:10202000039B1E600DF082FF6468F3E704AC00219F
:1020300044F80C5D2046FFF74FF802212046FFF7D9
:10204000AFFF04B070BD00BFAB7001008C07002073
:1020500038B583680446BBB1124B1B68A3B1006856
:10206000FFF7C4FFA36800251D602379032B0CD85C
:10207000012B94BF0221294660790EF0C7F8A368AE
:102080005A7865F303025A7038BD402B03D0422BB7
:10209000FAD1294600E002216079BDE838400EF00F
:1020A000B5B800BF3404002000230380704700004F
:1020B00013B50024234600942246214603480DF020
:1020C0009BF8034B1C8002B010BD00BFFC02002037
:1020D0003003002010B5044670B3204911F095F983
:1020E00058B31F49204611F090F940B31D492046CE
:1020F00011F08BF928B31C49204611F086F910B372
:102100001A49204611F081F9F8B11949204611F019
:102110007CF9E0B11749204611F077F9C8B11649AA
:10212000204611F072F9B0B11449204611F06DF952
:10213000002814BF00200E2010BD0120FCE7022063
:10214000FAE70520F8E70620F6E70A20F4E70B2077
:10215000F2E70C20F0E70D20EEE700BF0871010068
:102160002371010045710100377101004A710100BE
:10217000407101003B710100FF700100137101000B
:1021800010B50446002843D00378002B41D02D49D8
:1021900011F03BF900283ED02B49204611F035F9CB
:1021A00000283AD02949204611F02FF9002836D0CE
:1021B0002749204611F029F998B32649204611F005
:1021C00024F980B32449204611F01FF968B323494C
:1021D000204611F01AF950B32149204611F015F9A3
:1021E00038B32049204611F010F920B31E4920468B
:1021F00011F00BF908B31D49204611F006F9F0B1B2
:102200001B49204611F001F9002814BF00200C20C2
:1022100010BD1846FCE70220FAE70120F8E7082085
:10222000F6E70520F4E70620F2E70720F0E70920AB
:10223000EEE70A20ECE70B20EAE70320E8E70420BA
:10224000E6E700BF2F7101000B7101004F71010023
:102250001B71010027710100177101001F7101003E
:102260002B71010054710100337101000F710100E5
:1022700059710100406910B103685B6918477047E4
:1022800010B50446406910B103685B689847204662
:1022900010BD000008B50322016804480BF06BFD77
:1022A00008B1007D08BDFF20FCE700BF8C070020BF
:1022B00010B503220C4601680F480BF05CFDD0B14D
:1022C000037C13F00D0F16D1022262F30303037493
:1022D00043690A4903F47F432343436108480CF0F0
:1022E000D3FF21460A2206480DF050F80448BDE805
:1022F00010400CF0D9BF10BD8C070020E272010025
:102300006C03002010B503220C46016808480BF04E
:1023100032FD58B1037C03F00F03022B01BF40696B
:1023200024F0FF04204000B218BF002010BD00BF01
:102330008C07002010B503220C46016808480BF0FA
:102340001AFD60B1037C13F00D0F08D1022262F375
:1023500003030374436904F47F442343436110BDC2
:102360008C07002010B50446406968B103689B697A
:10237000984718B1606903685B69984760690368AA
:10238000DB68984708B9012010BD2046FFF782FF9F
:1023900020B14FF480712046FFF7CCFFA368002BDB
:1023A000F1D04FF400712046FFF7C4FFEBE70000C7
:1023B00010B503220C46016807480BF0DCFC48B15D
:1023C000037C13F00D0F05D14369E44364F47F44AB
:1023D0001C40446110BD00BF8C07002038B50C467E
:1023E0004168054609B9002038BD0B7C03F00F0396
:1023F000022B03D1002CF6D14869F5E7052BF2D169
:1024000005480BF0B0FC8442EDDAE2B2696802489C
:102410000BF0B1FC4069E7E78C07002038B50D46AA
:102420004168044621B9DFED1A7A17EE900A38BDEB
:102430000B7C03F00F03052B15D116480BF093FC12
:10244000854210DAEAB2616812480BF094FC002869
:10245000E9D0037C03F00F03022B0FD1D0ED057AF6
:10246000F8EEE77AE1E7002DDDD16268137C03F036
:102470000F03022B07D1D2ED057AF1E7032BD2D15E
:10248000D0ED057AD1E7032BCDD1D2ED057ACCE79B
:10249000000000008C07002008B5416869B10B7C82
:1024A00003F00F03022B06D0052B06D104480BF0D6
:1024B0005AFC00B208BD0120FCE70020FAE700BF8B
:1024C0008C07002008B5816809B9002008BD087C88
:1024D00000F00F039A1E012A00D90BB90009F5E795
:1024E000052BF2D1002203480BF045FC0028ECD06C
:1024F000007CF3E78C070020826810B5BAB1137C2A
:1025000003F00F039C1E012C00D983B9516183682D
:102510001A7C022161F303021A748268137C03F0AF
:10252000F001602902BF0A2161F30713137410BD83
:10253000826810B5BAB1137C03F00F039C1E012C06
:1025400000D983B9516183681A7C032161F30302C6
:102550001A748268137C03F0F001602902BF07211E
:1025600061F30713137410BD836853B11A7C02F032
:102570000F02901E012800D91AB91A7C61F30712C4
:102580001A74704708B5C16809B9002008BD0B7CF2
:1025900003F00F03022B01D14869F7E7052BF4D1B3
:1025A000002203480BF0E7FB0028EED04069EDE77E
:1025B0008C0700202DE9F041C36804460E46A3B9FC
:1025C00001681948184F0BF0CEFB0546042D0CDCB2
:1025D0003846D4F800800BF005FC41460246E06026
:1025E00038460BF0DDFB0135F0E7E268CAB1137C39
:1025F00013F00F0113D1022161F303031374E36895
:102600000A495E610A480CF03FFE31460A2208483A
:102610000CF081FE0648BDE8F0410CF045BE0229F1
:10262000EDD0BDE8F08100BF8C070020EA72010008
:102630006C030020006828B1007C00F00F00431FED
:102640005842584170470000F8B50446FFF7F2FFC2
:10265000002831D021683748364F0BF084FB0546FF
:10266000032D266809DC38460BF0BCFB31460246D8
:1026700038460BF095FB0135F2E7002231462D4834
:102680000BF079FB436923740122216829480BF080
:1026900072FB02226060216826480BF06CFB04226A
:1026A000A060216823480BF066FBE060207C0C28CA
:1026B0002CD002D803280ED0F8BD102830D0122814
:1026C000FAD10C200DF048FC1B4B4460036005461A
:1026D00006F07EF818E010200DF03EFC174B03606A
:1026E0000546446000212046FFF778FE03B2002B28
:1026F000B6BF40422B8128816868FFF7CDFE104BA2
:102700002B6000236881AB816561D5E714200DF053
:1027100023FC0C4B44600360054605F0F7FCF3E72F
:102720000DF01AFC084B44600360054606F030FAD1
:10273000EAE700BF8C07002034830100846F0100AA
:1027400088830100548201002884010010B5002311
:1027500004460160436103768362FFF775FF2046FC
:1027600010BD000070B5056806462F21284610F000
:10277000C9FE044698B1002300F8013BFFF700FDB5
:102780000B4905460B480CF07FFD0A2229460948F3
:102790000CF0E3FD07480CF087FD284670BD284685
:1027A000FFF7EEFC05460028F7D03460F5E700BFE0
:1027B000E97001006C0300202DE9F04389B000248A
:1027C00000F118080546CDF804804461047684625F
:1027D0000E4600293BD01F4B1F68002F37D02F21FA
:1027E000304610F005FE814650B3234602AAF05C45
:1027F00019B238B12F2805D0142B02D0D054013390
:10280000F5E7194608AB1944002301F8183C1248B3
:1028100039460BF0B8FA0F22286009F10101404651
:1028200010F04FFE01A8FFF79DFF019BA86203B9BE
:102830002B762846FFF708FF284609B0BDE8F0834D
:102840003246394604480BF09EFA2860F1E700232F
:102850002B60EEE7D80300208C07002008B5436901
:102860003BB9007C052809D014280CBF0020FF20AC
:1028700008BD1A681846526B9047F3E75020F7E7F7
:1028800018B1034903480CF0FFBC0349FAE700BF45
:10289000F57001006C030020FA7001002DE9F0438F
:1028A0009FB04FF0000802AC84E8060006461022F4
:1028B00041460AA81D46269FCDF824800FF02DFE24
:1028C0002046CDE906888DF8208002F0FBF8EB0564
:1028D0001BD5204601F0D6FE172800F2CE8001233A
:1028E00003FA00F047F6424318420AD18B4B0340EB
:1028F000002B40F0C68010F0240F00F0BE80884905
:1029000000E0884906A810F08AFD87480BF010FD0A
:10291000002800F0AA80854B93F900209846002AF1
:1029200040F0A380002F44D13B46032240210EA853
:1029300006F076FF33683F2219680EA810F09BFD61
:10294000A80540F1AD80204601F09CFE022800F071
:10295000A780204601F096FE052800F0A1802046C1
:1029600001F092FE012840F08F804FF001094FF4F2
:102970000073142209A9CDF80090204601F09CFFB5
:102980004B4609AA0EA968480BF02FFF6849694811
:102990000CF07AFC0EA967480CF07FFC664965488C
:1029A0000CF072FC09A963480CF077FC61480CF04C
:1029B0007BFC204601F0C7FC05F4805908B1AA054C
:1029C00003D4B9F1000F00F09880002303224021C6
:1029D0000EA806F025FF33683F2219680EA810F0F4
:1029E0004AFD47B155490EA810F0F3FC3F22394685
:1029F0000EA810F040FD51490EA810F0EAFCB9F104
:102A0000000F63D04E490EA810F0E3FC204601F001
:102A10003BFE043801285BD81722214604A801F0A8
:102A2000E0FE002300934FF44073142209A92046CE
:102A300001F042FF3E493F480CF026FC0EA93D48FC
:102A40000CF02BFC3C493B480CF01EFC09A9394812
:102A50000CF023FC37480CF027FC33480BF068FCE3
:102A600018B198F90030002B3CD0304629B2FFF75E
:102A700061FC00201FB0BDE8F08332492D480CF006
:102A800003FC25F4807540E7204601F0FDFD022897
:102A90003FF46BAF204601F0F7FD08283FF465AF27
:102AA000E90586D5012306AA0EA91F480BF09DFE55
:102AB0001F4920480CF0E8FB0EA91E480CF0EDFB66
:102AC0001D491C480CF0E0FB06A96CE71E499AE77B
:102AD0000023B9F1000F009314BF4FF440734FF47B
:102AE0000073A2E70EA9012309AA0F480BF07DFE8F
:102AF0004FF400713046FFF75BFCEB0571D52046C3
:102B000001F0C0FD01380D2824D8DFE800F0722361
:102B1000232323722323231F6C75706E0100800012
:102B20002371010008710100E4030020B4030020B8
:102B3000957101006C03002056700100537A01006A
:102B40000F710100877101002F7101002B4906A848
:102B500010F065FC0023032240210EA806F060FE61
:102B600033683F2219680EA810F085FC47B124494C
:102B70000EA810F02EFC3F2239460EA810F07BFC68
:102B80001F490EA810F025FC1E490EA810F021FCCC
:102B90001D491E480CF078FB0EA91C480CF07DFB6B
:102BA0001B491A480CF070FB06A918480CF075FB7D
:102BB00016480CF079FB17480BF0BAFB00283FF4DD
:102BC00054AF98F90030002B7FF44FAF0EA90123CA
:102BD00006AA10480BF009FE4FF480713046FFF74B
:102BE000E7FB012046E70C49B1E70C49AFE70C4988
:102BF000ADE7337C052BADD10A49A8E74A71010046
:102C0000537A01000B710100957101006C030020E3
:102C100056700100E40300204071010013710100AF
:102C2000FF7001003B710100F0B5CB070C4644BFBB
:102C300021F4006424F0010414F4006785B0054613
:102C40000CD004F440712846FFF774FB1449154872
:102C50000CF01AFB4FF0FF3005B0F0BD06F067FD39
:102C60009528EED902F040FD0028EAD002AE3A469F
:102C70003946304601F0D8F94FF4407229463046C3
:102C800001F0C4FD4FF440712846FFF73BFB00976D
:102C900040EA040396E806002846FFF7FFFDDBE75D
:102CA0005D7101006C03002010B54FF440710446C3
:102CB000FFF728FB014670B1074B93F90030062B54
:102CC00009D12046FFF7B0FF20464FF44071BDE820
:102CD0001040FFF76DBB10BDDC03002043691BB142
:102CE0001A681846526B1047007C70472DE9F04F68
:102CF0008FB008AD07939DF86030069385E8060015
:102D000006460DF0BDF80590284601F071FD81469C
:102D1000044602F0E9FC079B04901BB11A78002AD4
:102D200040F02C85337E13B106F118030793002C75
:102D300040F03D85079B002B40F02385D6F8289076
:102D4000B9F1000F00F03385284601F051FD00284D
:102D500040F02D855FFA89F229460CA801F04CFD60
:102D600000F025BD284601F0ADFE079B63B11B783E
:102D7000242B09D1BF49C0480CF086FABE480CF09C
:102D800093FA6FF0030B22E03168002900F03B85D5
:102D9000B9F1040F65D1B948DFF8E0820AF0E3FF2A
:102DA0000446052C376809DC40460BF01BF8394611
:102DB000024640460AF0F4FF0134F2E705223946A4
:102DC000AE480AF0D8FF044628B94FF0000B584629
:102DD0000FB0BDE8F08F284601F054FC0F28F4D85E
:102DE000284601F0EBFA002803DD237C13F00D0FD9
:102DF0000DD0237CA249A0486FF3071323740CF075
:102E000043FA9D480CF050FA4FF0010BDFE70DF04C
:102E100037F80646284601F0D1FA237C022262F3F5
:102E20000303304460612374284601F02BFC237CAB
:102E3000944960F3071323748F480CF025FA284651
:102E400001F0BCFA0A2201468B480CF064FA8E4964
:102E500089480CF019FA0A22616987480CF05BFA7C
:102E6000CFE7284601F00EFC092800F2A781DFE831
:102E700010F00A00A501A501A5012A01A501A501DF
:102E8000A5014701470100220DF1280A11465046CD
:102E900001F0CAF8284601F056FA0746002800F06B
:102EA0001081B9F10B0F00F28981DFE819F00C00F5
:102EB00087015A0087018701870187018701870100
:102EC000C500B100F300304600F082FE0028D4BFF8
:102ED000002101210A22044667480CF03EFA6B49A2
:102EE00065480CF0DAF9284601F068FA0A22014632
:102EF00061480CF010FA60480CF0D6F9002C284616
:102F000040F3348401F05AFA80BB022229460CA80F
:102F100001F067FC40F201144FF0010808E00122C3
:102F200029460CA801F05DFC40F201144FF00008A6
:102F30004FF400723146504602F054F9504601F009
:102F4000A3FB042814D1284601F09EFB022814D1CB
:102F5000284601F099FB0AA902460CA801F097FB4C
:102F60000BE0002427464FF0FF38E1E70024D3E7C9
:102F7000504601F089FB0528E5D0337C072B08D1AA
:102F8000284601F0E7F920B102220AA90CA801F0B5
:102F90007EFB3046FFF7A2FE00B200900DF1280B39
:102FA0000DF1200A0CA89AE80C00594601F004FE25
:102FB000584601F087FD3FB1504601F065FB0228FD
:102FC00016D1584602F03AF99BE8030044F4206415
:102FD0008AE803004FF0000A337C072B40F0A08101
:102FE000039BB3F5AF7F80F2EC80294900F005BC6C
:102FF000504601F049FB0128E3D0504601F044FB64
:103000000A28DED0504601F03FFB0B28DCD1D8E780
:1030100031464FF40072504602F0E4F8284601F0C1
:10302000EBF8C1B2504601F08FF898B9BA460027C4
:103030003C464FF0FF38CFE731464FF40072504620
:1030400002F0D0F8284601F0D0F80146504601F0D1
:1030500061F8EAE79AE80300022285E803002946BE
:103060000CA801F0C9FB4FF4206400274FF0000AC0
:10307000DFE700BFBB7101006C0300208C0700205C
:10308000CF710100D9710100E4710100F8700100F5
:10309000EA7101004FF400723146504602F0A2F886
:1030A000284601F088F80146504601F05EF89AE89B
:1030B000030085E803004FF0000A4FF420645746F0
:1030C000B7E78246B4E7304600F082FD00280BDD0A
:1030D000022229460CA8012701F083FB40F20114CB
:1030E0004FF0000AB84677E7012229460CA84FF0B6
:1030F000000A01F076FB40F201140127D0466BE78D
:1031000095E803000DF1280888E80300284601F03F
:103110001AF9E0B90524284601F0B4FA4FF4007218
:1031200009283146284608BF644202F05BF80022B5
:1031300029460CA801F055FBB9F10A0F3ED8DFE88B
:1031400009F01F3D0D3D3D3D3D3D3D2135002846EB
:1031500001F00CF904460028DCD0DCE700273046FB
:10316000FFF77CFB21460246284601F047F804465B
:1031700008BB98E803004FF0010A85E8030058E710
:103180000127ECE72146284601F094F828B10222F5
:1031900029460CA801F030FB8DE798E8030085E88C
:1031A000030000244FF0010A274642E72146284643
:1031B00001F0A5F8EAE74FF4206457E70024A2469F
:1031C000F2E7069B5BB17068037C03F00F03052BED
:1031D00005D1049B1BB1079A08A900F081FC08A83F
:1031E00001F050FA0338042828D8DFE800F003275C
:1031F0007A4C2A003046FFF74DF80528804602D069
:103200004FF0030BE3E5B349B3480CF03DF80A2255
:103210004146B1480CF0A1F8AF480CF045F84FF426
:1032200000723146284601F0DDFF012229460CA834
:1032300001F0D7FA44F4807444F001044FF0000820
:1032400037E03046FFF726F8062880460ED1A3491E
:10325000A1480CF019F80A2241469F480CF07DF86D
:103260009D480CF021F8022208A9E0E79C499A4801
:103270000CF00AF80A22414697480CF06EF896487E
:103280000CF012F8BCE7304600F0A2FC002823DC6A
:103290004FF400723146284601F0A4FF012229466E
:1032A0000CA801F09EFA44F4807444F001044FF03D
:1032B000060808A801F03BF830BB08A844F0010458
:1032C00001F041F818B344F400744FF0010BBAF167
:1032D000000F7FF456AD63E182497F480BF0D4FFC5
:1032E0008EE7304600F074FC00280BDD022208A9AE
:1032F0000CA844F4807401F074FA44F001044FF017
:103300000508D6E77849E8E744F48074D5E74FF438
:103310000072314608A801F079FA0028D3D1D4E729
:10332000B8F1FF3F08D1304600F052FC0028D4BF6E
:103330004FF000084FF00108B8F1000F6B496648E4
:1033400018BF01270BF0A0FF0A22414662480CF08B
:1033500004F8674960480BF097FF0A2239465E4837
:103360000BF0FBFF5C480BF09FFF079808B3FEF7DC
:10337000B1FE03903046FEF78DFF0FFA80FB039BF2
:10338000BBF1000F01D10FFA88FB4BB39B450ED068
:10339000584951480BF078FF59460A224E480BF025
:1033A000DCFF4D480BF080FF6FF0020B0FE50023B0
:1033B000079308A801F066F90E2800F2D980DFE82B
:1033C00010F0E600B0009B001C00E60079006300EE
:1033D0004800E600E600C500C500C500C500C50000
:1033E000706900283FF4F1AC0368009708AA9C6A52
:1033F000079B06CAA0478346E9E43046FEF74AFF2A
:10340000052807467FF4FCAE324933480BF03CFFF9
:103410000A22394630480BF0A0FF2F480BF044FF3A
:103420004FF40072314608A801F0DCFE337C052B16
:103430000CBF0C22012208A90CA801F0D2F944F417
:10344000807444F001044FF000084FF0FF3B012767
:103450003DE73046FEF71EFF062807460DD11F49FF
:103460001D480BF011FF0A2239461B480BF075FF6F
:1034700019480BF019FF0222DDE7194916480BF035
:1034800003FF0A223946F7E6B8F1000F7FF424AFB4
:103490004FF400723146284601F0A4FE44F48074D3
:1034A000012229460CA801F09CF944F001044FF0D8
:1034B0000608CAE7B8F1000F3FF424AF022208A9BA
:1034C0000CA844F4807401F08CF944F001044FF02E
:1034D0000508BAE7107201006C0300201F7201009A
:1034E00030720100487201005C72010073720100C9
:1034F0007B7201008272010008A800F018FF0746E5
:10350000002843D03046FEF7C5FE05283FF478AECC
:1035100044F4807444F001044FF000084FF0FF3B86
:10352000D5E608A800F003FF80B3B8F1000F0DD076
:10353000B749B8480BF0A8FE30460121FEF7B8FEA7
:103540004FF410613046FFF76FFB59E608A800F012
:10355000EEFE0746D0B108A800F0F5FE28B94FF4FA
:103560000072314608A801F03DFE44F44074D1E7F2
:1035700008A800F0D7FE08B144F4807408A800F051
:10358000E2FE074610B144F40074C5E70127BAF122
:10359000000F7FF4F6AB002C45D0D0464FF0FF3B38
:1035A0002246314608A801F0E1FDD6F814A0BAF190
:1035B000000F3CD0DAF8003000979F6A079B95E82F
:1035C00006005046B8478346706903685B6B9847AE
:1035D000052801D144F00104B8F1000F03D04146A1
:1035E0003046FEF765FE049B1BB121463046FFF7CF
:1035F0001BFB894987480BF047FE0A22594685483C
:103600000BF0ABFE854983480BF03EFE0CF038FC16
:10361000059B0A22C11A7F480BF0ABFE7D480BF0D8
:1036200043FEFFF7D4BBA0464FF0FF3BBDE7337C22
:10363000052B4BD0062BCFD151463046FEF7CEFEA0
:1036400005B2074608A801F01DF8002DC4D0BCBF84
:103650007D422DB205F1FF339BB2B8BF4FF0010A96
:10366000192BB9D807B2012128460CF0CFFDBAF1C9
:10367000000F24D0012F20D00C3F18BF012739465E
:1036800028460CF0EBFD664962480BF0FDFD0A226E
:10369000294660480BF061FE62495E480BF0F4FD7C
:1036A0000A2239465B480BF058FE5A480BF0FCFDE5
:1036B00044F4807444F0010452E00027DFE7012F56
:1036C000DDD0A7F10C035F425F41D8E7B9F1020FEB
:1036D00049D0B9F1030F09D0B9F1010F7FF47CAFE4
:1036E00044F4807444F00104CB4675E73046FEF79D
:1036F00049FF030C074605D133684B491A684B480C
:103700000BF05EF8284600F079FE0EF0BFF8484B4B
:1037100000220EF013F90EF0C1FB0FFA80F9082019
:1037200006F0A6FA69F30F07054660F31F47414903
:1037300038480BF0A9FD0A22494636480BF00DFE29
:103740003D4934480BF0A0FDA9B20A2231480BF0E4
:1037500004FE30480BF0A8FD39463046FEF72AFF3C
:103760004FF0010B38E744F40074A3E700F026FEA5
:1037700000287FF4D4AB0446FFF7D8BBB9F1000FA3
:1037800015D11B78002B3FF4D9AA07A8FEF7EAFF52
:103790008146284601F02CF828B95FFA89F22946BB
:1037A0000CA801F029F8B9F1000F3FF4C7AA05F001
:1037B000BEFF2249039017480BF066FD0A220399C9
:1037C00014480BF0CAFD1E4912480BF05DFD33682A
:1037D000104819680BF061FD1A490E480BF054FDB2
:1037E00007990C480BF059FD17490A480BF04CFD9E
:1037F000039BC72B3FF7B6AA144915480BF044FDAD
:1038000013480BF051FD4FF0FF3BFFF7E0BA00BF4C
:10381000497201006C030020B5720100BF72010003
:1038200098720100D77001009D720100E40300202E
:1038300000005940AC720100B07201009B710100A0
:10384000A0710100A7710100F8700100AD710100C5
:10385000880300202DE9F0478EB08046CDE9022193
:10386000002900F036810AB113782BB998F8183086
:1038700013B108F118030293029B63B9D8F82860CA
:1038800096B90024039D2F5D0FB3384610F00DFE4E
:1038900028550134F6E71B78002BEFD002A8FEF77D
:1038A00061FF06460028E9D00C2EEAD108AC0022C0
:1038B0001146204600F0B8FB039A21460AA800F002
:1038C00084FF324621460AA800F096FF69E02846A8
:1038D00000F078FB04ACC2B205463946204600F041
:1038E000A3FB052E20D0062E08BF17255FFA86F908
:1038F0000AAF4A462146384600F07EFF092D15DC06
:10390000082D80F2D880AA1C03DB6B1C40F3E180F9
:10391000B5B103A805F06AFE0246002841D0214651
:10392000384600F0D2FE3CE01825DFE7172D00F006
:103930009180182DEDD100222146384600F051FF2C
:1039400006AD03A9284605F072FE4A4629463846C8
:1039500000F052FF284600F097FE10F1000918BF52
:103960004FF001094FF0000A039A0FFA8AF35AB197
:10397000BAF1030F07D003A805F038FE47F82A0074
:103980000AF1010AF0E753460A2E15D00B2E1BD080
:10399000092E21D1284600F011FD81B2204600F009
:1039A000B9FB0123009394E80600029B4046FFF711
:1039B0009DF90EB0BDE8F087284600F0FFFCC1B2CB
:1039C000204600F0C1FBECE7284600F0F7FC01467A
:1039D000204600F0CAFBE4E74B449BB2013B032BBB
:1039E00030D8DFE803F00207122095E8030084E8EE
:1039F0000300D6E7284600F0E1FC9DF8283082B2AB
:103A0000214608A800F0AAFECBE7284600F0D6FC25
:103A10009DF82C2000929DF8283082B2214608A8FB
:103A200000F085FEBDE7284600F0C8FC9DF82C207C
:103A30000092214682B29DF8283008A800F077FE57
:103A40000C99C5E7244925480BF01EFC23480BF0D0
:103A50002BFCA6E700222146384600F0C2FE0025D6
:103A6000039A2BB242B1042D0AD003A805F0BEFD83
:103A700047F825000135F3E7032B10D0042B90D134
:103A80009DF8341001919DF8301000919DF82C3074
:103A90009DF82820214608A800F084FE81E79DF8C3
:103AA000301000919DF82C309DF82820214608A860
:103AB00000F068FE75E708AC03A9204605F0B7FDE5
:103AC000EAB22146384600F08CFE4A462146384686
:103AD000FAE600206DE700BFC672010088030020EF
:103AE0002DE9F0470E468EB09146002853D0037C56
:103AF00003F00F03052B62D1324DC4682B78DFF839
:103B0000C8A0DFF8C88001332B70002C54D0237C70
:103B100003F00F03042B4DD16269DAF80010404620
:103B20000AF031F90746002844D0037C03F00F0364
:103B3000052B3FD1014603A8FEF708FE5EB103A89E
:103B4000FEF778FD38B100230093316872684B4668
:103B500003A8FFF7CBF80022394640460AF00BF9DC
:103B6000E0B1037C03F00F03022B17D14369072B4D
:103B700014D10122394640460AF0FDF84A46314642
:103B8000FFF7AEFF9EB990B12B7803A8013B2B70D5
:103B9000FEF776FB01200EB0BDE8F0873EB903A822
:103BA000FEF748FD18B103A800F012F8EBE703A8F0
:103BB000FEF766FB6468A8E72B78013B2B700020BA
:103BC000E9E700BF69030020D80300208C0700202C
:103BD00073B5002205461146684600F025FA2B68A9
:103BE000464819680BF059FB454944480BF04CFB1B
:103BF0002846FEF71FFD58B9424940480BF044FBE8
:103C00003E480BF051FB4FF0FF34204602B070BD30
:103C10002846FEF73FFB0646686958B10368DB6A31
:103C2000984704B2002C05DB14BF01200020FEF7EA
:103C300027FEEAE72B7C072B14D0701C0D2811D827
:103C4000012606FA00F043F68404044004D110F083
:103C5000490F07D02046EAE72B4928480BF014FB10
:103C60003446D2E74FF400722946684600F0CEFD94
:103C70002B7C033B062B39D8DFE803F0341F3838A0
:103C800004341F006B681B7C03F00F03052B33D13A
:103C90001E491A480BF0F8FA002211466868FFF72F
:103CA0001FFF1B49044615480BF0EEFA2046FEF7AD
:103CB000E7FD12480BF0F8FAA7E70021684600F08C
:103CC00075FC044613490D480BF0DEFA21460A2222
:103CD0000A480BF042FB09480BF0E6FA003418BF23
:103CE000012492E7684600F069FBEAE70A490348C5
:103CF0000BF0CAFA002488E70024E3E76C030020F5
:103D0000F8700100F6720100F5700100D97501002C
:103D1000FF7201000C730100027301002DE9FF41E5
:103D20002C4BB3F900600546002E4DD14FF4806155
:103D3000FEF7E8FA00284AD002AC32463146204667
:103D400000F072F94FF440722946204600F05EFD03
:103D5000214922480BF098FA28464FF48061FEF77B
:103D600027FB6869002832D0036801270097D3F841
:103D7000288094E806003346C047431C044626D0FA
:103D80002B681648196884B90BF087FA1449134850
:103D90000BF07AFA134911480BF076FA0F480BF042
:103DA00083FA204604B0BDE8F0810BF076FA0C49A6
:103DB0000A480BF069FA0C4908480BF065FA074805
:103DC0000BF072FA3C46ECE74FF0FF34E9E70224CF
:103DD000E7E700BF3E0300206E7101006C03002086
:103DE000E8710100907B0100837101002DE9F04131
:103DF000244BB3F900308CB0002B3FD1224E234F1F
:103E00003278013232703A68002A35D0D568DFF84E
:103E1000888001243A680AB305B32B7C03F00F03B2
:103E2000052BF8D12946404609F09DFF0128F1D91C
:103E3000294601A8FEF78AFC01A8FEF7FBFB30B17A
:103E400001A8FFF76BFF00B20028D8BF00240CF0D8
:103E50006DF801A86D68FEF713FADBE70C480BF06C
:103E600023FA3378013B337054B10A4B00221A70A5
:103E700020460CB0BDE8F0810124F2E70024F7E70A
:103E80000124F5E73E03002069030020D803002049
:103E90006C0300203C0300208C0700202DE9F04734
:103EA0003C4B1B7886B004468A460BB1FFF79EFF59
:103EB00005222168384809F05EFF0746002851D0E6
:103EC00090F8108046694FEA18180BF0D9FFB8F146
:103ED000000F47D002AD361A42460B2128460DF19D
:103EE000100900F0A1F832462946484600F0EDFBE3
:103EF000BAF1040F17D10023009395E806004FF4A0
:103F000080532046FEF7CAFC0A224FF47A712348F8
:103F100096FBF1F10BF0FFF9214920480BF0B4F9C1
:103F20001E480BF0C1F9002E1CDA1E4B9E4219DB15
:103F3000002600964FF4805395E806002046FEF7D1
:103F4000ADFC42463146484600F06EF8012300932E
:103F500099E8060033462046FEF7C8FE3B7C66F330
:103F600007133B74BAF1010F02D12046FEF79CFE05
:103F7000606918B9002006B0BDE8F08703689B6946
:103F800098470028F6D0606903680FFA8AF19B68A9
:103F90009847F0E73C0300208C0700206C030020CA
:103FA000D37201000200008007B5002300931A4677
:103FB000194603480BF020F903B05DF804FB00BF7D
:103FC00034030020F8B50646F0B10378E3B12D2B99
:103FD0001ED0A3F13002092A1AD9252B1AD07B2B27
:103FE0001AD0232B1BD00F4F012404EBC4053D44F2
:103FF00028460FF038FA2946024630460FF04FFAAD
:1040000020B10134192CF0D14FF0FF342046F8BD17
:104010000024FBE70824F9E76FF00104F6E7172412
:10402000F4E700BF2973010010B500238370C3704B
:10403000037143718371C37161F30713437002709D
:1040400010BD10B50023072403708370C37064F3A0
:1040500007134370416010BD93B2112B70B5164623
:104060009CBF134AD25C4B7888BF002262F30713CF
:104070004B7005460C460F480F490BF005F90A2214
:1040800031460C480BF069F90C490A480BF0FCF872
:10409000617808480A2209090BF078F905480BF005
:1040A00003F923682B6063686B60284670BD00BF0E
:1040B000177301006C030020807401008B740100F1
:1040C0004B781B09013B082B1AD8DFE803F0160ECA
:1040D0000E19191919050C000C4B4B600B68036085
:1040E0004B68436070470A4BF7E764238B71CB79C9
:1040F00023F00103CB7100234B71FF230B71EDE71C
:1041000000230B714B718B71CB71E7E70000A0416D
:104110000000964243781A0903D0022A05D00020F5
:104120007047022262F30713437040F26D13994205
:10413000A8BF1946C379817123F00103C1F300219F
:104140001943C1710120704743781A0903D0022A2C
:1041500005D000207047022262F3071343706429E0
:10416000A8BF642141710120704713B50446084679
:1041700031B9E37960F34703E371012002B010BD68
:10418000642300934FF4FA72002399210BF003FD8E
:1041900063781A0908D0032A0BD820EAE070642853
:1041A000A8BF64200130E4E7022262F307136370C2
:1041B000F3E70020E2E707B5C27912F0FE0F11D055
:1041C00043781B09013B022B0CD850084FF4FA73BB
:1041D000009364229923002101380BF0DCFC03B02A
:1041E0005DF804FB4FF0FF30F9E7C379827903F003
:1041F000010342EA032070474079704743781B0966
:10420000013B10B50A2B53D8DFE803F006065252E3
:1042100052482F2F2F1010000279642391FBF3F1E5
:10422000114481F308010171012010BD6329446824
:104230004FF064030FDC03FB04112AB1534399428E
:10424000A8BF194621EAE17143784160062262F372
:1042500007134370E8E791FBF3F12144E2B1914287
:10426000A8BF114621EAE17116E0436807EE903AD3
:10427000FDEEE77A642417EE903A91FBF4F11944CD
:1042800022B19142A8BF114621EAE17107EE901ACE
:10429000F8EEE77A17EE901A4160C5E743681944D3
:1042A000002AF9D0642353439942A8BF1946D9E79D
:1042B0000020BAE743781B09022B1ED1C27983790B
:1042C00002F0010243EA0223642291FBF2F1194455
:1042D000B1F5B77F0FDA40F26D1331EA210128BF43
:1042E0001946C379817123F00103C1F300211943F9
:1042F000C171012070470021F3E700207047437827
:104300001B09022B0CD14379642291FBF2F1194471
:1043100021EAE1719142A8BF114641710120704725
:10432000002070470078003018BF012070474378A4
:1043300003F00F03012B04D80078003018BF0120D0
:10434000704700207047437813F0F00F14BF01202E
:1043500000207047407800F0E000202804D0A0F151
:1043600040035842584170470120704743781B0969
:10437000013B0A2B1ED8DFE803F00A0A1D06061BC4
:104380000F0F0F06060043686420584370470079FA
:10439000642310FB03F0704743689FED077A07EE34
:1043A000903A67EE877AFDEEE77A17EE900A70474B
:1043B00040687047002070470000C84243781B09DE
:1043C000013B0A2B18D8DFE803F00808170606128D
:1043D0000A0A0A060600406870470079704740687C
:1043E00007EE900AFDEEE77A17EE900A70474068F4
:1043F000642390FBF3F070470020704743781B095B
:10440000013B0A2B1ED8DFE803F013131D06060E2E
:10441000191919060600436807EE903AF8EEE77A94
:1044200017EE900A70474368642293FBF2F3F3E7B8
:10443000037907EE903AF8EE677AF1E7436807EE02
:10444000903AEDE7DFED017AEAE700BF00000000F7
:1044500043781B0907B50B2B60D8DFE803F0621621
:10446000165F5F5F44245F5F0606406849B1D0F184
:10447000640056D46428A8BF642000B203B05DF87D
:1044800004FB0028F6DA0846F8E7007931B100218C
:1044900000916423FF220BF07EFBEEE76423009380
:1044A000FF220B46F7E7436807EE903A99B19FED7C
:1044B0001F7A77EE677AF5EEC07AF1EE10FA30D413
:1044C000F4EEC77AF1EE10FA2DDCFDEEE77A17EE86
:1044D000903A18B2D2E7F5EEC07AF1EE10FAD2D4E3
:1044E0009FED127AECE7436861B142F27372934236
:1044F00017DC13F1630F16DB6FF0630093FBF0F032
:104500006430BAE713F1630FBDDB42F2737293427A
:104510004FF06400B2DC93FBF0F0AEE74FF0FF30F9
:10452000ACE70020AAE76420A8E700BF0000C8426B
:1045300013B50446084663781B09013B0A2B32D8A1
:10454000DFE803F00F0F313131281A313106060050
:10455000FF2300930023642219460BF01CFB6060CC
:1045600007E0FF2300930023642219460BF013FB9E
:104570002071012002B010BDFF23009300236422AC
:1045800019460BF008FB07EE900AF8EEE77A17EEF3
:10459000900AE4E746F29C33009300236422194614
:1045A0000BF0F9FA60600020E4E7000043781B0993
:1045B0000B2B5FD8DFE803F06117175E5E5E461EC7
:1045C0005E5E0606406841B1002839DBFF28A8BFBF
:1045D000FF20C0F1FF0001B20AE0002808DBFF283D
:1045E000A8BFFF20F7E700790029F4D0C0F1FF0150
:1045F000084670474368A9B107EE103AB5EEC07A95
:10460000F1EE10FA1CD4DFED1E7AB4EEE77AF1EE8B
:1046100010FA32DC77EEC77AFDEEE77A17EE903AC1
:1046200019B2E5E707EE903AF5EEC07AF1EE10FA2E
:10463000DED49FED137AF4EEC77AF1EE10FAEBDDDB
:10464000FF21D5E7406859B110F1630FF8DBB0F5F1
:10465000C84F12DA6FF0630190FBF1F0FF30BAE758
:1046600010F1630FC4DBB0F5C84FE9DA642190FBA9
:10467000F1F0B0E74FF0FF31BAE70021B8E700BF33
:1046800000007F43007870474078000970474B78FE
:1046900010B562F307134B700B6803604B684360FF
:1046A00010BD4B7810B51C09013C012C84BF0124BE
:1046B00064F3071382F30802D2B288BF4B700B6811
:1046C0000A7103604B68436010BD4B784A6030B597
:1046D0000A2565F307134B700B6803604B68436052
:1046E00030BD4B784A6030B5072565F307134B7032
:1046F0000B6803604B68436030BD4B7830B50625CE
:1047000065F307134B700A235A434A600B68036032
:104710004B68436030BD4B784A6030B5062565F381
:1047200007134B700B6803604B68436030BD70B576
:104730004C788A71022666F307144C70C2F3002489
:10474000CA794B7122F001029DF810300B7122439F
:104750000B68CA7103604B68436070BD70B54C78DC
:104760008A71032666F307144C70C2F30024CA79D9
:104770004B7122F0010222430B68CA7103604B683F
:10478000436070BD70B54D784B71042666F3071514
:104790009DF810304D700B718A710B6803604B6887
:1047A000436070BD70B54D784B7105269DF8103093
:1047B0000B7166F307159DF814304D70CB718A713B
:1047C0000B6803604B68436070BD4B784A6030B53E
:1047D0000C2565F307134B700B6803604B6843604F
:1047E00030BD10B50A700B6803604B68436010BDA4
:1047F000407800F00F0070474B7810B562F3030368
:104800004B700B6803604B68436010BD2DE9F041AD
:10481000044616460D4619B900273846BDE8F08112
:104820000846FDF707FF07460028F5D02846FDF7A4
:1048300049FEF305804603D52846FDF72BFD207081
:1048400006F40076B8F1000F09D0637868F3071317
:104850006370002EE1D0AB685B696360DDE7002E1A
:10486000DAD0AA68137C03F00F03022B03D0032BCA
:1048700009D04746D1E76378526962600A2161F343
:1048800007136370C9E753696278072161F3071260
:104890006270E2E710B50023044603704370837032
:1048A000C370037143718371C3714FF40072FFF7DA
:1048B000ADFF204610BD00002DE9F0432DED028B29
:1048C00085B00446154699469DF838800F46002964
:1048D00048D0002A00F0DC8000230B70017871B30F
:1048E00019F4807F2BD06B4B01EBC1011944384682
:1048F0000EF0E7FD637813F0F00F07D019F4007F96
:1049000004D02A46644938460EF0B5FD38460EF00C
:10491000AAFD2D1A3E18013D637813F0F00F21D047
:1049200019F4007F1ED01B09013B0B2B1AD8DFE8BE
:1049300003F00835669BA125707070221FA93E46C2
:10494000EAE72079B8F1000F06D064230093002332
:10495000FF2219460BF01FF9504A034629463046FC
:104960000EF076FC384605B0BDEC028BBDE8F08356
:1049700063684B4AF2E763684A4AEFE7616864227A
:1049800091FBF2F302FB1312002AB8BF52420092CD
:10499000454A294630460EF05BFCE3E72046FFF728
:1049A0000AFCE279A37994F8059001B200292079F4
:1049B00002F0010202DBB8F1000F14D043EA022436
:1049C000B8F1000F06D0642300930023FF2219469C
:1049D0000BF0E1F8CDE900902346344A29463046F1
:1049E0000EF036FCBEE7CDE90101CDF8009043EAB8
:1049F00002232F4A294630460EF02AFCB2E7E3791B
:104A0000A2796179009103F0010342EA0323294A64
:104A1000BFE7636808EE103AB5EEC08AF1EE10FA0F
:104A20004CBFF1EE487AF0EE487AFDEEE78AB8EE38
:104A3000E87A77EEC77A9FED207A67EE877A17EEED
:104A4000900A0BF0D1FC07EE900AB5EEC08AFDEE9D
:104A5000E77AF1EE10FACDED007A18EE903A01D532
:104A6000164A96E7164A94E72279A3790192627969
:104A70000092B2E7E279A3790292227901926279F7
:104A80000092B6E72A46616830460EF01AFD69E7E3
:104A9000174667E729730100F8700100A17401004F
:104AA000A4740100A8740100AC740100B874010082
:104AB000B5740100BB74010000007A44C1740100A8
:104AC000C274010030B58BB0134C00232022009338
:104AD00002A94FF440730546FFF7EEFE02A92046F7
:104AE0000AF0DBFB0D4920460AF0CEFB69780A226A
:104AF000090920460AF04AFC094920460AF0C4FB8D
:104B000069780A2201F00F0120460AF03FFC204696
:104B10000AF0CAFB0BB030BD6C0300208E7401009C
:104B20009374010070B54B78B2EB131F86B0054645
:104B30000C46164606D123682B6063686B602846D6
:104B400006B070BD184919480AF09EFB61781748F5
:104B50000A2209090AF01AFC154914480AF094FBC4
:104B60000A22314611480AF011FC12490F480AF096
:104B70008BFB0023CDE9043366F3071322788DF80D
:104B800011304FF0FF338DF81020009302A86368B6
:104B9000226804A900F010F8029B2360039B636065
:104BA0002046FFF78FFFC6E7CA7401006C030020A0
:104BB00056700100F87001002DE9F04F8DB004AD82
:104BC00085E80C00BDF85830112B98BFB64A8046D6
:104BD00028460C4694BF12F803904FF00009FFF7E7
:104BE000EAFA011E02DB2046FFF7BFFA9DF81130FA
:104BF0006278C3F3030161F3030262709DF8101041
:104C00002170C2F303120B2A38D8DFE812F0A0009B
:104C10000C000C00C9002F010D01A800CF00CF002F
:104C2000CF00A800A8001B090C2B77D8DFE803F001
:104C3000265244180A073955767630306E009DF8B2
:104C40001720E2719DF81620A2719DF8152062715F
:104C50009DF814202271627863F3071262700DE0F0
:104C6000BDF81630C3F30802E379A27123F0010303
:104C700043EA1223E3719DF815306371B9F1000F17
:104C800000F0FC804A46214606A8FFF74BFFF5E0FE
:104C9000059B002B36DBFF2BA8BFFF23DBB2237164
:104CA000ECE7059B13F1630F2CDBB3F5C84F2BDA50
:104CB000642293FBF2F3F1E7BDF81630C3F3080268
:104CC000E379A27123F0010343EA1223E3719DF813
:104CD000153063719DF81430E1E7DDED057AF5EEEE
:104CE000C07AF1EE10FA0DD49FED707AF4EEC77A27
:104CF000F1EE10FA08DCFCEEE77ACDED027A9DF8D1
:104D00000830CCE70023CAE7FF23C8E763780C220A
:104D100062F307136370059B6360AFE764496548FE
:104D20000AF0B2FA9DF8111062480A2209090AF045
:104D30002DFB61495F480AF0A7FA61785D480A22B5
:104D400009090AF023FB5B480AF0AEFA96E762789D
:104D50001B0963F307120598627060608EE71B09F8
:104D6000032B04D00C2BD1D0059A626073E700218D
:104D70002046FFF71BFCBDF816302071C3F3080274
:104D8000E379A27123F0010343EA1223E3719DF852
:104D9000153063716378022262F3071363706DE765
:104DA00000212846FFF702FC2071F3E71B090C2BBA
:104DB000B4D801A252F823F07D4C0000F74D00005A
:104DC000254E00006F4D0000254E0000254E0000CE
:104DD000ED4D0000194E0000194E0000194E000064
:104DE000054E0000134E00000D4D0000059B636052
:104DF00006226378D0E79DF8143007EE903AF8EE7B
:104E0000677A03E0DDED057AF8EEE77A17EE903A7F
:104E100082E7DDED057AF2E7627863F307126270EC
:104E2000059B79E7627894E701271B090C2B3FF675
:104E300075AF01A252F823F07D4C0000914E0000A6
:104E4000E54E0000914E0000714E0000714E0000D2
:104E5000914E0000914E00001D4D00001D4D0000C0
:104E6000914E0000914E00000D4D00000027DCE740
:104E7000059A6260627863F3071262702368C8F86B
:104E800000306368C8F8043040460DB0BDE8F08FCC
:104E9000013B0A2B00F2CD80DFE803F0BACB10CB48
:104EA000CBBFC4CBCBBDBD001773010000007F4357
:104EB0000A7401006C03002056700100FF23BDF846
:104EC00016208DF81430642161F30802ADF8162025
:104ED00000228DF815209DF81120022161F30712A0
:104EE0008DF811200023FF259DF815000095642200
:104EF00019460AF050FE0028C0F29D8000239DF85C
:104F000015000095642219460AF045FEA84208DC07
:104F1000002300959DF81500642219460AF03BFE17
:104F200005469DF81400FBF793FA0646002F47D07C
:104F30009DF817707F08013F3FB27B1C40F08880CE
:104F40007F2D4FF0FF0778DC0023C5F17F00194665
:104F500047F68162704300970AF01DFE4FF4FF731D
:104F6000009300231946E0717F2228460AF013FEC1
:104F70000023194600903A4630460AF00CFE00978E
:104F80000646642328467F2200210AF004FEBE4222
:104F90000546A8BF3E466B496B480AF075F90A22E0
:104FA000294669480AF0D9F9684967480AF06CF956
:104FB0000A22314664480AF0D0F963480AF074F9CD
:104FC00000231A46194606A809F0D7FFBDF81600B7
:104FD0004FF6FF7300930023194640F26D12C0F3A1
:104FE00008000AF0D8FDF2B2E9B280B209F0DBFFA6
:104FF000030CA371030A63712071554952480AF0EA
:1050000043F92046FFF75EFD06A809F04BFF35E6A1
:105010009DF8143053E7059B51E7059B642293FBF1
:10502000F2F34CE7DDED057AFDEEE77A17EE903A04
:1050300045E7002343E7002573E7642328460097EC
:105040003A4680210AF0A7FD00230546E371A2E756
:105050004FF01E0B64231A46CDF800B000213846ED
:105060000AF099FD4FF0640A03905B463846CDF88C
:1050700000A0524600210AF08EFD7F2D83464FF09E
:10508000FF0754DCC5F17F00002370431946314A05
:1050900000970BFB00F00AF07EFD4FF4FF73E07108
:1050A0000398009300231946E32228180AF073FDA1
:1050B00000231946029000903A4630460AF06BFDF4
:1050C00000230646009728467F2219460AF063FD12
:1050D000BE420546A8BF3E461F491B480AF0D4F809
:1050E0000A22039918480AF016F91C4916480AF0D2
:1050F000CBF80A22594614480AF00DF9184912480B
:105100000AF0C2F80A2229460F480AF026F9154982
:105110000D480AF0B9F80A2231460B480AF01DF989
:10512000114909480AF0B0F80A22029942E75346A9
:10513000284600973A4680210AF02DFD00230546B7
:10514000E371C9E71C7401006C030020297401009D
:105150005C740100646A3100377401003D74010021
:10516000437401004B74010053740100F8B5054607
:1051700017460C4611B900263046F8BD0846FDF723
:1051800059FA06460028F6D0FA0503D529782046B4
:10519000FDF78EF8BB050DD56B7869681B09073BD9
:1051A0002046042B11D8DFE803F00303100D0D0097
:1051B000FDF7BEF909490A480AF066F82846FFF7E4
:1051C00081FCD9E7FDF798F9F4E7FDF795F96978DF
:1051D00020460909FDF7C8F9ECE700BF9A74010001
:1051E0006C03002073B504460D46FFF70FFB06461F
:1051F000E8B9104910480AF047F82846FDF76EFD57
:10520000214602B26846FEF727FF21466846FEF7B0
:1052100057FF29464FF400722046FFF7A7FF2046AC
:10522000FFF750FC4FF420612846FDF7FDFC3046A7
:1052300002B070BD637401006C03002043781B0949
:10524000013B012B37B5054620D80023FF24007908
:105250000094642219460AF09EFC002814DB002307
:1052600028790094642219460AF095FCA04207DCD4
:10527000002300942879642219460AF08CFCC4B2F9
:105280002C71012003B030BD0024F9E70020F9E7BC
:1052900007B5002300931A461946034809F0ACFFEE
:1052A00003B05DF804FB00BF4003002002F0FEBC29
:1052B00002F0C2BC07B5002300931A461946034802
:1052C00009F09AFF03B05DF804FB00BF480300201B
:1052D00038B5094D01244FF47A700AF005FE2146D5
:1052E00001340A222846E4B20AF050F8142CF2D114
:1052F0004FF4FA7038BD00BFB803002008B5044968
:10530000044809F0C1FF04F025FB4FF4FA7008BD12
:10531000B3790100B803002010B5044604300AF048
:1053200044FC204610BD00000128F8B507460C4695
:10533000174E184D13DD48680CF069FEC1B21648CF
:105340003170FBF77DFC022F07D0A0680CF05FFEE8
:10535000C1B211482970FBF784FCC82401E04FF466
:10536000C8740E490E4809F08FFF0A2231780C48A4
:105370000AF00CF80B490A4809F086FF0A2229783E
:1053800007480AF003F8064809F08EFF2046F8BDEA
:10539000050000200600002040040020487B01009A
:1053A000B80300205C7B010030B587B000230446C1
:1053B00000931A460D4602A8194609F01DFF04A8DD
:1053C00009F012FF042C12DD04A9286904F0B7F9D2
:1053D00068B104A92348FBF736FB04A9E86804F088
:1053E000AEF950B104A91F48FBF779FB0BE002A905
:1053F0001C48FBF728FB032CEFDC02A91948FBF73C
:105400006EFB022C18DD04A9A86804F098F998B185
:1054100004A91448FBF73DFB04A9686804F08FF960
:1054200080B104A90F48FBF7E8FA0F490F4809F0CB
:105430002BFFC82007B030BD02A90A48FBF729FBA3
:10544000012CE9DC02A90748FBF7D7FA012CECD1C3
:1054500002A90448FBF7D1FA0549044809F014FFF2
:10546000E3E700BF4004002039760100B8030020C4
:105470002976010008B548B149680548FBF742F9AB
:105480000449054809F000FFC82008BD0146F4E7BB
:10549000400400209B760100B803002008B548B105
:1054A00049680548FBF759F90449054809F0ECFE3D
:1054B000C82008BD0146F4E7400400209D790100A2
:1054C000B803002030B5144D144C85B0772201216B
:1054D0002846FBF7D7FD00230193114B0093114998
:1054E00002954FF0FF332046039309F0CDFE0E4B9B
:1054F0000E4819686A4608F00FFC2846FBF768FD5D
:105500000B49204609F0C0FE204609F0CDFE0948AF
:10551000FBF790FC05B030BD58040020B803002014
:105520008888010003790100340400208C070020E2
:105530001D79010040040020012810B50C4622DD31
:10554000124960680DF027FF18B901211048FBF7D8
:1055500047FB104960680DF01EFF014610B90C486A
:10556000FBF73EFB0C490D4809F08EFE0848FBF79F
:105570002EFB0A220146094809F0EFFE074809F010
:1055800093FEC82010BDFFF79DFFFAE76B81010075
:10559000400400206E8101002D790100B803002035
:1055A00070B52DED028B08EE102A8EB01C22334B05
:1055B00006930C460DEB020000210CF0AEFF06AA8C
:1055C0000821204603F0CAFF2D4B1B6800258DF8EB
:1055D0002950002B4ED02B4809F066FE2A49294855
:1055E00009F052FE18EE100A0CF050F902230246A0
:1055F000009324480B4609F085FF2449214809F00F
:1056000043FE06A91F4809F048FE21491D4809F03C
:105610003BFE1C4809F048FE1E4B1F48196806AAAD
:1056200008F0B1FBDFED1D7AB4EE678AF1EE10FAF7
:1056300006461FD0DFED1A7AB4EE678AF1EE10FA53
:1056400018D0B5EE408AF1EE10FA13D018EE101A09
:1056500004AC02A8FEF7F5FC032202A92046FFF7DE
:10566000CBF8CDE900554FF0FF3194E80C003046FF
:1056700004F09AF90EB0BDEC028B70BD4E494C009F
:10568000340400206C030020AD720100437F010050
:1056900057700100280400208C0700200000FEC283
:1056A0000000AA4210B50C48FBF77EFB18B10B496D
:1056B0000B4809F0E9FD0B4C722201212046FBF753
:1056C000E1FC237D1BB1FF212046FBF795FC05483B
:1056D000FBF77EFCC82010BD40040020A47C010024
:1056E000B803002058040020034B93F9000005384C
:1056F00018BF0120704700BFDC03002030B593B015
:1057000000230A460546402101A804F089F801A8B3
:105710000DF0A9FE01A90446024628460DF0BFFE81
:1057200000280CBF2046002013B030BDF0B5044661
:105730009DB00E4601B18AB96E496F4809F0A4FDCB
:105740006E496D4809F0A0FD21466B4809F0A5FDA2
:105750006B49694809F098FD674821E000258D54A0
:1057600003F0E5FF63490746634809F08DFD0A220F
:105770003946614809F0F1FD62495F4809F084FD4E
:1057800021465D4809F089FD5F495B4809F07CFDD1
:10579000B7F59D7F08DA5D495D4809F075FD5C4805
:1057A00009F082FD1DB0F0BD04215A485A4F03F0A4
:1057B0004DFE5A49504809F067FD31464E4809F000
:1057C0006CFD56494C4809F05FFD4B4809F06CFDF3
:1057D0003C2229460DA80C950CF09FFE97F900205D
:1057E000052A2FD103212046FFF788FF05B2002D9F
:1057F00034D14B4BDB681B78DB07D3D50221204625
:10580000FFF77CFF00B2A8B1242120460DF07AFEFC
:105810000028C7D14349384809F036FD21463648AB
:1058200009F03BFD344809F03FFD21463C4808F0B3
:1058300068FFB7E701212046FFF760FF00B20028AC
:10584000B0D0E1E701212046FFF758FF05B2C5B906
:1058500002212046FFF752FF05B2C5B12544324967
:1058600028460DF0D2FDA0B930460DF0FCFD012810
:105870000FD921462A4808F044FF304608F036FB8D
:1058800090E73F2221460CA80DF01BFEE6E72749D2
:105890005FE7204624210DF035FE0446002881D123
:1058A000294601A8FCF788FF01A8FCF7C3FEE0B178
:1058B0002246314601A8FDF7CDFF002815DD9DF8F1
:1058C000303093B197F90030052B0ED018490A48B3
:1058D00009F0DAFC0CA9084809F0DFFC064809F0D9
:1058E000E3FC0CA90E4808F00CFF01A8FCF7C8FC6B
:1058F00058E700BFA98801006C030020D2750100A1
:10590000E88D0100DB750100DE750100E175010025
:105910008803002038040020DC030020D46F01003D
:10592000E4030020EE750100F98001000676010015
:10593000117601002DE9F04116491748174E184F0E
:10594000154D09F0A1FC0024A6F10F0816F8013F3F
:105950000F2B03D83946284609F09FFC052C4FF041
:1059600010020DD03178284609F0D5FC0D492846A3
:1059700009F08AFC0134E4B2062CE7D1BDE8F081DD
:1059800098F81510284609F0C6FC284609F08CFC4A
:10599000F0E700BF3E790100B80300204F0400206B
:1059A0006C880100E871010010B58AB00DF11F0389
:1059B00004930DF12503039309AB0C4602930DF1FB
:1059C000230301930DF12203009308AA0DF1210393
:1059D0000E4960680DF070FC05280BDC0C490D4881
:1059E00009F052FC61680B4809F057FC4FF4C8708D
:1059F0000AB010BD08A90848FAF737FEFFF79AFF6A
:105A00000649074809F040FCC820F1E7C5790100C4
:105A1000D97901008803002040040020EB790100BF
:105A2000B803002008B508B9002008BD037C03F0C6
:105A30000F03052BF8D1CAB20146064808F09BF9BE
:105A40000028F1D0037C03F00F03042BECD1406954
:105A5000EBE700BF8C070020F7B53C4C2678002E02
:105A60006CD13B4B93F90030012B67DD394B196842
:105A7000002963D0384A394808F085F905460028DE
:105A80005CD00146354808F06EF907B2002F55D0BA
:105A900031462846FFF7C6FF012F064650D029465B
:105AA00001222E4808F067F94569684605F07AF842
:105AB00010222B49684603F067FE2A492A4809F05C
:105AC000E3FB3146284809F0E8FB2849264809F05D
:105AD000E4FB0A222946244809F03FFC23492248D6
:105AE00009F0DBFB1E49204809F0D7FB1E4809F0EE
:105AF000DBFB40F202211E4805F0ECFAAAB2314667
:105B00001C481D4D09F0BEFA15491A4809F0BEFAA5
:105B10001A4B186818B10021FFF784FF2860296824
:105B200089B1144809F0BAFA0021124809F0BEFA06
:105B3000012313490C48237009F0A6FB03B0F0BD04
:105B400040F20225B1E70F49EBE700BF78040020DF
:105B5000DC030020340400209B7501008C0700202A
:105B600058030020A2750100B8030020E87101006D
:105B7000B80400209404002084030020E0030020E7
:105B8000B1750100BF81010010B5114C11492046CB
:105B900009F07AFB1049204609F07FFB4FF4FA70B8
:105BA0000AF0A2F9012115200AF030FB002115208E
:105BB0000AF054FB4FF4FA700AF096F9152001210F
:105BC0000AF04CFB4FF4FA70BDE810400AF08CB9B3
:105BD000B8030020D6800100F680010070B592B0B5
:105BE00002A809F001FB04A809F0FEFA06A809F0D2
:105BF000FBFA08A809F0F8FA55495648564E09F03C
:105C000043FB544809F050FB02A95448FAF721FE1F
:105C1000002877D052494F48524C10AD09F034FB60
:105C2000039B10942846119303F0D4FD04A94B481C
:105C3000FAF779FE00285DD04B49464809F024FB6D
:105C4000059B10942846119303F0C4FD06A9434810
:105C5000FAF79EFE002841D044493E4809F014FB63
:105C6000079B10942846119303F0B4FD08A93B4804
:105C7000FAF724FE10B33E49364809F005FB099BAC
:105C800011932846109403F0A5FD039B0095CDE9E0
:105C90000B34059B37480A94CDE90D34079BCDE9B9
:105CA0000F34099B11930CAA0EAB0AA904F0A4FEB1
:105CB000284809F0F9FA022333703BE0039B2D4892
:105CC0000C94CDE90D34059BCDE90F34079B11935E
:105CD0000EAA2B460CA904F0BFFEE9E7039B25485A
:105CE0000E94CDE90F342A46059B11930EA904F0BA
:105CF000DBFEDDE7039B1F4810942946119304F057
:105D0000EDFED5E71C49134809F0BEFA4FF47A625C
:105D100042F6E061174804F0E5FD68B917491848F4
:105D200009F0B2FA1749164809F0AEFAF6233370B3
:105D3000FFF72AFF12B070BD1349064809F0A4FA14
:105D400010A804F02FFF10A803F044FDB0E700BF37
:105D5000E27B0100B8030020DC03002040040020A7
:105D6000EF7B010054890100057C01000B7C0100E0
:105D7000107C010050040020177C0100237C0100EE
:105D800088030020657C0100947C010007B5104960
:105D9000104809F079FA684604F004FF684603F0F9
:105DA00019FD0D4B00930D4B68465B68019303F0A2
:105DB00011FD684604F03AFF684603F00BFD6846A3
:105DC00004F012FF684603F005FD03B05DF804FB24
:105DD000BC7B0100B8030020548901007806002034
:105DE00018B10349034809F04FBA0349FAE700BF65
:105DF000D4800100B8030020EB8D010010B5264CC3
:105E00002649204609F040FA2549204609F03CFA87
:105E1000244B1868003018BF0120FFF7E1FF22492A
:105E2000204609F031FA214B1868003018BF0120D4
:105E3000FFF7D6FF1E49204609F026FA1D4B1868C9
:105E4000003018BF0120FFF7CBFF1B49204609F0A7
:105E50001BFA1A4B1868003018BF0120FFF7C0FF6B
:105E60001749204609F010FA164B1878FFF7B8FFCB
:105E7000204609F019FA1449204609F005FA03F002
:105E800056FC0A220146204609F073FA2046BDE876
:105E9000104009F009BA00BFB8030020117B0100CF
:105EA0001E7B0100D8030020267B0100D4030020C4
:105EB0002F7B0100E0030020367B01002804002036
:105EC0003F7B0100780400209B71010010B5424C1B
:105ED0004249204609F0D8F94149204609F0D4F951
:105EE0004049204609F0D0F93F49204609F0CCF955
:105EF000204609F0D9F93D49204609F0C5F93C4949
:105F0000204609F0C1F93B49204609F0BDF93A495C
:105F1000204609F0B9F93949204609F0B5F9384960
:105F2000204609F0B1F93749204609F0ADF9364964
:105F3000204609F0A9F93549204609F0A5F9344968
:105F4000204609F0A1F93349204609F09DF932496C
:105F5000204609F099F93149204609F09EF9304967
:105F6000204609F091F92F49204609F08DF92E4974
:105F7000204609F089F92D49204609F085F92C4978
:105F8000204609F081F92B49204609F07DF92A497C
:105F9000204609F079F92949204609F075F9284980
:105FA000204609F071F92749204609F06DF9264984
:105FB000204609F069F92549204609F065F9244988
:105FC000204609F061F92046224909F05DF9204692
:105FD000BDE8104009F068B9B8030020B47C0100A6
:105FE000D67C0100E97C0100F77C0100FF7C010008
:105FF0000F7D01001B7D0100287D01003D7D01001A
:106000004C7D0100547D01005F7D0100697D010030
:10601000787D0100807D01008C7D0100F68001000B
:10602000A27D0100C17D0100D67D0100E37D01005C
:10603000F17D0100FD7D0100057E0100107E010063
:106040001D7E0100257E0100307E01003F7E0100A3
:10605000487E0100567E010008B5FFF737FFFFF7C5
:1060600095FE0349034809F00FF9C82008BD00BF99
:10607000B2760100B803002070B594B003F057FB6E
:10608000064609F0FDFE0546234808F051F90028B0
:106090003FD0224B1C7864B2002C3AD12346012217
:1060A000402104A803F0BCFB1D4904A80DF091F9A0
:1060B0001C4904A80DF08DF91B4904A80DF089F9BD
:1060C0003146684603F02AFC01236A4604A91248B7
:1060D00008F08BFB23460122402104A803F0A0FB1B
:1060E0000F4904A80DF075F90E4904A80DF071F9D7
:1060F0000E4904A80DF06DF968464FF47A71B5FBAE
:10610000F1F103F00BFC01236A4604A9024808F0F0
:106110006CFB14B070BD00BFE4030020B40300208A
:10612000B0810100537A01000C810100C881010097
:1061300010B50C4C2046FAF769FA78B90A490B48B1
:1061400009F0A2F8DE232374AD236374BE23A37485
:10615000EF23E374FE232375FF236375BDE810402E
:10616000FFF7E8BB4004002076790100B803002067
:1061700008B5002007F064FF1A491B4809F084F8AD
:106180001A491B4807F0F6FE1A491B4807F0F2FEB1
:106190001A491B4807F0EEFE1A491B4807F0EAFEB1
:1061A0001A491B4807F0E6FE1A491B4807F0E2FEB1
:1061B0001A491B4807F0DEFE1A491B4807F0DAFEB1
:1061C0001A491B4807F0D6FE1A491B4807F0D2FEB1
:1061D0001A491B4807F0CEFE1A491B48BDE8084083
:1061E00007F0C8BE437901006C030020596000002D
:1061F00047790100395500004C7901008D6D000090
:1062000051790100997000002C820100A959000009
:1062100056790100D15200005A790100A9530000BB
:106220005F79010075540000657901009D540000FC
:1062300062790100A556000069790100FD52000055
:106240006F790100295300009E7501002DE9F04F80
:10625000494F3B6887B08046002B00F08A80474C4E
:1062600025786DB2002D40F084802278444EDFF80E
:106270001C91013252B222703278013252B2327025
:10628000D9F800A009F0FCFD2B4601460B22504630
:1062900003F070FB00283AD03B68DFF8F4A0DD681B
:1062A000DFF8F0B04DB32B7C03F00F03062B22D1A7
:1062B00052462946584607F066FD98B1037C03F024
:1062C0000F03052B0ED1C368ABB119462A4603A8AC
:1062D0000193FAF769FF414603A8FBF761FE019BB2
:1062E0005B68F1E72946002203A8FAF75DFF414603
:1062F00003A8FBF755FE6D68D4E7B8F1030F03D090
:1063000009F0BEFDC9F800001E48FBF7CDFEB8F14C
:10631000030F26D01C4DD5F8008009F0B1FD0023F5
:10632000014641F28832404603F024FBA846C0B142
:106330003B68DD688DB12B7C03F00F03062B08D181
:106340002946002203A8FAF72FFF012103A8FBF733
:1063500027FE09F0EBFD6D68ECE709F091FDC8F848
:1063600000003378013B5BB233702378013B5BB2B2
:10637000237007B0BDE8F08FD4030020D1030020C4
:106380006903002030030020880400207C040020E2
:10639000AB7001008C0700200320FFF757BF0000FF
:1063A00010B5094C237801335BB2237009F0BEFDB0
:1063B0000320FFF74BFF09F0B9FD07F035FE237806
:1063C000013B5BB2237010BDB403002030B5114B0C
:1063D000196885B0D9B1104CCD682278013252B21B
:1063E000227085B12B7C03F00F03062B07D100220E
:1063F000294601A8FAF7D8FE01A8FBF729FE09F003
:1064000095FD6D68EDE72378013B5BB2237005B025
:1064100030BD00BFD4030020690300202DE9F04FF8
:10642000914C23688FB0002B00F019818F4F3B787F
:10643000002B40F014813B788D498E488E4D0133FE
:106440005BB23B7008F020FF8A4808F02DFF8B4AB2
:1064500021688B4807F097FC8A4A286021688848A1
:1064600007F091FC884B894A18602168844807F03E
:106470008AFC874B874A18602168814807F083FCB3
:10648000854B1860FFF7E8FA844A21687C4807F0DA
:106490007AFC834BA946186030B3824D2B781BBB26
:1064A000C468814802F02CFE002814BF0123002399
:1064B0002B7003D07D496F4808F0E6FE7C4B00222C
:1064C0001A608CB12B787BB1237C03F00F03062B71
:1064D00006D1206803A903F072F803A802F04CFF6C
:1064E00009F024FD6468ECE7724A00231360D9F8D0
:1064F00000309246002B00F09480D3F80C80DFF837
:10650000D8B16D4CD9F80030002B00F0AB80B8F159
:10651000000F00F0838098F8102002F00F02052A87
:10652000F2D14146564807F01EFC0128EAD94146FF
:1065300003A8FCF70BF903A8FCF77CF8A8B103A8A3
:10654000FBF710FF064680B9014603A8FBF746FF9C
:10655000051E03A8BCBF6D420126FBF79BFE9DF8FC
:106560001C20052A09D0062A32D009F0DFFC03A836
:10657000D8F80480FBF784FEC4E718B9022103A809
:10658000FBF796FE4FF4807103A8FBF7D3FE059B43
:1065900023B14FF4007103A8FBF7CCFE012128467C
:1065A00009F034FE0021284609F058FE59462046DD
:1065B00008F06AFE29460A22204608F0CEFE3F492E
:1065C000204608F061FE3E49204608F05DFECCE71B
:1065D00001900121284609F019FE019BD6B113F163
:1065E000FF3618BF01263146284609F037FE3549E7
:1065F000204608F049FE0A222946204608F0ADFE52
:106600003149204608F040FE0A223146204608F073
:10661000A4FED8E7013B5E425E41E4E7DB68CAF8CE
:1066200000302548294C08F03FFEFFF7CFFEFFF76A
:10663000E5FB274B274801221A7004F057FB20B1D5
:10664000244804F015FC0423237094F90030072B30
:1066500004BF042323703B78013B5BB23B700FB057
:10666000BDE8F08FDB68FFDE340400206903002002
:106670005E750100B8030020D80300206E7501008C
:106680008C070020187F010090040020107001008A
:10669000D403002074750100E00300207975010027
:1066A000280400202C040020A15500007C75010066
:1066B00038050020300400206C0300209475010090
:1066C0009975010098720100D7700100DC03002069
:1066D00068030020A00300208C7501002DE9F04321
:1066E0003B4C23688DB0002B6ED03A4D2E6809F0DC
:1066F000C7FB002301464FF47A72304603F03AF9A3
:10670000074610B109F0BCFB2860334DDFF8D49088
:106710002B7801335BB22B702368DE687BB2002BD1
:1067200014BF4FF004084FF002082268F2B1EEB136
:10673000337C03F00F03052BF8D13146484607F0B0
:1067400012FB0128F1D9314601A8FBF7FFFF01A890
:10675000FBF770FF18B1414601A8FDF79FFB09F058
:10676000E5FB01A87668FBF78BFDDEE72B78013BA4
:106770005BB22B70194B93F90030052B24D01FB35B
:10678000174F00263D463968F1B1EEB90B7C03F096
:106790000F03052B0CD101A8FBF7D8FF012101A89D
:1067A000FDF77CFB061C01A818BF0126FBF768FD5E
:1067B0002B684BB109F0BAFB2B685B682B60002B90
:1067C000E1D12368DB682B600DB0BDE8F08300BF2A
:1067D000D80300208404002069030020DC0300208B
:1067E000300400208C07002070B580EAE074A4EB30
:1067F000E0740E4605460121204609F007FD022EF1
:106800000CD10021204609F029FD0B490B4808F066
:106810003BFD0A48BDE8704008F046BD36B9E94383
:10682000C90F204609F01AFD0549EFE7E90F204698
:1068300009F014FD0349E9E7CA7501006C03002063
:106840009D820100A88201002DE9F0472DED048B07
:10685000754B94B01C6809F013FB0023014647F206
:106860003052204603F086F8002800F0D7806F4BA6
:106870001A68002A00F0D2806D49D4680B78DFF8DE
:10688000EC819FED6C9A01335BB20B70002C00F031
:10689000BA80237C03F00F03052B12D1002221467E
:1068A000404607F068FA4369052B0AD1214609A83A
:1068B000FBF74CFF09A8FBF7BDFE20B909A8FBF7C1
:1068C000DFFC6468E2E709A907A8FDF7E3FF09A870
:1068D000FBF758FE0021064609A8FBF77FFD054699
:1068E00007A8FDF78BFD08EE900A09A8FBF7D2FC7C
:1068F00033B207EE903AF8EEE77A824687EE898A5D
:1069000009A8FDF765F94C4981464C4808F0BCFCE4
:10691000022718EE900A0AF0B9FF009702460B46CC
:10692000CDE90401454808F0EDFD4549434808F02C
:10693000ABFC18EE100A0AF0A9FF009702460B46BE
:10694000CDE902013D4808F0DDFD3E493B4808F035
:106950009BFC51460A22394808F0FFFC5FEA164AC0
:106960004CD0082003F084F94FF6FF7381B240F653
:106970002712504602F0FEFFA8B12168324808F005
:106980008CFC3249304808F07FFC2268304931489D
:1069900007F016FFB1B209A8FBF70CFE39462846EE
:1069A000FFF722FF8AE7DFED2C7AB4EEE78AF1EEFB
:1069B00010FA04DD22682949264807F001FFB9F1E1
:1069C000000F01D10121EAE70022254BDDE9040196
:1069D0000AF0FCFDDDE902230BF040FA08B10021CA
:1069E000DDE7F4EEC88AF1EE10FAEBD91D49134841
:1069F00008F04AFC114808F057FC5FE71A490F48B5
:106A000008F042FC5AE70A4A1378013B5BB2137064
:106A100009F036FA044B1860FFF72EFB14B0BDECFA
:106A2000048BBDE8F08700BF8C040020D803002051
:106A3000690300200000C8421A7501006C030020A1
:106A400020750100427201008803002026750100B4
:106A500036750100E4030020000018424275010071
:106A60000000F03F4F7501002C7501008C070020DD
:106A70002DE9F043664E33688DB0002B00F0C580E1
:106A800064496548654CDFF8E48108F0FDFB624825
:106A900008F00AFC09F0F4F9274605462378F3B11B
:106AA00009F0EEF90023014642F21072284602F086
:106AB00061FFA0B907F0B8FA98F80030002B4FD169
:106AC000574B93F90030052B01D0FFF707FEFFF776
:106AD000BBFE0220FFF7BAFB09F028FADEE73B789D
:106AE000002B44D101274F494F4D4B4808F0CCFBB8
:106AF000494808F0D9FB2B784C4A01335BB22B7024
:106B000013689046002B3BD0DC68DFF84491002CE2
:106B100036D0237C03F00F03052BF8D121464846DD
:106B200007F021F90028F2D0237C03F00F03052B96
:106B300014D12146484607F016F978B1216801A81A
:106B4000FBF73AFE01A8FBF775FD10B101A8FBF7B2
:106B500091FB09F0EBF901A8FBF792FB6468D6E71B
:106B6000334B1B68002BABD002F0F0FBA8E7314998
:106B7000314808F089FB304808F096FB0027B2E75F
:106B80002E4B2F49244800241C6008F07DFB22482E
:106B900008F08AFB642009F0A7F92A4B2A491C70E7
:106BA0002A4B1D481C7008F06FFB02F0C0FD0A2242
:106BB0000146194808F0DDFB3168254806F0ECFC79
:106BC000244B25491C60254B13481C60244B346022
:106BD0001C60244BC8F800401C60154B1C6008F07A
:106BE00053FB02F0A4FD0A2201460B4808F0C1FB4A
:106BF000094808F059FB1C4B1C702B78013B5BB219
:106C00002B7038460DB0BDE8F0830127F9E700BFCF
:106C100034040020668001006C030020690300201A
:106C2000DC0300209E80010079040020D8030020AE
:106C3000280400207B80010088030020300400200D
:106C4000B480010078040020BC80010068030020AB
:106C50008C070020D4030020127301009004002050
:106C6000E0030020840300206A0300202C0400209D
:106C700030B5394B1D786DB289B0002D37D1374909
:106C8000374C384808F000FB364808F00DFB7222FC
:106C900001212046FAF7F6F92046FAF79DF97B28FC
:106CA00036D1314B04934FF0FF330793059506948B
:106CB000FFF7DEFE04A92D482D4D06F087FF286062
:106CC0002046FAF785F92C689CB92A492A4808F029
:106CD000DBFA294808F0E8FA284901A808F0AAFFD9
:106CE00001A92748FAF722F801A808F05EFF002062
:106CF0000CE024491B4808F0C7FA1A4808F0D4FAF7
:106D0000FFF78CFB1E48FAF7D7F8012009B030BD19
:106D10002046FAF741F998B1237D1BB1FF212046A7
:106D2000FAF76AF9154904A808F084FF04A9144881
:106D3000F9F7FCFF04A808F038FF1148FAF77AF8D1
:106D40000748FAF745F91049064808F09DFA054842
:106D500008F0AAFACBE700BF69030020717B0100AD
:106D600058040020B8030020888801008C07002008
:106D7000340400208C7B010088030020AA880100D5
:106D800040040020987B0100AB7B010008B5FFF7B1
:106D90006FFF28B9034BF6221A704FF4FA7008BD42
:106DA000C820FCE7DC0300202DE9F041C0B0002141
:106DB0001C2214A813910BF0B0FB202213A99B48AE
:106DC000F9F7F6FC78B92022994913A80CF079FB61
:106DD0009849994808F058FA13A9974808F05DFABD
:106DE000954808F061FA914D6A7D2B7C04922A7DCA
:106DF0000392EA7C0292AA7C01926A7C0092402172
:106E00008E4A1BA80CF024FA8D498B4808F03CFAF6
:106E100013A9894808F041FA1BA9874808F03DFAF0
:106E2000854808F041FA4FF47A730022CDE90F2328
:106E3000844A0E922BAC08228DF84820ADF84A30D7
:106E400013AA50230EA9204606F024F84FF47A63C3
:106E50007D497E483B9308F017FA02F068FC0A224D
:106E600001467A4808F085FA784808F01DFA20466D
:106E700006F03FF81BA9204606F062F97449064661
:106E80000AA808F0D7FE294607A8F9F70BFF079ACA
:106E90000A99204606F032F807A808F086FE0AA8EC
:106EA00008F083FE204606F048F9002E40F0B68038
:106EB000204606F053F9DFF8DC810646204606F04E
:106EC000BFFA074600B3214607A806F0BDF94146C0
:106ED0000AA808F0AFFE0AA907A808F054FF074661
:106EE0000AA808F062FE07A808F05FFE002FE5D0B0
:106EF00021460AA806F0C2F90AA92846F9F716FFA2
:106F00000AA808F052FED9E752494B4808F0BCF9EC
:106F10000A223146484808F020FA474808F0C4F9E8
:106F2000C82E6FD14C4B4D490A9348480C944FF0F2
:106F3000FF330D930B9708F0A7F902F0F8FB0A2234
:106F400001464248464D08F014FA404808F0ACF9B2
:106F5000FFF78EFD43493D4808F096F93B4808F09D
:106F6000A3F93E49394808F08FF902F0E0FB0A2204
:106F70000146364808F0FDF9344808F095F90AA9A9
:106F8000394806F023FE2860204605F0A7FF2C684C
:106F9000C4B93649364808F077F9364907A808F0E9
:106FA00049FE07A92148F9F7C1FE07A808F0FDFD31
:106FB0002646314B2B933DA808F0F7FD304640B0F4
:106FC000BDE8F0812D49214808F05EF902F0AFFBE1
:106FD0000A2201461D4808F0CCF91C4808F064F963
:106FE000FFF71CFA2649144808F04EF9254B1B7888
:106FF000002BDED00D48F9F7EAFD0028D9D0FEF7C6
:1070000061FAD6E7B6F5987F0CBF1F491F491848AB
:1070100008F03AF9204605F061FFCAE71C49144818
:1070200008F032F94FF0FF36C3E700BF40040020FC
:1070300031810100F4790100B8030020127A0100C7
:10704000417A0100E8860100557A01006C030020B6
:107050006B7A01007E7A010088880100C67A0100FF
:1070600034040020917A01008C070020A77A0100E7
:1070700088030020AA880100F4870100BE7A01007D
:10708000CC7A010068030020D37A0100E77A01007E
:10709000017B0100797A0100012838B50C4630DD0A
:1070A0004D682F4928460CF076F928B901212D4862
:1070B000F9F7B3FDC82038BD2B4928460CF06BF911
:1070C00001460028F3D02949294808F0DDF8254871
:1070D000F9F799FD0A220146254808F03EF92448AF
:1070E00008F0E2F861681F48F9F788FB61682048FA
:1070F00008F0D3F81F491E4808F0C6F81C4808F0ED
:10710000D3F81D4C94F90030012B1FDDFFF74CFE26
:10711000C82802D104232370CDE7431C10D117499E
:10712000174808F0B1F8164808F0BEF8154B164895
:1071300000221A700323237003F09AFEC920BAE7D5
:10714000124B1B78002BE5D10F23E4E710491148BF
:1071500008F09AF80F4808F0A7F84FF4FA70AAE779
:107160006B810100400400206E8101004C7601001B
:10717000B80300206C760100DC0300207376010068
:107180006C0300206A030020A00300206803002095
:107190008E760100880300202DE9F3470024314D4D
:1071A00000942246214623462F48304FDFF8FCA0AA
:1071B00008F022F828464FF47A762D4B6C60AE60CA
:1071C00040F8143B4FF0080808F00EF885F82080CE
:1071D0002946284D0122384607F03CFF4FF00109AF
:1071E00000943B4629460722234802F07BF93B46A0
:1071F0002946CDF800900322204802F073F900944C
:107200003B4606221E4F1F4829461F4D02F06AF9D1
:107210004FF48053C5E901462B611C491C4B2B6080
:10722000381D08F007FD3D601A4D1B49524638468F
:1072300009F0D4F8C5E90146184C194B19482B60E0
:10724000494685F810806E8202F0FEF829462046F5
:1072500007F0FAFB14495246204602B0BDE8F04759
:1072600009F0BCB8B80400205003002094040020AA
:1072700044870100E80700206C03002088030020F9
:1072800040040020B803002058040020AA88010010
:107290001C700100A003002019530000E40300202B
:1072A000E8860100380400209DE000000000002076
:1072B0002DE9F0470024C8B03C22214609A80894D3
:1072C0000BF02BF97C22214629A828940BF025F9F4
:1072D00023460122402108A802F0A2FAAF49B04E8D
:1072E000B04F08A80CF075F87F22AF4928A80CF021
:1072F000E8F8012328AA08A9AC4807F076FA234643
:107300000122402108A802F08BFAA94908A80CF034
:1073100060F87F22A74928A80CF0D3F8A64928A82E
:107320000CF057F8012328AA08A9A04807F05DFA35
:1073300023460122402108A802F072FA9F4908A8BA
:107340000CF047F87F229E4928A80CF0BAF80123D8
:1073500028AA08A9954807F048FA234601224021A7
:1073600008A802F05DFA974908A80CF032F87F22CD
:10737000954928A80CF0A5F8012328AA08A98B484C
:1073800007F033FA33783D6801335BB23370002D78
:1073900000F03B818D4BDFF86092B3F80080ADF8D0
:1073A00000801E2221460DF102000BF0B6F83E22AD
:1073B00021460DF16200ADF86080DFF840A2DFF8F1
:1073C00040820BF0AAF8ED683B68002B00F0AE801D
:1073D000002D00F0AB802B7C03F00F03052B40F059
:1073E0008E802946404606F0BEFC002800F08780CB
:1073F00028680CF038F8013404440022294640463D
:1074000006F0B9FC4369112B12D8DFE803F07C8742
:10741000877C7C097C7C7C7C1111111111111187F6
:107420001F226B4968460CF04CF800238DF8603041
:1074300000230122402108A802F0F2F93F22296826
:1074400008A80CF018F8494608A80BF0C2FF5146EE
:1074500008A80BF0BEFF01235E4A544808A907F0B4
:1074600029FA00230122402108A802F0D9F93F227D
:10747000296808A80BF0FFFF494608A80BF0A9FFF0
:10748000554908A80BF0A5FF0123544A474808A90D
:1074900007F010FA00230122402108A802F0C0F9E9
:1074A0003F22296808A80BF0E6FF4D4908A80BF019
:1074B00090FF514608A80BF08CFF01236A4608A9EB
:1074C0003A4807F092F99DF86030C3B100230122D9
:1074D000402108A802F0A4F93F22296808A80BF06F
:1074E000CAFF3F4908A80BF074FF3B4908A80BF0FE
:1074F00070FF012318AA08A92C4807F076F908F0B4
:1075000015FD6D6860E71F22364968460BF0D9FF0C
:1075100035493F2218A80BF0D4FF89E71F223349D1
:1075200068460BF0CEFF3F223149F3E700230122EA
:10753000402108A802F074F92E49DFF8C4901B4DD1
:1075400008A80BF046FF0123621E08A9174807F0A0
:10755000C6F93B68DC683B68002B53D0002C51D047
:10756000237C03F00F03052B14D12146484606F077
:10757000FAFB78B1D4F8008040460BF074FF414626
:107580000246284606F07BFD63681BB12C21284685
:1075900006F068FD08F0CAFC6468DCE7A981010018
:1075A00069030020D8030020A3810100E403002028
:1075B00083810100E2810100CF810100B0810100DF
:1075C0001B8101009581010015810100D674010025
:1075D0008F8101007E810100B78101003D810100A2
:1075E00046760100768101002B810100898101002E
:1075F000728101009C81010040760100028101003E
:107600008C070020044806F022FE3378013B5BB271
:10761000337048B0BDE8F087E40300202DE9F04F57
:10762000A7B0002397488DF81330CDE90533CDE995
:10763000073306F07DFE944F054610B105233B70DD
:10764000FAE0924C216841B99149924807F01CFE3A
:10765000904807F029FE0F23F1E78F4806F083FBDF
:107660000FFA80F8B8F1010FEEDD294620688B4E45
:10767000FEF7D8F9002800F0E28030608849894898
:1076800007F002FE3168874807F007FE854807F0DB
:107690000BFE01212068FEF7C5F9B8F1020F824602
:1076A00000F0D080022221687B4806F064FBB8F12C
:1076B000030FD0F8149000F0C78003212068FEF774
:1076C000B1F90546102205A97748F8F7F5FF00281B
:1076D00040F0BD80B8F1040F40F3B9800421206868
:1076E000FEF7A0F9714904466E4807F0CDFD6D48DC
:1076F00007F0DAFD1FFA89F25146624807F084F973
:107700000DF124086A495F4807F081F90DF1340B47
:107710001022684940460BF0D4FE002301222021AC
:10772000584602F07DF8644958460BF052FE634912
:107730005C4807F0A9FD51465A4807F0AEFD604984
:10774000584807F0A1FD0A224946564807F005FEB1
:107750005C49544807F098FD2946524807F09DFDC2
:107760005949504807F090FD2B780BB91C461D462F
:10777000CDF80C804FF002094FF001082A46CDE900
:107780000198CDF800B0234631683E484F4D06F0D1
:10779000E5FE00285DD04E4B4E49424800241C7047
:1077A00007F072FD31683F4807F077FD3D4807F06C
:1077B0007BFD494B032283F800804121234615A815
:1077C00002F02EF8454915A80BF003FE15A92D4827
:1077D00007F0E8F823464A46412115A802F020F8B0
:1077E0003F4915A80BF0F5FD15A93E4807F06CFDC3
:1077F00015A9244807F0D6F842462346412115A88A
:1078000002F00EF8364915A80BF0E3FD15A936482D
:1078100007F05AFD15A91B4807F0C4F8FFF748FD0B
:1078200005233B7008F02CFB304928601D4807F009
:107830002BFD1C4807F038FD27B0BDE8F08F2C4B1E
:1078400033601BE740F25B790DF113053AE705ACB5
:1078500050E728490F4807F017FD0A4807F0D9F804
:107860000A2201460B4807F078FD2349094807F032
:107870000BFD084807F018FD08F002FB0C232860F8
:10788000DDE600BFE4030020DC030020E00300206D
:10789000647E0100880300208C0700208403002000
:1078A0009A7E0100B803002040040020A77E01005A
:1078B0002D5700005E810100A9810100C77E0100F3
:1078C000E8710100E77E010099800100800400203A
:1078D00024040020EE7E01006A030020FC7E0100EB
:1078E000547001006C030020E8070020027F0100B3
:1078F000BF8101001F7F01002B7F010030B5A14C2B
:1079000094F900300B3393B01A2B2BD8DFE813F027
:10791000EC00DC002A002A002A002A002A002A00A3
:107920002A002A002A001B00420045004E008C005D
:10793000A900CC002A002A002A002A002A00FC0004
:1079400009011E011801904B90481B78002B14BFB1
:107950000921012101F079FD03F0D6F8022801D0B8
:10796000FEF73CF994F90030012B40F33C8103F021
:10797000D5F8054603F0C8F8022800F02B81681EF0
:10798000042800F23081DFE810F0320134014201B6
:107990004401250102232370E4E77D4D2B781BB9B8
:1079A000FEF75AF801232B700323F4E7764D77484E
:1079B0002B78002B14BF0B21032101F046FD754BE2
:1079C0001B78002B40F027817348F9F71CF9E8B1C8
:1079D000724B1B78C3B9FFF7E7F9C82801D104231C
:1079E000D9E72B783BB16E496E4807F04DFC6D48E6
:1079F00007F05AFCF3E701A803F0D4F8029B002B30
:107A000000F0BE800F23C6E76749EDE72B784BB146
:107A1000042366496348237007F036FC614807F089
:107A200043FC9FE70F23F4E7574B58481B78002B84
:107A300014BF0B21032101F008FD5D4B196841B90A
:107A40005C49584807F020FC564807F02DFC0723F6
:107A5000A1E7594806F087F90128F1D9FFF7DEFDC3
:107A600080E7564B1D6808F00BFA002301464FF4DF
:107A7000FA52284601F07EFF00283FF473AF00233E
:107A80000322412101A801F0CBFE4D4901A80BF0D2
:107A9000A0FC01A94B4806F088FF06234A4941484B
:107AA000237007F0F1FB5DE7374B38481B78002B5C
:107AB00014BF0A21022101F0C8FC424806F038FC3C
:107AC00000287FF44FAF8AE708F0DAF93B4B1860E3
:107AD000F52323702C4B2D481B78002B14BF092154
:107AE000012101F0B2FC3DE7344B1D6808F0C8F9F4
:107AF0000023014641F28832284601F03BFF00286E
:107B00003FF430AF002346E72E4806F011FC10B1D9
:107B10002C4806F0DAFB08F0B3F9284B18600D2367
:107B200039E7264B1D6808F0ABF90023014642F205
:107B30001072284601F01EFF00287FF450AF11E7B5
:107B400008F09EF91D4B18600E2324E71B4B1D689F
:107B500008F096F90023014641F28832284601F0E8
:107B600009FF00283FF4FEAE1849194807F08CFBC6
:107B7000174807F099FBFFF77BF800287FF42FAF39
:107B8000F62308E7DC030020680300203804002007
:107B9000D003002069030020400400206A03002075
:107BA000457F0100B80300206C7F01007C7F01004D
:107BB000E0030020B67F01008C0700208004002035
:107BC000FC7E0100E4030020C97F0100E07F01008A
:107BD0006C0300201149124807F056FB104807F0CB
:107BE00063FBF623237094F9000013B030BD0D49F8
:107BF000F1E70D490D4807F047FB01A802F0D2FF5D
:107C000001A801F0E7FD094807F04EFBEBE7084942
:107C1000E1E70849EEE70320E7E700BFFD7F010049
:107C200088030020068001001A800100B8030020AC
:107C3000378001004A80010008B5164801F007FCB2
:107C400008F074F906F0F0F9FFF758FE022802DD9B
:107C5000114806F095FC08F069F9104B1B7823B128
:107C60000F4B1B680BB101F071FB0E4B1B6853B13E
:107C70000D4B93F90030052B01D0FEF72FFD08F0D6
:107C800055F9FEF7E1FD08F051F90220BDE8084082
:107C9000FEF7DCBA38040020E40300202C040020A6
:107CA00028040020D8030020DC03002008B5194870
:107CB0004FF4E13107F000FE1748F8F77FFC30B9C8
:107CC0001649144807F0F6FA1348F9F76DF8124808
:107CD000F8F7D8FF124B18700F48F8F7DBFF114B7D
:107CE0001870FEF745FAFEF7F1F8FEF721FA1420B6
:107CF00008F0FAF80C4801F08FFB0C490C4806F02C
:107D000086FE4FF4FA7008F0EFF8BDE80840FEF781
:107D1000AFBF00BFE807002040040020F674010058
:107D20000500002006000020996300002D57000088
:107D3000E403002007B5002300931A4619460348C0
:107D400007F05AFA03B05DF804FB00BFDC04002022
:107D500007B5002300931A461946034807F04CFA6A
:107D600003B05DF804FB00BFE4040020012070476D
:107D7000014B1868704700BFF404002003207047CF
:107D80007047000010B504460B490C4807F09CFAF8
:107D9000A17C94F9080008F061FAA17C94F909002B
:107DA00008F05CFA60680021FAF704FC044B00223A
:107DB0001A60012010BD00BF308201006C0300205A
:107DC000F404002073B56E460546304686E806008A
:107DD000FCF70EFD04463046FCF7A4FA10B1002C67
:107DE00008BF01244FF400516868FAF7A3FA012C88
:107DF0001BD0022C04D0FCB91C491D4807F044FAE2
:107E00003046FCF7A0FA70B36868FAF7BBFB18B904
:107E10000124204602B070BD00206C6801F028FFEC
:107E200001462046FAF7C6FBF2E73046FCF72AFC8B
:107E300001280AD0022808D00E490D4807F024FA7C
:107E40000B4807F031FA0024E3E76868FAF79AFB79
:107E50000028DDD000206D6801F00AFF01462846A9
:107E6000FAF7A8FBD5E70446D3E700BFEC81010091
:107E70006C030020FD81010010B5044608F070F885
:107E8000204610BD2DE9F043012985B0044600F0DD
:107E9000B8804FF400514068FAF734FA002800F037
:107EA000B0804FF480416068FAF72CFA68B98E4DC3
:107EB00095F90030002B00F0A4804FF480416068F9
:107EC000FAF738FA2B78013B2B706068FAF75AFB07
:107ED00000221146814602A8FCF7A6F84FF4007272
:107EE000616802A8FCF792FC002102A8FCF75EFB87
:107EF00080466068FAF7CEF9022801D0052801D142
:107F00004FF0000894F90A00A0F10E03DBB2072B32
:107F100000F2CF8008F084F8FF25E289218A0095DD
:107F20000023074607F037FE061EC0F2BE80AE42B1
:107F300000F3BD80B9F1000F40F0C180A8EB060549
:107F400007E06A496A4807F09FF9694807F0ACF909
:107F500000256849664807F097F90A2294F90A1043
:107F6000634807F0FAF96449614807F08DF90A227D
:107F700039465F4807F0F1F960495D4807F084F938
:107F80000A2231465A4807F0E8F95D49584807F097
:107F90007BF90A224146564807F0DFF9594954480F
:107FA00007F072F90A222946514807F0D6F95048DD
:107FB00007F07AF915F10A0F2CDA94F90900A17C7F
:107FC00008F04CF96068FAF7DDFA30B9666801F03C
:107FD0004FFE01463046FAF7EDFAA37C6842A3B1A2
:107FE00000210091FF23192207F0D5FDFF2801464B
:107FF000A8BFFF21462994F90800B8BF462108F020
:10800000B3F8002005B0BDE8F083FF2200921946C6
:108010001922E9E70A2D27DD94F90800A17C08F070
:108020001DF96068FAF7AEFA30B9666801F020FE13
:1080300001463046FAF7BEFAA37C83B100210091D5
:10804000FF233322284607F0A6FDFF280146A8BFDC
:10805000FF214629B8BF462194F90900CFE7FF2246
:10806000009219463322EDE72749214807F02CF901
:10807000A17C94F9080008F0F1F8A17C94F90900BA
:1080800008F0ECF800216068FAF794FA4FF4005118
:108090006068FAF78DF94FF480416068FAF788F963
:1080A000114A137801331370ABE7002642E72E46DE
:1080B00040E74FF0FF37B9F1000F0FD03E4607F011
:1080C000DFFE00230146B4F90C20484601F052FCC3
:1080D00000287FF436AF731C7FF430AFA8F17F0522
:1080E0004FF0FF3635E700BF040000200982010091
:1080F0006C030020178201001B820100537A0100EB
:10810000567001002182010029820100002110B572
:10811000044681744068FAF761F943B2002BBBBF93
:108120004042207223720123B8BFA374237A60688F
:10813000013B182B84BF202323720121FAF74EF94B
:1081400043B2002BBBBF4042607263720123B8BFD1
:10815000A374637A6068013B182B84BF2123637288
:108160000221FAF73BF9C3B2192B8ABF0023A07290
:10817000A37203216068FAF731F980B2431EB3F5A8
:10818000806F26BF0023E381E08104216068FAF755
:1081900025F980B2B0F5806F8ABF4FF480632082EA
:1081A000238205216068FAF719F900B20028D6BFCA
:1081B00042F21073A081A38110BD000010B50446E7
:1081C000F8F702F92046FFF7A1FF1849184807F011
:1081D0007BF894F90800012108F018F894F90900D7
:1081E000012108F013F8A17C94F9080008F036F892
:1081F000A17C94F9090008F031F894F90A000021F3
:1082000008F004F860680021FAF7D4F960684FF4C8
:108210000051FAF7CDF860684FF48041FAF7C8F8DA
:10822000044B01201860044B187010BD3E82010001
:108230006C030020F40400200400002007B5002394
:1082400000931A461946034806F0D6FF03B05DF8BE
:1082500004FB00BFEC04002001207047014B1868AC
:10826000704700BF000500200020704703207047C2
:1082700070470000F8B50446F8F7A6F8A468002C8B
:108280003CD0E468224E234D234F64B3236843B3AC
:108290001B7833B332462146284605F074FD30B9C9
:1082A0004FF0FF3332462146284605F0B0FD3A46EE
:1082B0002146284605F067FD30B94FF0FF333A46B6
:1082C0002146284605F0A3FD144A2146284605F01C
:1082D0005AFD30B94FF0FF33104A2146284605F0C9
:1082E00096FD6468D1E70E490E4806F0CDFF0D48B3
:1082F00006F0DAFF0C4B01201860F8BD0B49094865
:1083000006F0C2FF074806F0CFFF2046F5E700BFA2
:10831000FF8201008C07002005820100138201000A
:10832000038301006C03002000050020128301007C
:1083300010B5064C0649204606F0A6FF204606F07A
:10834000B3FF044B00221A60012010BD6C03002013
:10835000ED820100000500202DE9F04F91B008AC3E
:108360008046204684E806000693FCF741FA8346DF
:108370002046FBF7D7FF20B1BBF1000F08BF4FF03D
:10838000010B2046FBF7CEFF90B12046FCF730FAF8
:1083900007280DD12046FCF775F9112869D012285D
:1083A00069D0102804D1FF2221460EA8FCF779F9E4
:1083B000D8F80850002D00F04B814FF00009EC6810
:1083C000CDF80C90CA464D46CDF80890002C00F030
:1083D000DA80A14AA148214605F0D5FCA04A2146F1
:1083E00006469E4805F0CFFC9E4A074621469B481C
:1083F00005F0C9FC0590002E00F08780002F00F0EA
:108400008480337C03F00F03022B7ED13B7C03F08E
:108410000F03022B79D1944A9048214605F0B3FC12
:1084200043690493069B002B5AD0194620680AF032
:10843000ECFF002854D108A8FBF774FF00BBBBF188
:10844000070F6CD008AA10460792FBF77CFF079A2B
:10845000002839D0104600210792FCF7A7F8706178
:10846000FDF742F9079A78B3236800934FF400733D
:1084700025E0802298E70A212046FCF759F897E783
:1084800008A8FCF7FFF8786108A8FCF7FBF80128BA
:108490003DD0022841D07B69012B08D17369132B91
:1084A00005DC1E22726108A90EA8FCF7FAF8FDF798
:1084B0001BF948B12368009308AA4FF4407306CA19
:1084C000D8F80400FAF7EAF9059B4BB10023CDE98F
:1084D000003308AB0CCB4FF0FF31059801F064FA84
:1084E0007B69022B0FD001330DD07369049A029976
:1084F0004B4502FB03F21144C4BF9946049B029111
:10850000C4BF92460393049B1D4464685EE772698E
:1085100008A90EA8FCF7C5F8BDE70022F8E708A8EF
:10852000FBF711FF00288DD008A8FBF747FF7B69F8
:10853000A8B1022B01D001330CD14C494C4806F0B4
:10854000ACFE4B4806F0B0FE01227A6108A90EA8E5
:10855000FCF747F908A8FBF731FF7061A7E7022B8A
:108560000ED001330CD04349414806F096FE4048F6
:1085700006F09AFE02227A6108A90EA8FCF731F9EA
:108580000023736193E7002D62D03B493848029B7A
:1085900093FBF5F706F078FE0A222946344806F0E8
:1085A000DCFE3649324806F06FFEFF25029B30485C
:1085B00093FBF5F10A2206F0D0FE31492C4806F073
:1085C00063FE0A2239462A4806F0C7FE2D4928488C
:1085D00006F05AFE9AFBF5F10A22254806F0BDFE88
:1085E0002949234806F050FE0A220399204806F044
:1085F000B4FE26491E4806F047FE1D4806F054FE0C
:10860000234AD8F80810154805F0BDFB0EAE814688
:10861000224621460AA8FBF707FD3A460AA930463A
:10862000FCF73FF80CAD002F14BF012202223146A7
:108630002846FCF7D6F8CDE900444FF0FF3195E825
:108640000C00484601F0B0F9D8F8083013BB0125FA
:10865000284611B0BDE8F08FFF8201008C07002092
:10866000058201009082010094820100968201003F
:108670006C030020A1820100AD820100B6820100DE
:10868000C1820100C8820100D6820100DD820100A2
:10869000AA880100DD68434FDFF824B1002DD6D051
:1086A000414A2946384605F06EFB5A464469294638
:1086B000384605F068FB3D4A80462946384605F0B5
:1086C00062FB3B4A81462946384605F05CFBB8F11F
:1086D000000F60D0B9F1000F5DD000285BD098F892
:1086E000102002F00F02022A55D199F8102002F052
:1086F0000F02022A4FD1027C02F00F02022A4AD155
:10870000002C48D04269022A47D0013245D0BAF144
:10871000000F44D0D9F814302968264803FB04F927
:10872000039BC9EB092292FBF4F45C4306F0B5FD10
:1087300094FBFAF420491F4806F0AFFD0A22FF21FE
:108740001C4899FBF1F106F008FE1C49194806F097
:108750009BFD0A222146174806F0DDFD154806F06C
:10876000A3FDD8F81430A34215D0002211460AA860
:10877000FBF75AFC22460AA93046FBF792FF00237A
:10878000CDE900334FF0FF3196E80C00284601F0A8
:108790000BF9C8F814406D6880E70024E1E75446FF
:1087A000DFE700BF8C07002094820100FF820100F8
:1087B000058201006C030020E1820100E7820100D4
:1087C0001382010010B5044607F0CAFB204610BD15
:1087D0000023836043683BB15B682BB11A7C02F0D5
:1087E0000F02062A08BF83607047000007B5002308
:1087F00000931A461946034806F0FEFC03B05DF8E4
:1088000004FB00BFF8040020014B1868704700BF4C
:108810000C05002043687BB1B0F90A20042A05D07A
:10882000052A05D0032A05D1022070470120704790
:1088300011207047187C7047184670477047000039
:1088400010B504461E491F4806F01EFD0A22B4F961
:1088500008101C4806F081FD1B491A4806F014FD5B
:10886000184806F021FD236820465B6B98470128D5
:1088700005D002280AD00021B4F9080019E003212C
:108880002046F7F775FE002107F0C0FC00212046C6
:10889000F7F76EFE002107F0B9FC01212046F7F73B
:1088A00067FE002107F0B2FC02212046F7F760FEC8
:1088B000002107F0ABFC054B00221A60012010BD1F
:1088C000708301006C0300207A8301000C050020F6
:1088D0002DE9F041044688B040689DF8383002AE7A
:1088E00086E8060000286ED0B4F90820002A69D076
:1088F000002B6BD00021F9F771FD236880465B6B7C
:108900002046984705B2022D51D0032D2BD0012DC2
:108910000CBF05210121002204A8FBF785FB4FF0C5
:10892000FF33009396E80C0004A906A8FCF744F96D
:10893000012D3ED0022D38D19DF81610B4F9080053
:1089400007F012FC01212046F7F712FE9DF81510E2
:1089500007F00AFC02212046F7F70AFE9DF81410E2
:1089600007F002FC21E04FEAD8713046B4F90870F4
:10897000FBF71CFE01460546384607F0F5FB144997
:10898000144806F081FC0A22B4F90810114806F0D8
:10899000E4FC11490F4806F077FC0A2229460D48ED
:1089A00006F0DBFC0B4806F07FFC01200BE0042105
:1089B000B1E703212046F7F7DBFD9DF8171007F01C
:1089C000D3FBB9E7104608B0BDE8F0811846FAE7D6
:1089D000987201006C030020D770010010B50446A6
:1089E00007F0BEFA204610BD38B50446F7F7ECFC98
:1089F0002249234806F048FC0A22B4F9081020480E
:108A000006F0ABFC1F491E4806F03EFC1C4806F071
:108A10004BFC606870B3B4F9083063BB2368204630
:108A20005B6B98470128054605D002280AD0012132
:108A3000B4F9080019E003212046F7F799FD29460B
:108A400007F0E4FB00212046F7F792FD012107F033
:108A5000DDFB01212046F7F78BFD012107F0D6FB56
:108A600002212046F7F784FD012107F0CFFB064BDA
:108A70000120186038BD0020FCE700BF70830100B2
:108A80006C0300208E8401000C05002007B5002334
:108A900000931A461946034806F0AEFB03B05DF892
:108AA00004FB00BF04050020014B1868704700BF9D
:108AB00018050020032070477047000010B50446D9
:108AC000F7F782FC1849194806F0DEFB0A22B4F9D0
:108AD0000810164806F041FC1549144806F0D4FB6E
:108AE000124806F0E1FB0121B4F9080007F08EFB03
:108AF000B4F90800A17A07F0B1FB606810B1002159
:108B0000F9F758FD0B4B606801221A60FBF760F81B
:108B1000002807DD0020646801F0AAF8014620461D
:108B2000F9F748FD012010BDFE8301006C03002011
:108B30008E8401001805002038B50E4C0E490546FC
:108B4000204606F0A1FB0A22B5F90810204606F0DF
:108B500004FC0A49204606F097FB204606F0A4FBD9
:108B6000B5F90800002107F051FB054B00221A60FF
:108B7000012038BD6C030020FE8301007A830100D0
:108B80001805002010B5044607F0EAF9204610BD8C
:108B9000002110B5044681724068F0B1F9F71EFC5F
:108BA00003B2002BBBBF4042208123810123B8BF09
:108BB000A37223896068013B182B84BF2023238183
:108BC0000121F9F72BFC08F061FE0022054B08F0AB
:108BD000B5FE09F08BF908B1E06010BD41F28833B1
:108BE000E360FAE700408F4030B5044687B00023C9
:108BF0002F22CDE90023ADF80830B0F90800A37AA0
:108C00000D4600295DD083F0010107F027FBE368E2
:108C1000B3F57A7F53D33149314806F035FB0A2248
:108C2000B4F908102E4806F098FB2E492C4806F09F
:108C30002BFB0A2229462A4806F08FFB284806F01B
:108C400033FB294968460AF0C4FB6068F9F722FB48
:108C5000002D3ED00D2838D00E2834D00B2836D128
:108C6000224903A80AF0DBFB21491D4806F00CFB52
:108C700063681968236809685D6A03AA6B46204621
:108C8000A8470A220146164806F067FB194914480E
:108C900006F0FAFA636812481B68196806F0FDFAD4
:108CA00069460F4806F0F9FA13490D4806F0ECFA48
:108CB00003A90B4806F0F1FA094806F0F5FA07B0E7
:108CC00030BD1946A1E70D49CBE70D49C9E70D496C
:108CD000C7E702280CBF0C490C49C2E70A8401000F
:108CE0006C03002012730100D5830100E3830100AF
:108CF0000F840100E87101001B840100DC83010086
:108D0000C8830100EB830100CC830100D083010004
:108D10000129F7B5044644D04368002B41D0002216
:108D200011466846FBF780F94FF4007261686846A7
:108D3000FBF76CFD00216846FBF738FC05466846EA
:108D4000FBF7A0FC6068F9F71DFC064607F098F8F1
:108D5000E268FF216A430023B2FBF1F2014630468C
:108D600000F008FE0746E6B107F08AF80023014646
:108D7000E268304600F0FEFD064620B3002066683B
:108D800000F076FF01463046F9F714FC4DB1207A29
:108D900000F078FFA37A834203D101212046FFF738
:108DA00023FF002003B0F0BD9FB131462046FFF7FE
:108DB0001BFF6068FAF70CFF01460028F1D16068DC
:108DC000F9F7F8FBEDE7207A00F05CFFA37A834225
:108DD000EAD1002DE5D0207A00F054FFA37A834237
:108DE000DFD1002FDDD1D8E7F7B56D4685E8060065
:108DF00004463F493F489DF820601F4606F044FA6C
:108E00002846FBF75FFE2FB13B4938460AF0FDFAD2
:108E1000002844D06068002841D02846FBF782FA39
:108E200000283ED12846FBF7E3FC012839D011D3B6
:108E300002280ED0044631492E4806F025FA0A22AF
:108E400021462C4806F089FA2A4806F02DFA00201F
:108E500025E08EB100212846FBF7A8FB00283DD075
:108E60006068F9F78FFBC8B9646800F001FF01463C
:108E70002046F9F79FFB11E06068F9F70BFA0E281E
:108E80000CD8012303FA00F045F60243184205D03E
:108E900031462846FBF78AFB0028E1D1012003B0C8
:108EA000F0BD2846FBF7EEFB022817D012D80128A8
:108EB000D6D013490F4806F0E7F92846FBF7E2FB46
:108EC0000A2201460B4806F061FA0A4806F0ECF95E
:108ED0000124B0E70A380428EBD8C1E76068002114
:108EE000F9F768FB00212046FFF77EFED6E700BFBA
:108EF000F38301006C030020D58301006A6F010039
:108F00005D6F010007B5002300931A461946034818
:108F100006F072F903B05DF804FB00BF10050020F5
:108F20000139C9B2FF2906D0435C0139C9B2002B0F
:108F3000F8D0002070470120704700002DE9F04F65
:108F400085B006F09DFF634B029018689A4608B101
:108F500001F0F2F8604C614F2568386800210BB2CF
:108F6000AB4201F10101C0F29D805D4DDFF88C91B3
:108F7000DAF80000002800F09C8021682B6803EBE1
:108F8000C10101F061FA002840F393802368132B9C
:108F900000F38F8006F074FF0023014641F288320F
:108FA000029800F0E7FC0646002840F082802B681B
:108FB0002068072103EBC00001F0AEF82B68019395
:108FC000019A236802EBC30B9BF807208242CFD1A2
:108FD0000FFA86F84345039325DD019B082203EB36
:108FE000C800594609F066FA0136039B0028EFD104
:108FF0003968019031F818303A4843F0010321F8FC
:109000001830394906F040F92B682068019A03EBC3
:10901000C000082100F082FA3449324806F04AF9CB
:10902000B8F1000FA4DAD9F80030002BA0D02268E4
:109030002868082100EBC200FFF772FF06460028EF
:1090400096D13B682748012123F81210284906F0E1
:109050001BF90A222168234806F07FF92549214897
:1090600006F012F92B682068324603EBC000082195
:1090700000F054FA1B4806F017F922682B6803EB3E
:10908000C20113F83230282B08D10C22D9F8000085
:1090900001F0FBFADAF8000001F020F9236801334F
:1090A000236065E730F8132022F0010220F8132036
:1090B00055E711490B4806F0E7F80A2221680948EC
:1090C00006F04BF9074806F0EFF8012005B0BDE8BF
:1090D000F08F00BF24050020380500204005002047
:1090E0003C0500206C03002021850100288501003B
:1090F0002F85010034850100128501003005002014
:10910000F8B5424D2B6807460BB1012054E04049A9
:109110004048414E06F0B8F83E4806F0C5F83F49D1
:109120003C4806F0B1F800F002FB0A22014639483B
:1091300006F01FF9374806F0B7F8142006F00CFFC8
:10914000044600F0B3FFA0202C6006F007FF34496E
:1091500030603048334C06F097F800F0E8FA0A2205
:1091600001462C4806F005F92A4806F09DF828200B
:1091700006F0F4FE2C492060264806F085F800F041
:10918000D6FA0A220146234806F0F3F8214806F0F1
:109190008BF833680BB123687BB92449244806F067
:1091A00073F800F0C4FA0A220146214806F0E1F8FB
:1091B0001F4806F079F80020F8BD1E4B1E481F60BE
:1091C00000F0DAFD286800F08BFF0446B8B11B49B7
:1091D000104806F06FF8286801F0BEF8286800F023
:1091E0008BFF17490B4806F065F8286801F0F8F87E
:1091F00000288AD01349074806F05CF885E7124931
:10920000044806F057F82046D6E700BF24050020A2
:10921000738401006C0300203C050020C67A010025
:109220009484010040050020A0840100AD84010069
:109230008803002028050020B0050020C584010017
:10924000D8840100F8840100048501002DE9F04173
:10925000364E306800F03CFF02280DD134493548C5
:1092600006F012F8334806F01FF8306801F0B8F83D
:1092700042F21070BDE8F0812F4C304F2568EDB9F7
:109280001C2006F069FE31682D4E804601F060F921
:109290004046C4F8008001F03BFA3A6820682BB2DF
:1092A000934205F1010506DA31680C2201EBC30196
:1092B00001F0EBF9F1E7002101F068FA214E3A687C
:1092C000B6F900309342374606DBFFF737FE00233E
:1092D00033804FF4FA50CDE7194D286800EBC301F5
:1092E00010F8330028281AD1206801F0DFFA164B55
:1092F0001B6802462BB1B6F90000296801EBC001DA
:1093000098472B68B7F90010206803EBC10101F002
:1093100073FA3B8801333B8040F6C410AAE701335F
:109320004FF4FA60338090FBF2F0A3E724050020AD
:10933000648401006C030020300500203805002003
:109340003C050020340500202805002038B5094CD4
:10935000256806F095FD0023014641F28832284633
:1093600000F008FB20B1FFF771FF06F089FD2060D7
:1093700038BD00BF2C0500202DE9F0411F4C2049CD
:10938000204D0746204805F07FFF0A2221681E482D
:1093900005F0E3FF1D491C4805F076FF2B682068A7
:1093A000002203EBC000082100F0B8F8164805F0D1
:1093B0007BFF2268132A1FDCD5F8008008EBC20669
:1093C00008213046FFF7ACFDB0B9114B1B680121F5
:1093D00023F812103B6848F832307B6873602268CB
:1093E0002B6813F83230282B03D10A4B186800F091
:1093F00075FF236801332360BDE8F0813805002044
:109400002F8501003C050020B803002034850100B1
:109410004005002024050020034B0146186808B1D0
:1094200000F054BE704700BF2405002007B500239C
:1094300000931A461946034805F0DEFE03B05DF8B6
:1094400004FB00BF1C050020704770477047704741
:1094500007B5002300931A461946034805F0CCFED1
:1094600003B05DF804FB00BF44050020184B1B78D7
:1094700070B504460D469BB1164B027A1B789A4292
:109480000ED8154A0A291368164616D1134A002128
:10949000D154406910B1217A05F074FE0023336085
:1094A000E06898B10E4B227A1B789A420ED8036876
:1094B00029461B68BDE8704018474E2BF0DC0D298B
:1094C0001FBF591C1160054AD554E9E7012070BD42
:1094D0007804002006000020A40500205405002088
:1094E0000500002030B5002545604361034D9DF81F
:1094F0000C300560C1600272037430BD4485010008
:1095000007B5002300931A461946034805F074FE78
:1095100003B05DF804FB00BF4C050020F8B5441E05
:109520000D4D16466718BC420ED014F8011F1022CC
:109530000909284605F0EFFE2178102201F00F01FD
:10954000284605F0E8FEEEE726B10348BDE8F840FE
:1095500005F0AABEF8BD00BFB803002070B5013801
:109560000C4D13464618B04203F102030CD010F81C
:10957000014F24112C5D03F8024C047804F00F0411
:109580002C5D03F8014CEEE709B2002302F811301C
:1095900070BD00BF97850100A0F16103052B02D8C3
:1095A0005738C0B27047A0F14103052B01D83738B6
:1095B000F7E73038C0B20A2828BF0020704738B516
:1095C0000139841C00F1120514F8020CFFF7E4FFC6
:1095D0000001C2B201F8012F14F8010CFFF7DCFF03
:1095E00002341043AC420870EED138BD38B50546A0
:1095F000D8B10468ACB124789CB1286803783BB139
:109600002D2B05D0303B092B02D901302860F4E71F
:1096100008F0FDFC2C210446286809F0E9FE10B989
:109620002860204638BD0130FAE70446F9E72DE905
:10963000F34100220F4606218046FAF7F5FC002F81
:109640004ED03B68002B4BD01B78002B48D03C6899
:10965000267886B12D2E68D0A6F13003092B02D9C9
:1096600001343C60F3E72146002216B201328B5DE3
:10967000303B092BF9D92E21204609F0B9FE08B359
:10968000002211B2431801325B78303B092BF8D924
:109690004378A3F13002092A01D82F2B01D80022E8
:1096A00002E0392B88BF09220A2555438278A2F1AE
:1096B0003003092B05D82F2A16D9392A88BF092348
:1096C0001D4499B9204608F0A6FC4146024668466A
:1096D000FAF7FBFF2C21386809F08AFE18BB3860C6
:1096E000404602B0BDE8F0810023E9E702292046A8
:1096F0000FDC072E0DDC08F08EFC6422002802FB34
:1097000000F2B8BF6D422A4441466846FBF703F8B1
:10971000E0E708F079FC08F009FC4146024668469B
:10972000FAF7DFFFD6E70130D9E7611C9CE708B5FF
:1097300000200AF0A5FEADEB000008BD704730B573
:10974000441E224612F8013F002BFBD11A460A257F
:1097500014F8010F70B1032A14DC2E2806D1FF2B58
:1097600010DC8818013203710023F1E7303805FB63
:109770000303EDE7FF2B04DC032A02DC1144012084
:109780000B7130BD0020FCE72DE9F3410024DFF828
:1097900040800C700D461746061D0A2201A916F8D6
:1097A000010B08F051FE3A4601A9284609F063FE74
:1097B000032C04D03A464146284609F05CFE0134A9
:1097C000A3B2042B1CB2E8D1284602B0BDE8F08158
:1097D0009C8001002DE9F0410E4D0F4FDFF83C80D9
:1097E00006460024032C0ED033190A221979284684
:1097F00005F091FD41462846013405F045FD042C55
:10980000F0D1BDE8F081F1790A22284605F083FD08
:109810003946F0E7B8030020F87001009C80010091
:109820002DE9F047DFF8F0A0DAF8005004460E46C4
:1098300017469946002D49D02B7C03F00F03062BC9
:1098400043D12C4A2C48294604F09DFA022F804629
:1098500037D0032F37D1294ADAF80010264804F010
:1098600092FA0546B8F1000F30D098F8103003F0A6
:109870000F03042B2AD1D8F814103246204609F0E1
:1098800020FE32461E49204609F0F5FD0DB32B7C23
:1098900003F00F03042B1CD169693246204609F0FE
:1098A000EAFD32461649204609F0E5FDB9F1000F00
:1098B00004D032464946204609F0DDFD2046BDE889
:1098C000F087104AC8E70025CCE7002532460E494C
:1098D000D4E7022F0AD0032F05D0012FE1D10B4B83
:1098E00032461968DAE732460949D7E7324609496C
:1098F000D4E700BF8D8501008C0700201382010092
:10990000537A010092850100B18501008403002093
:10991000AB850100A88501009004002030B585B01A
:10992000002301AA0A2541B1B1FBF5F405FB14118E
:109930003031D15421460133F5E71A44411EC41891
:1099400012F8015D01F8015FA142F9D10022C25471
:1099500005B030BD10B5054C0549204605F09DFC0D
:109960002046BDE8104005F09FBC00BF6C030020FE
:109970007D85010010B54AB102441BB1B2FBF3F47E
:1099800003FB14228A4208D288420AD9012010BD62
:10999000884294BF00200120F9E78242F8D80020D5
:1099A000F5E78242F5E700002DE9F04F99B00DF19F
:1099B00008090C4689E80C00DDE922AB06460028C0
:1099C00000F0C880037C03F00F03062B19D8DFE8F2
:1099D00003F0BC181818B8041A00954BC5681A781B
:1099E00001321A701E464DB1CDE900AB284699E808
:1099F0000C002146FFF7D8FF6D68F4E73378013B90
:109A0000337000200EE001468A4A8B4804F0BBF90F
:109A1000054650B10023CDE90033214699E80C00FA
:109A2000FFF7C2FF19B0BDE8F08F844A8248314683
:109A300004F0A9F9824A804631467F4804F0A3F930
:109A400007461CB1012C62D02C460CE07D4A7A48B6
:109A5000314604F098F905467B4A7748314604F0D0
:109A600092F9044605B93546002C08BF3446B8F1D2
:109A7000000F6DD0002F08BF5F4635B12B7C03F07F
:109A80000F03042B0CBF6D690025002C65D0237CCF
:109A900003F00F03042B60D16469B8F1000F7FD08D
:109AA000002D66D069496A4805F0EEFBD8F814101D
:109AB000674805F0F2FB6749654805F0E5FB294674
:109AC000634805F0EAFB624805F0EEFB4846FAF70A
:109AD000F9FF002F40F0A48098F8103003F00F0336
:109AE000042B40F09B80D8F8141008A8F8F764FE07
:109AF00008A8F8F79FFD30B1002D48D00022294674
:109B000008A8F9F7A7FE08A8F8F7BAFB86E0524ABA
:109B10004948314604F037F9504A0546314646482F
:109B200004F031F90446002D7DD1464A42483146C1
:109B300004F029F90546002C8ED0002808BF3546D0
:109B400095E700242746A0468DE7002425462746B2
:109B5000D0468FE75F46D04605460023102200938B
:109B60000DEB02014FF440734846FAF7A5FE044698
:109B700093E73B49364805F087FBD8F81410344882
:109B800005F08BFB3349324805F07EFB9EE701234D
:109B9000009399E806002B4608A8F9F7A7F8B2E762
:109BA000002F3BD0002C39D03B7C03F00F03042B5B
:109BB00030D12C49264805F067FB7969244805F027
:109BC0006CFB2449224805F05FFB2146204805F044
:109BD00064FB1F4805F068FB4022796908A809F07A
:109BE00070FC214804F0A4FBA0B1204B93F9003095
:109BF00083B92F2108A809F0FBFB28B97B69032250
:109C0000402108A8FFF70CFE0123224608A91648A8
:109C100004F0EBFDB8F1000F7FF45EAF012001E727
:109C2000002CC1D158E700287FF421AF14E700BF12
:109C300069030020AB7001008C070020A2700100B6
:109C4000E47001004C850100518501006085010030
:109C50006C03002067850100568501005B850100CB
:109C60006C85010076850100E4030020B403002028
:109C700010B5044606F004F9E040431E033388BFE4
:109C8000012010BD054B1A68054B53F82010012325
:109C90008B40134214BF012000207047080500507C
:109CA000E488010007B5002300931A4619460348CB
:109CB00005F0A2FA03B05DF804FB00BFA805002080
:109CC0002DE9F84380460D46174601EB02090C4684
:109CD0004C45A4EB05060BD0D8F8003014F8011B56
:109CE0001B68404698470028F2D13046BDE8F8830B
:109CF0003E46FAE77047203005F02FBC203005F0D3
:109D00001EBC203005F02FBC38B5437F0D460BB983
:109D1000002038BD00F16804204605F02CFC002826
:109D2000F6D12046294605F0FBFB0120F1E70000B3
:109D30002DE9F0411E4600254FF47A73C0E9015326
:109D40000C4B044640F8203B8846174605F0DFFBE5
:109D500004F1680005F0DBFB9DF8183063769DF890
:109D60001C302676C4E90487A37665772046BDE8D3
:109D7000F08100BFC0850100817E284A0123C3769F
:109D800070B552F82140417E52F821104FF0A045A5
:109D900004F5E07401F5E07140F20C6645F82460CA
:109DA00045F8216001694FF0CC74C1F82445016980
:109DB0000624C1F80045847E016952F82440C1F8A8
:109DC0000845447E016952F82420C1F80C2590F919
:109DD0001820510902F01F0293406031104A42F8E6
:109DE000213090F91830002BBDBF03F00F0302F6AD
:109DF000FC32D2189B18B5BF40234022137683F85B
:109E0000002390F918300122590903F01F0302FAC8
:109E100003F3034A42F8213070BD00BFE48801001B
:109E200000E100E02DE9F041044688461F46154652
:109E3000002A50D000F12006304605F07CFB236953
:109E4000C3F88885236901221A622369C3F834653F
:109E50002369C3F8385523691A602269D2F84C3156
:109E60001BB9D2F82431002BF8D00023C2F84C31B2
:109E70002269D2F85C311BB9D2F82431002BF8D01A
:109E80000023C2F85C3122696FB9D2F8243153B98A
:109E90000123D3612369D3F84821002AFBD0002293
:109EA000C3F8482109E0012353612369D3F8042151
:109EB000002AFBD00022C3F804212369D3F824210F
:109EC00012B10022C3F824212369D3F83C0520668F
:109ED000C0B2BDE8F0811046FBE70123FFF7A2BF47
:109EE00010B5044680F8B010683005F024FB01235B
:109EF000637710BDF8B500234377036990F8B0206D
:109F0000C3F88825036901261E62036900F168050C
:109F10000446C3F8445528460F4605F01EFB236946
:109F2000C3F8480523699E602369D3F850211AB904
:109F3000D3F82421002AF8D00022C3F85021284663
:109F400005F00BFB236930B1D3F860211AB9D3F8BF
:109F50002421002AF8D00022C3F8602123696FB9B8
:109F6000D3F8242152B90122DA612369D3F84821B8
:109F7000002AFBD00022C3F8482109E001225A61DF
:109F80002369D3F80421002AFBD00022C3F804215E
:109F90002369D3F8240168B10022C3F8242123697E
:109FA000D3F8C404C3F8C404022803D004280CBFA7
:109FB00003200420F8BD0121FFF79CBF70B5436961
:109FC000D3F86421044692B10022012500F1200655
:109FD000C3F864210577304605F0ADFA6369C3F82C
:109FE000346563694022C3F8382563691D6363697A
:109FF000D3F86821DAB10025C3F8685104F1680686
:10A00000012363772577304605F095FAD4F8B4300C
:10A0100003B19847636965773046C3F8446505F036
:10A020009CFA6369C3F84805636901225A6363694E
:10A03000D3F8042162B10022C3F80421237F3BB18D
:10A040006369D3F83C05D4F8B830206603B198476B
:10A050006369D3F8242152B10022C3F82421636933
:10A06000D3F8D024C3F8D024636901225A6170BDAB
:10A070000148FFF7A3BF00BFB005002007B51623B6
:10A080001722CDE900324FF0402204231146034845
:10A09000FFF74EFE03B05DF804FB00BFB0050020E3
:10A0A0000148FFF788BF00BFB005002010B54FF48E
:10A0B000C053038000230446837003610248FFF706
:10A0C0005BFE204610BD00BFB00500200161704757
:10A0D0008078704741780148FFF702BFB005002043
:10A0E00008B5FFF7F7FF0348FFF765FFB0FA80F008
:10A0F000400908BDB0050020012303707047FF230D
:10A10000C37200230373C370037143718371C371FE
:10A11000037243728372704710B5064A01440023EC
:10A12000884204D010F8014B6340D35CF8E718462E
:10A1300010BD00BFD8850100FFF7E1BF38B5084C5E
:10A140000D46FFF7C7FFE1212046FFF7DDFD294659
:10A150002046FFF7D9FDBDE83840FFF7A1BF00BF9B
:10A16000B005002010B5054C417801222046FFF7CC
:10A17000B4FE2046FFF7C2FDC0B210BDB0050020FE
:10A1800010B5F0210446FFF7D9FF2046BDE8104086
:10A19000FFF7E8BF70B5054605F072FE002400F534
:10A1A0007A7605F06DFEB04246D22846FFF7E8FF0A
:10A1B000C307044642D52B6903B1984714200138E0
:10A1C00000BF00BF00BF00BF00BF00BF00BF00BF97
:10A1D00000BF00BF00BF00BF00BF00BF00BF00BF87
:10A1E00000BF00BF00BF00BF00BF00BF00BF00BF77
:10A1F00000BF00BF00BF00BF00BF00BF00BF00BF67
:10A2000000BF00BF00BF00BF00BF00BF00BF00BF56
:10A2100000BF00BF00BF00BF00BF00BF00BF00BF46
:10A2200000BF00BF00BF00BF00BF00BF00BF00BF36
:10A2300000BF00BFC3D1B4E70123AB70204670BD9F
:10A2400010B5E1210446FFF779FF2046BDE8104034
:10A25000FFF788BF10B50446FFF79CFF2046FFF7C5
:10A2600039FF96210648FFF74FFDFFF719FF2046FB
:10A27000FFF790FF2046BDE81040FFF7E1BF00BFA9
:10A28000B0050020FFF7E6BF10B5C3210446FFF775
:10A2900055FF2046BDE81040FFF764BF38B50446BF
:10A2A0000D46FFF777FF2046FFF714FFD2210A483B
:10A2B000FFF72AFDE94345EA0111C9B20648FFF755
:10A2C00023FDFFF7EDFE2046FFF74CFFA8421CBF21
:10A2D0000423A37038BD00BFB005002010B50446AC
:10A2E000FFF7D2FF40F00401C9B22046BDE810409C
:10A2F000FFF7D4BF70B5164604460D46FFF74AFF78
:10A3000016B12046FFF7EAFF2046FFF7E3FEA5213E
:10A310000548FFF7F9FC29460348FFF7F5FCBDE8BF
:10A320007040FFF7BDBE00BFB005002070B5002231
:10A330000C4655210646FFF7DDFF651E073415F86C
:10A34000011F00223046FFF7D5FFA542F7D170BDAF
:10A35000FFF7ECBFFFF7CEBF10B50446FFF7BAFE1C
:10A3600020460022F021FFF7C5FFBDE81040FFF7AF
:10A3700097BE000070B5164605460C46FFF70AFF6B
:10A3800016B12846FFF7AAFF2846FFF7A3FE87214C
:10A390000648FFF7B9FC002C0CBF2146802103487A
:10A3A000FFF7B2FCBDE87040FFF77ABEB0050020B1
:10A3B00010B5002204460121FFF7DCFF2046FFF71D
:10A3C000E9FEC0F3401010BDFFF7F2BF10B5044620
:10A3D000FFF75AFF20460021BDE81040FFF75EBF9F
:10A3E00038B50446FFF7D6FEC30729D42046FFF749
:10A3F000EDFF2046FFF7CEFE2046FFF76BFEB421AF
:10A400001048FFF781FCFFF74BFE2046FFF7C2FE26
:10A4100010F00403054602D00223A37002E0A278E4
:10A42000022AFAD0237843B12046FFF72DFF40F0EF
:10A430000101C9B22046FFF731FFC5F3400038BD26
:10A440000020FCE7B00500202DE9F74F057B04460E
:10A450000F46002D6BD1FFF7C3FF002869D02046BF
:10A46000FFF798FE2A46F0212046FFF743FFDFF86A
:10A47000C8804FF0FF394FF0010A94F90B30EEB26B
:10A480004FEAD60B9D4206F007060AFA06F623DAD3
:10A4900004EB0B03DB78334020460193FFF77AFE91
:10A4A0002046FFF717FE78214046FFF72DFC019B61
:10A4B000002B0CBF194680214046FFF725FCFFF713
:10A4C000EFFD2046FFF766FE820600F0400307D549
:10A4D0005BB16FF0010027E00CBF01230023DBE735
:10A4E0001BB9030658BF4FFA85F904EB0B030106AD
:10A4F00093F9032076B205F101054CBF3243B24314
:10A50000402DDA70B9D1B9F1FF3F04BF01232373A5
:10A5100084F80B90E31C013F0B3413F8012B07F870
:10A52000012FA342F9D1012003B0BDE8F08F002034
:10A53000FAE74FF0FF30F7E7B005002008B5FFF766
:10A5400083FF20EAE070C0B208BDFFF749BF704743
:10A55000054A8261002202710270092242700122C2
:10A5600081608270C27070474FA5000010B50C4624
:10A5700020460721FFF7D0FDE3791B1A58425841C6
:10A5800010BD70B5044680680E461546FFF7DDFF26
:10A59000B8B13146A068FFF7DBFE0022BE21A068FB
:10A5A000FFF7D8FE6E1E0835A068FFF76BFE06F8B1
:10A5B000010FAE42F8D1A068FFF7C7FF431E584213
:10A5C000584170BD10B51446FFF7DBFF38B10821C4
:10A5D0002046FFF7A1FD237A1B1A5842584110BDAF
:10A5E00070B504460D4680681646FFF7AEFF294653
:10A5F000A068FFF7ADFE00224E21A068FFF7AAFE7B
:10A600000022B178A068FFF7A5FE0022F178A068CB
:10A61000FFF7A0FE2B78102B04D000223179A06820
:10A62000FFF798FEA068FFF790FF2946A068FFF7A4
:10A630008FFE2278A0684821FFF78CFE142005F0D9
:10A6400053FC237813B10A2005F04EFCA068BDE846
:10A650007040FFF77ABF38B504460D468068FFF7B3
:10A6600074FF2946A068FFF773FE0022B421A0689A
:10A67000FFF770FEA068FFF7A7FE0546A068FFF78A
:10A6800064FFB5FA85F0400938BDF0B585B01446D1
:10A6900001AA07460E46FFF795FF054690B13378AD
:10A6A000102B0FD00B2C10D00C2C03D00A2C0ED159
:10A6B0003F2300E07F2301AA314638468DF8083059
:10A6C000FFF78EFF284605B0F0BD5F23F3E71F2399
:10A6D000F1E71FB50B78102B10D001AAFFF772FF1E
:10A6E00078B19DF808303F2B0ED003D81F2B0DD02A
:10A6F000002006E05F2B03D07F2BF9D10C2000E077
:10A700000B2005B05DF804FB0A20FAE70920F8E702
:10A71000F0B587B0044605F0B3FB00F51C55A06802
:10A72000FFF70AFD002310352371012601A9A06857
:10A73000FFF704FF40B305F0A3FBA84224D201A910
:10A740002046FFF713FF0028F0D023782BB901A98A
:10A750002046FFF780FF00B1267003AA01A920461A
:10A76000FFF70FFF01A920466778FFF7B2FF874286
:10A7700005D960782379607001332371D6E701A988
:10A780002046FFF7A6FFF5E707B0F0BD81707047E0
:10A790001FB501AAFFF7F5FE9DF80400003018BFB1
:10A7A000012005B05DF804FB0939C9B20229F8B5EA
:10A7B00098BF104B0546164694BF33F9114040F23E
:10A7C000EE248AB1C3787BB103786BB905F058FBEE
:10A7D000074631462846FFF7DBFF20B905F050FB5E
:10A7E000001BB842F5D3F8BD2046BDE8F84005F09F
:10A7F0007BBB00BFD8860100F8B504460F46FFF7C3
:10A8000068FF064610B900252846F8BDA068FFF786
:10A810009CFE0028F7D03946A068FFF799FD227802
:10A82000A0684421FFF796FDA5782DB13A46314640
:10A830002046FFF7B9FFE7E70125E5E710785378F1
:10A84000C00040EAC3200B78102B00B20BD1D179A5
:10A850009379C000CB1ADB0120F07F0093FBF1F36A
:10A86000103B184400B2704730B585B001AA0446C9
:10A870000D46FFF7A7FE30B101AA29462046FFF793
:10A88000DDFF05B030BD0148FBE700BF80E4FFFFFE
:10A8900010F5DC5FCABF07EE900ADFED037AFAEE2F
:10A8A000EC7A17EE900A70470000FEC208B5FFF779
:10A8B000DBFFBDE80840FFF7EBBF014604220120A3
:10A8C00001F0AABA01460422052001F0A5BA01460A
:10A8D0000622092001F0A0BA014604220F2001F04F
:10A8E0009BBA00002DE9F04F3D4E3E4C336813F00B
:10A8F000010387B082468B4615460ED1E3644FF4C0
:10A900007A732365384BA36404F15C0004F06CFC9B
:10A91000082384F8683001233360344E346001F03A
:10A920004DFC0027002859D04FF000494FF0020895
:10A93000CDF80C9005978DF8108003AC94E80E00CC
:10A940002B4805F015FD5046FFF7C1FF3B463A4640
:10A9500039460097204604F04FFC04A8FFF7BCFFDF
:10A96000234805F011FD2B465A465146306801F048
:10A970008FFF012805462DD1CDF80C9005978DF855
:10A98000108094E80E001A4805F0F2FC3168204669
:10A9900001F0E5FC04A8FFF79FFF3168204601F0B5
:10A9A000ECFC04A8FFF789FF3168204601F0DEFCCB
:10A9B00004A8FFF787FF0E4805F0E6FC3168204643
:10A9C00001F0E2FC0B4B049A5A6005F073FA80B276
:10A9D00000F08EFD284607B0BDE8F08F0546F9E788
:10A9E0006C060020840600204487010080060020B9
:10A9F0006008002078060020F0B585B007460E46B6
:10AA000014461D4601F0DAFB00B34FF000430193FA
:10AA10000023039302238DF8083004AB13E90E00E2
:10AA20000B4805F0A5FC3846FFF751FF301DFFF736
:10AA300053FF281DFFF741FF0A980430FFF742FF3C
:10AA4000034805F0A1FC034B62685A6005B0F0BDF5
:10AA50006008002078060020F0B58DB01D46002368
:10AA60000F460093FF230446164619461A4602A8CD
:10AA700004F0C2FB0B4B7A680493CDE9052372689E
:10AA8000CDE907236A68CDE90923039B0B930AAB41
:10AA9000009306AA08AB04A92046FFF7ADFF0DB04E
:10AAA000F0BD00BF5489010000B50B4B49685268E6
:10AAB00089B0CDE90231CDE9052304930123019149
:10AAC0008DF80730019B079304AA06AB02A9FFF794
:10AAD000C3FF09B05DF804FB548901007FB5094B41
:10AAE0004A680493CDE90232012301928DF80730C0
:10AAF000019B059304AA02A9FFF7D6FF07B05DF8F2
:10AB000004FB00BF5489010008B501F0BDFB01281A
:10AB100003D002280CBF0220002008BD7FB51E4EC6
:10AB20003068002836D001F0CBFE0228044601D060
:10AB300004282CD14FF000430193002303930223F8
:10AB400001AD8DF8083095E80E00144805F010FCB2
:10AB50003168284601F003FC02A8FFF7BDFE31680A
:10AB6000284601F00AFC02A8FFF7A7FE3168284634
:10AB700001F0FCFB02A8FFF7A5FE084805F004FC65
:10AB80003168284601F000FC054B029A5A602046C5
:10AB900004B070BD0446FAE780060020600800207B
:10ABA0007806002030B585B0044604F01DFB4FF058
:10ABB00000430193002303930A4D02238DF80830CC
:10ABC00004AB13E90E00284605F0D2FB0422A118BD
:10ABD0000F2001F0D9F9284605F0D6FB204605B034
:10ABE00030BD00BF6008002030B585B0044604F0D9
:10ABF000FBFA4FF000430193002303930A4D022315
:10AC00008DF8083004AB13E90E00284605F0B0FBC0
:10AC10000422A118052001F0B7F9284605F0B4FB7D
:10AC2000204605B030BD00BF6008002030B585B0BB
:10AC3000044604F0D9FA4FF0004301930023039334
:10AC40000A4D02238DF8083004AB13E90E002846A4
:10AC500005F08EFB0422A118012001F095F9284689
:10AC600005F092FB204605B030BD00BF6008002013
:10AC700007B5002300931A461946044804F0BCFAAD
:10AC8000034803B05DF804EB04F0AEBA7006002090
:10AC900078060020007C07288CBF00200120704728
:10ACA00081F0010070470846704708B50368DB6B08
:10ACB000984780F00100C0B208BD4182704713B5CB
:10ACC00002AB026803F8011D546819460122A0472F
:10ACD00002B010BD037C087C984204D107288CBFC9
:10ACE00000200120704700207047000010B5044686
:10ACF000007C072816D800F0A1FD182806D80A4BBA
:10AD000023FA00F0C04300F0010010BD1C2807D159
:10AD1000236820469B689847003018BF0120F4E75D
:10AD20000120F2E70020F0E701001001F0B591B03A
:10AD3000044604A80F46164604F056FA00224FF4C3
:10AD40007A73CDE908230CA8184B079304F04CFA4A
:10AD5000082368468DF83C3004F046FA207C07282A
:10AD600007D800F06BFD10B1207C00F0CBFD08236C
:10AD700023740F4B0F4D5B68039302A904A802953F
:10AD800001F0DDFD41F288336A46394604A801F03E
:10AD90005FFF40B12368019A9B6903920295324696
:10ADA00002A92046984711B0F0BD00BF44870100BA
:10ADB000780600205489010008B5007C072802D8D5
:10ADC00000F02EFF08BD0020FCE710B50446207CF3
:10ADD00007280BD800F032FD172801D01C2805D118
:10ADE000207C00F01DFFB0F5006FF0D310BD38B52A
:10ADF0000546007C0728144605D892B200F092FE62
:10AE000010B901236B600024204638BD08B5007CD2
:10AE1000072802D800F02EFE08BD0020FCE7007CC9
:10AE2000072802D812B200F08BBD0020704707B58A
:10AE300001220DF10701007C00F082FD0028CCBF4B
:10AE40009DF807004FF0FF3003B05DF804FB10B52C
:10AE5000037C072B044602D94FF0FF3010BD036876
:10AE60009B6898470028F7D0207C00F02FFEF5E77C
:10AE700038B50446007C07280AD800F043FD04F0EA
:10AE8000FFFF0546207C00F0D9FC10B9082323748D
:10AE900038BDFBF785FA012005F026F804F0F0FF35
:10AEA000638A401B9842EDD3207C00F0E5FCEDE77F
:10AEB0007FB50446007C07280D46164607D800F0EB
:10AEC000BDFC10B1207C00F01DFD0823237400217F
:10AED000684604F09DF96A68019B9A4202D10020FD
:10AEE00004B070BD4FF0FF3102A804F091F96A6818
:10AEF000039B9A42F3D00021212000F003FB072896
:10AF00002074ECD8291D324600F0D4FC04F0B8FFC0
:10AF10000546207C00F092FC172815D01C2813D081
:10AF20000028DCD004F0ACFF638A401B984205D8AF
:10AF3000FBF736FA012004F0D7FFEAE7207C00F0A7
:10AF40009BFC08232374CAE70120C9E710B4144608
:10AF5000064A127801EB022101EB00201A46214635
:10AF600080B25DF8044B01F00FB800BF500700201D
:10AF70007FB5037C072B05464FF000041BD84FF02C
:10AF8000004302260394019301AC8DF8086094E815
:10AF90000E000A4805F0ECF9334622460421287CCD
:10AFA000FFF7D4FF9DF804309DF80540034844EABC
:10AFB000032405F0E9F9204604B070BD60080020C4
:10AFC0007FB50B7C072B05460E4605D9002104F002
:10AFD0001FF9284604B070BD4FF0004301930023D1
:10AFE0000393022301AC8DF8083094E80E00084862
:10AFF00005F0BEF9042322460C21307CFFF7A6FFA2
:10B00000034805F0C1F92146284604F007F9E0E7B6
:10B01000600800207FB5037C072B05464FF0000435
:10B020001BD84FF0004302260394019301AC8DF826
:10B03000086094E80E000A4805F09AF93346224663
:10B040001021287CFFF782FF9DF804309DF8054011
:10B05000034844EA032405F097F9204604B070BD84
:10B060006008002007B5002300931A4619460348DC
:10B0700004F0C2F803B05DF804FB00BFF006002046
:10B0800003681B6B18470000024A02608A6942602D
:10B09000704700BF54890100808B7047008A704759
:10B0A000408C704713B502AB026803F8011D546869
:10B0B00019460122A04702B010BD704710B50446E2
:10B0C00090F82000072804D800F0D6FB082384F865
:10B0D000203010BD38B5044690F8200007280D46F2
:10B0E00001D800F0C9FB2946022000F00BFA07281E
:10B0F00084F820004FF000009EBF6084258201206C
:10B1000038BD0000F0B591B0044604A80F461646BD
:10B1100004F06AF800224FF47A73CDE908230CA8F2
:10B12000134B079304F060F8082368468DF83C3011
:10B1300004F05AF80F4B104D5B68039302A904A862
:10B14000029501F0FCFB41F288336A46394604A8B7
:10B1500001F07EFD012808D12368019A1B6A039241
:10B160000295324602A92046984711B0F0BD00BFB3
:10B1700044870100780600205489010008B50023A7
:10B18000C383043190F8200000F09CFD08BD08B591
:10B1900090F8200000F0C4FD08BD10B593B204463D
:10B1A0000A46C18B90F8200000F060FDE38B034459
:10B1B000E38310BD13B5438C04461BB94FF0FF3039
:10B1C00002B010BD01220DF1070190F8200000F03F
:10B1D000B7FB0028F2DD638C9DF80700013B638418
:10B1E000EEE710B5438C044613B94FF0FF3010BDA5
:10B1F000934294BF1AB212B290F8200000F0A0FB64
:10B200000028F2DD638C1B1A6384F0E708B590F820
:10B210002030072B05D8428C1AB1184600F056FC96
:10B2200008BD4FF0FF30FBE773B5044690F82000EF
:10B2300007280E46154601D800F01EFB094B009367
:10B240002A46736801936946822000F017FA07289E
:10B2500084F820004FF000009EBF6084012025820A
:10B2600002B070BD5489010013B50446628C2AB146
:10B27000236800211B6B20469847F7E794F82000CD
:10B2800000F0F8FBD8B10822694694F8200000F0DD
:10B2900057FB002813DD694604F1140003F0C6FFD4
:10B2A0009DF804209DF805309DF8070003EB02236C
:10B2B000A3839DF8063000EB032080B2608402B0C7
:10B2C00010BD000007B5002300931A461946034835
:10B2D00003F092FF03B05DF804FB00BFF806002006
:10B2E00007B5084B1B7801EB032101EB002001227D
:10B2F0000DF1070180B200F047FE9DF8070003B092
:10B300005DF804FB5007002007B5084B1B7801EBE4
:10B31000032101EB002002A980B201F8012D0122D6
:10B3200000F07AFDC0B203B05DF804FB50070020C6
:10B3300010B41446064A127801EB022101EB0020FA
:10B340001A46214680B25DF8044B00F065BD00BF8F
:10B35000500700202DE9F7430C4617461E4601AA68
:10B36000022324210546FFF7F1FD9DF804209DF8F6
:10B37000053043EA0223224A1C441378332B0CBFC6
:10B3800005F1080005F11000A4B2C002C4F30A09D7
:10B3900080B24844372B904680B22DD009EB06038B
:10B3A000B3F5006F28DDC9F500691FFA89F94A462F
:10B3B000394600F031FD98F80030332B0CBF05F111
:10B3C000080005F11000C002A6EB090280B292B29B
:10B3D00007EB09013444A4B200F01EFD23128DF8DE
:10B3E000043001AA0223242128468DF80540FFF7E6
:10B3F0009FFF03B0BDE8F08332463946EAE700BF5D
:10B400005107002008B50321FFF76AFF08BD07B503
:10B410000B128DF804308DF80510022301AA0421C7
:10B42000FFF786FF03B05DF804FB08B50A46042366
:10B430000C21FFF77DFF08BD07B50B128DF8043016
:10B440008DF80510022301AA1021FFF771FF03B048
:10B450005DF804FB07B5022301AA2021FFF776FD62
:10B460009DF804009DF8053043EA002003B05DF824
:10B4700004FB000038B50546FFF7ECFF04462846FC
:10B48000FFF7E8FF8442034604D1034B03EBC503F7
:10B490009C8038BD1C46F2E70807002007B5022350
:10B4A00001AA2621FFF752FD9DF804009DF8053002
:10B4B00043EA002003B05DF804FB07B5022301AAAC
:10B4C0002821FFF743FD9DF804009DF8053043EA6D
:10B4D000002003B05DF804FB044B1B78332B0CBF3A
:10B4E0000C301830C00280B2704700BF51070020F6
:10B4F000034B1A88C0F30D0050401880704700BFFE
:10B50000080000202DE9F043574B1B7885B0814699
:10B510000F468BB3332B4FF0004301934FF00005E0
:10B520004FF0020303958DF8083001AE96E80E0047
:10B530004E4814BF4FF008084FF0040804F018FFFD
:10B54000ECB22046FFF75EFF7055D8B10135EBB283
:10B550009845F5D800234FF03451F25C1D2ADCB237
:10B5600003D821FA02F2D20708D40133DAB24245F5
:10B57000F3D33E4804F008FF082465E0102120467C
:10B5800000F0C6FE3A4B002123F81410FA200138CF
:10B5900000BF00BF00BF00BF00BF00BF00BF00BFB3
:10B5A00000BF00BF00BF00BF00BF00BF00BF00BFA3
:10B5B00000BF00BF00BF00BF00BF00BF00BF00BF93
:10B5C00000BF00BF00BF00BF00BF00BF00BF00BF83
:10B5D00000BF00BF00BF00BF00BF00BF00BF00BF73
:10B5E00000BF00BF00BF00BF00BF00BF00BF00BF63
:10B5F00000BF00BF00BF00BF00BF00BF00BF00BF53
:10B6000000BF00BFC3D14A462046FFF77DFEFF22A0
:10B6100002212046FFF778FED7B139462046154D66
:10B62000FFF7F5FE00260121204600F071FE25F807
:10B6300034602046FFF741FF05EBC40358809E713C
:10B640009E800A4804F0A0FE204605B0BDE8F083C5
:10B65000094B1A88013292B2B2F5404F38BF4FF40D
:10B6600040421A801988D9E751070020600800205D
:10B670006C07002008070020080000202DE9F04793
:10B68000694B1B7886B082460E461746A3B3332B10
:10B690004FF0004303934FF000054FF00203059570
:10B6A0008DF810300DF10C0898E80E005F4814BFBB
:10B6B0004FF008094FF0040904F05AFEECB220469E
:10B6C000FFF7A0FE08F80500E0B10135EBB299459F
:10B6D000F4D800234FF0345118F803201D2ADCB2AF
:10B6E00003D821FA02F2D20708D40133DAB24A456C
:10B6F000F2D34E4804F048FE082485E0102120468D
:10B7000000F006FE4A4B002123F81410FA200138FD
:10B7100000BF00BF00BF00BF00BF00BF00BF00BF31
:10B7200000BF00BF00BF00BF00BF00BF00BF00BF21
:10B7300000BF00BF00BF00BF00BF00BF00BF00BF11
:10B7400000BF00BF00BF00BF00BF00BF00BF00BF01
:10B7500000BF00BF00BF00BF00BF00BF00BF00BFF1
:10B7600000BF00BF00BF00BF00BF00BF00BF00BFE1
:10B7700000BF00BF00BF00BF00BF00BF00BF00BFD1
:10B7800000BF00BFC3D152462046FFF7BDFDFF22D8
:10B7900002212046FFF7B8FD002F39D03946204658
:10B7A000FFF735FE5E238DF80630737903F07F03D3
:10B7B0008DF80730B3798DF808300125F3798DF8CD
:10B7C0000930311D2046ADF80450FFF72EFE3946F2
:10B7D0002046FFF731FE0623194601AA2046FFF74F
:10B7E000A7FD2946134D0026204600F091FD25F8BF
:10B7F00034602046FFF761FE05EBC40358809E715C
:10B800009E800A4804F0C0FD204606B0BDE8F087DF
:10B81000094B1A88013292B2B2F5404F38BF4FF44B
:10B8200040421A801988BAE75107002060080020BA
:10B830006C070020080700200800002030B585B004
:10B840004FF000430193002303930A4C02238DF829
:10B85000083004AB13E90E000546204604F088FDCD
:10B860002846FFF7CFFD0546204604F08DFD28460B
:10B8700005B030BD6008002030B585B04FF0004302
:10B880000193002303930A4C02238DF8083004AB84
:10B8900013E90E000546204604F06AFD28461021F3
:10B8A00000F036FD204605B0BDE8304004F06CBD28
:10B8B00060080020F0B585B04FF0004301930023ED
:10B8C00003930F4D02238DF8083004AB04460F4656
:10B8D0001646284613E90E0004F04AFD3946204674
:10B8E000FFF7A3FD31462046FFF7A6FD20460421C1
:10B8F00000F00EFD284605B0BDE8F04004F044BD60
:10B900006008002030B585B04FF00043019300235C
:10B9100003930A4C02238DF8083004AB13E90E00A0
:10B920000546204604F024FD2846082100F0F0FCDE
:10B93000204605B0BDE8304004F026BD6008002078
:10B940002DE9F04F85B04FF000430193464E0023A0
:10B950000393022336F830408DF8083001AB1746C8
:10B960000546894641480ECB04F002FDA7420EDD94
:10B970002846FFF793FD04462846FFF78FFDA042B7
:10B98000F9D106EBC5039B79E41A26F835408CB94A
:10B990002846FFF737FD142805D020B1B0F11C046C
:10B9A00018BF4FF0FF34314804F0EEFC204605B0DC
:10B9B000BDE8F08F4FEAC50BBC4206EB0B03A8BFF6
:10B9C0003C46B3F80280A7B2B9F1000F21D0284657
:10B9D000FFF782FD264A1278C8F30A0A5044372A34
:10B9E00080B23DD01AFA84F2B2F5006F38DDCAF5A4
:10B9F00000631FFA83FA5246494600F0C5FA28460A
:10BA0000FFF76AFDA7EB0A02D14492B2494600F063
:10BA1000BBFA06EB0B0236F835309179B844DB1BE4
:10BA20000F44BFB21FFA88F89BB2F92FA2F8028028
:10BA300026F8353000D8ABB95E440023B3714FEA25
:10BA400028238DF8043001AA0223282128468DF8E6
:10BA50000580FFF76DFC4021284600F059FCA2E765
:10BA60003A46D3E797719EE7080700206008002058
:10BA7000510700207FB5134D064635F83000F8B960
:10BA80004FF000430193022303908DF8083004AB7C
:10BA90000D4813E90E0004F06BFC3046FFF7FEFC86
:10BAA00004463046FFF7FAFCA042F9D1064804F0FC
:10BAB0006BFC05EBC6039879201A80B225F8360096
:10BAC00004B070BD08070020600800207FB54FF06B
:10BAD0000043019300230393104D02238DF8083097
:10BAE00001AC94E80E000646284604F041FC3046BE
:10BAF000FFF7F2FC0A4B03EBC60301225B88C3F39A
:10BB00000A031844214680B200F03EFA284604F0A9
:10BB10003BFC9DF8040004B070BD00BF600800202D
:10BB2000080700202DE9F04FB2F5006F87B028BF5D
:10BB30004FF40062DFF8E49005468A46164603ACEF
:10BB400002234FF000474FF000080397CDF8148010
:10BB50008DF8103094E80E00484604F009FC2846A1
:10BB6000FFF788FC83462846FFF74CFC01904846C7
:10BB700004F00AFC019B172B01D01C2B32D104F0DE
:10BB8000D5F9B345DCD303974FF000080227CDF871
:10BB900014808DF8107094E80E00204804F0E8FB43
:10BBA0004146334652462846FFF7D4FB202128461B
:10BBB00000F0AEFBDFF864804FF0004B0221284616
:10BBC000FFF78EFB10F0100A1FD12846FFF71AFC72
:10BBD000814648B9114804F0D7FB4E46304607B0BD
:10BBE000BDE8F08F4646CEE7404604F0CDFB04F0BA
:10BBF0009DF9CDF80CB0CDF814A08DF8107094E834
:10BC00000E00404604F0B4FBD8E71022022128467B
:10BC1000FFF77AFB014804F0B7FBDFE7600800207C
:10BC200030B585B04FF00043019300230393022306
:10BC30008DF8083004AB054613E90E000A4804F0FD
:10BC400097FB2846FFF716FC04462846FFF7DAFB69
:10BC50000546054804F098FB172D02D01C2D18BF8F
:10BC60000024204605B030BD600800202DE9FF41CA
:10BC70001C464FF00043019300230393104D022311
:10BC80008DF8083004AB06460F469046284613E967
:10BC90000E0004F06DFB3046FFF7ECFB844228BF3A
:10BCA0000446A4B22346424639463046FFF752FBCB
:10BCB000284604F069FB204604B0BDE8F08100BFCF
:10BCC000600800207FB50B7806460D4614462BB958
:10BCD0004B781BB98B780BB9C878D0B1DCB14FF079
:10BCE000004301930023039302238DF8083004AB33
:10BCF00013E90E00094804F03BFB29463046FFF7E4
:10BD000094FB21463046FFF797FB044804F03CFBC8
:10BD1000012004B070BD2046FBE700BF6008002092
:10BD20002DE9FF4700234FF000480227CDF804809B
:10BD300003938DF8087001AC94E80E0005461F4887
:10BD4000DFF8789004F014FB2021284600F0E0FA98
:10BD500002212846FFF7C4FA10F0100623D1022171
:10BD60002846FFF7BDFA10F0080A0BD0182202216E
:10BD70002846FFF7C9FA114804F006FB304604B024
:10BD8000BDE8F087484604F0FFFA04F0CFF8CDF89C
:10BD90000480CDF80CA08DF8087094E80E00484699
:10BDA00004F0E6FAD4E7102202212846FFF7ACFAA5
:10BDB000024804F0E9FA0120E1E700BF6008002032
:10BDC00007B5002300931A461946034803F014FAF6
:10BDD00003B05DF804FB00BF0007002070B5054606
:10BDE0000C468E18B44206D02178284604F0CDFACD
:10BDF00004F8010BF6E770BD024B0021187804F03F
:10BE00002DBA00BF0A000020024B0121187804F06F
:10BE100025BA00BF0A0000202DE9F3414F4B1B78E3
:10BE2000332B04460D4616461FD100EB02084C4F3B
:10BE30004D1E1FFA88F8A0457AD0FFF7DDFFF021EC
:10BE4000384604F0A2FA210A384604F09EFAE1B21C
:10BE5000384604F09AFA013415F8011F3846A4B2A6
:10BE600004F093FAFFF7D0FFE5E7342BC7B21DD1FA
:10BE7000FFF7C2FF330A241263F07F0304226946EE
:10BE800037488DF800408DF801708DF802308DF83C
:10BE90000360FFF7A3FF013D314CAF19AF4245D01E
:10BEA00015F8011F204604F070FAF7E7FFF7A4FF2A
:10BEB000FF2C08D800238DF800308DF80170042382
:10BEC0008DF802300DE0230419D4E41024F01F048F
:10BED000002344F00C048DF800308DF801708DF8CB
:10BEE0000240052E28D82A46531BDBB2B34218DA8B
:10BEF00002A8034412F8011B03F8051CF4E744F3FD
:10BF0000871323F01F03B4F5404F4FEA14228DF836
:10BF100000208DF8017034BF43F0140343F01C037C
:10BF2000CEE7F21C69460E48FFF758FFFFF76CFF9B
:10BF3000304602B0BDE8F081032269460848084F48
:10BF4000FFF74CFF731E6C1E15FA83F514F8011FE2
:10BF5000384604F01AFAA542F8D1E7E75107002065
:10BF60006008002007B502AB012203F8011D194645
:10BF7000FFF752FFC0B203B05DF804FB08B50146FD
:10BF80000020FFF7EFFF08BD2DE9F3413E4B1B7882
:10BF9000332B04460E46154620D100EB02083B4FDA
:10BFA0004E1E1FFA88F8A0453AD0FFF725FF0F2153
:10BFB000384604F0EAF9210A384604F0E6F9E1B21D
:10BFC000384604F0E2F90021384604F0DEF9013485
:10BFD00006F8010FA4B2FFF717FFE4E7342BC7B24E
:10BFE00022D1FFF709FF2412C5F3062304228DF89E
:10BFF00004408DF805708DF806308DF807500DEB74
:10C0000002012248FFF7EAFE2A460021304606F0E8
:10C0100084FA2A4631461D48FFF7E0FEFFF7F4FE9A
:10C02000284602B0BDE8F081FFF7E6FEFF2C07D8F6
:10C0300000238DF804308DF805708DF806300DE082
:10C0400023040ED4E41024F01F04002344F0080459
:10C050008DF804308DF805708DF80640032201A993
:10C06000CFE744F3871323F01F03B4F5404F4FEAA3
:10C0700014228DF804208DF8057034BF43F01003AE
:10C0800043F01803D9E700BF5107002060080020E3
:10C0900007B501220DF10701FFF776FF9DF80700B4
:10C0A00003B05DF804FB08B50020FFF7F1FF08BD01
:10C0B00010B58020FFF762FF1424FFF7F4FF40B1B2
:10C0C000013C0120A4B203F00FFF002CF5D1204663
:10C0D00010BD0120FCE7000008B50F4B33221A7099
:10C0E000FFF7E6FF08B9002008BD1020FFF746FF64
:10C0F000FFF7D9FF1028F6D11220FFF73FFFFFF717
:10C10000D2FF1228EFD10020FFF738FFFFF7CBFF57
:10C11000B0FA80F04009E7E75107002008B5124B5C
:10C1200034221A70FFF7C4FF08B9002008BD0820A8
:10C13000FFF724FFFFF7B7FF0828F6D11020FFF71D
:10C140001DFFFFF7B0FF1028EFD10020FFF716FF0B
:10C15000FFF7A9FF0028E8D11F20FFF799FFC31EB2
:10C1600058425841E2E700BF5107002008B5124B82
:10C1700037221A70FFF79CFF08B9002008BD08207D
:10C18000FFF7FCFEFFF78FFF0828F6D11020FFF71E
:10C19000F5FEFFF788FF1028EFD10020FFF7EEFE35
:10C1A000FFF781FF0028E8D13920FFF771FF031F57
:10C1B00058425841E2E700BF510700207FB52D4E9D
:10C1C0003478002C53D14FF40C7003F08DFE2A48C4
:10C1D00004F0B8F8294B0121187804F017F8FFF79C
:10C1E00013FE4FF00043019302238DF808300394AF
:10C1F00004AB13E90E00204804F0BAF8FFF78EFFF5
:10C20000B0B11F4B40221A70E5B202221E2128460F
:10C21000FFF77AF8013402221F212846FFF774F84D
:10C22000082CF1D11448012404F0AEF834701BE05E
:10C23000FFF79CFF18B1124B10221A70F2E7FFF7BC
:10C240004BFF044658B10E4B042255211B201A7097
:10C25000FFF788FE55211A20FFF784FEE2E7094B1D
:10C260001870054804F090F8204604B070BD012411
:10C27000FAE700BF52070020600800200A000020F3
:10C2800050070020510700201FB5FFF797FF38B176
:10C290001D4B1B78342B4FF0000003D0372B1BD0E5
:10C2A00004B010BD4FF000430193022303908DF8BA
:10C2B000083004AB13E90E00144804F059F8352097
:10C2C000FFF7E6FE0446114804F05EF814F0200F74
:10C2D00014BF01200220E3E74FF000430193022343
:10C2E00003908DF8083004AB13E90E00074804F002
:10C2F0003FF82E20FFF7CCFE0446044804F044F833
:10C3000014F0010FE4E700BF51070020600800208F
:10C3100038B50A4601210446FEF7F6FF054D240212
:10C32000287804EB0020013080B2FFF7B1FE00282E
:10C33000F6D138BD5007002007B5002300931A46F8
:10C340001946034802F058FF03B05DF804FB00BF34
:10C350004807002014220021103006F0DEB810B586
:10C360001031044602F05AFF204610BD10B51431BA
:10C37000044602F053FF204610BD10B518310446A4
:10C3800002F04CFF204610BD10B52031044602F0EB
:10C3900045FF204610BD30204B1C0870110902F0EB
:10C3A0000F02092A94BF3032373203F801290A46B6
:10C3B0000029F3D17047000007B5002300931A4607
:10C3C0001946034802F018FF03B05DF804FB00BFF4
:10C3D000540700202DE9F0418EB0044688461646E9
:10C3E0000021202206A806F098F8FF231A461946D5
:10C3F000009302A802F000FF04F14805554B049396
:10C400004322039B059304A92846FEF7B7FE01309B
:10C4100000F09D80504B069363688DF821601BBA35
:10C420000793330A8DF820301C22802306A9264664
:10C430002846ADF82230FEF7B0FE1A2200210DF199
:10C440001E0006F06AF856F8080F0690B388ADF89B
:10C450001C30102206A92846FEF79FFE202200214C
:10C4600006A806F05AF80627202206A92846FEF755
:10C4700094FE013FF8D1394B069340F23513ADF8E5
:10C480001C303D238DF81F3007238DF82030012309
:10C490008DF821303368CDF82230B388ADF82630DE
:10C4A0002F498DF81E8040F60C430DF12A00ADF89F
:10C4B000283006F0B4FFE27A0CA92046FFF76BFFA4
:10C4C000227B0DF132012046FFF765FF627B0DA94B
:10C4D0002046FFF760FF1E2206A92846FEF75DFEF4
:10C4E000B8F1030F24D140F23243ADF81830237C69
:10C4F0008DF81A30637C8DF81B30A37C8DF81C30CE
:10C50000E37C8DF81D3040F23643ADF81E30237FBA
:10C510008DF82030637F8DF82130A37F8DF8223095
:10C520000C22E37F8DF8233006A92846FEF735FE5E
:10C530000C4A0D4B06A9CDE906232846FF23092204
:10C540008DF82030FEF729FE2846FEF720FE0EB0BB
:10C55000BDE8F08154890100010106006382536344
:10C560008C87010037060103060F3A3B2DE9F043A3
:10C5700091B005468846164603F082FC05F1480452
:10C5800007462046FEF770FE00280BDC03F078FC1F
:10C59000C01B404500F2D280F9F702FF012003F0F2
:10C5A000A3FCEEE7242207A92046FEF71AFE9DF819
:10C5B0001C30022B40F0BD80B5F86430432B40F0B6
:10C5C000B880089F3FBA3760062205F108010EA81F
:10C5D00005F070FF064628B92B689F4202D36B68AE
:10C5E0009F4207D92046FEF768FD0026304611B06D
:10C5F000BDE8F0830B9B2B610146CC222046FEF761
:10C60000F0FD05F124072046FEF74AFD002840F31F
:10C6100091802046FEF7CEFD33287DD015DC012821
:10C6200044D006DC0028EED02046FEF7C3FDC2B29F
:10C6300053E0032844D00628F6D12046FEF7BAFD81
:10C640000422804605F1200141E03A284AD020DC4E
:10C65000352823D03628E7D12046FEF7ABFD05F17B
:10C660001C084146814601A802F0D8FD002103A81C
:10C6700002F0CEFD029A049B9A4230D0414605A8B2
:10C6800002F0CCFD2A6E069B9A4228D05FFA89F20E
:10C6900023E03B2833D0FF28B5D0C5E72046FEF77E
:10C6A00089FD2046FEF786FDC6B2ACE72046FEF7C0
:10C6B00081FD042205F114012046FEF792FDA2E758
:10C6C0002046FEF777FD0422804605F1180120463A
:10C6D000FEF787FD5FFA88F2043A0021ECE70422B6
:10C6E0004146E9E72046FEF765FD042205F12801F1
:10C6F0002046FEF776FDAB6A1BBAAB6283E72046A5
:10C70000FEF758FD042205F12C012046FEF769FDD5
:10C71000EB6A1BBAEB6276E72046FEF74BFD04227C
:10C7200039462046FEF75DFD6B6A1BBA6B622B63D0
:10C7300069E700262046FEF7C0FC57E7FF2655E7CD
:10C740002DE9F34704464FF4FA61012003F019FA8A
:10C750002746606047F8480B3846FEF7AFFC442197
:10C760003846FEF7B7FC002800F0908003F088FB05
:10C770004FF00009804600254FF0030A94F844303A
:10C78000032B1CD043BB63680133636003F078FB69
:10C790004FF47A72A0EB08000121B0FBF2F22046C0
:10C7A00092B2FFF717FE012384F84430002DE5D143
:10C7B00003F066FBA36BA0EB08009842DBD9384678
:10C7C000FEF77CFC63680133636003F059FB20646F
:10C7D000284602B0BDE8F087042B11D1636801330D
:10C7E000636003F04DFB4FF47A72A0EB0800032165
:10C7F000B0FBF2F2204692B2FFF7ECFD0223D3E742
:10C80000012B19D101AAE16B2046FFF7AFFE0228E8
:10C81000064638D1019B636003F032FB4FF47A7215
:10C82000A0EB08000321B0FBF2F2204692B2FFF722
:10C83000D1FD84F84460B9E7022BB7D101AAE16BBE
:10C840002046FFF793FE0528064617D1636A84F851
:10C8500044A013B94FF461736362A36A13B9636AA6
:10C860005B08A362E36A1BB9636AA3EBD303E362C9
:10C87000A36A2363E36A636301257FE7062802D185
:10C8800084F8449092E7FF2EFAD08FE705469FE7A1
:10C89000F8B500250F460446C0E90955C562C0E950
:10C8A0000E2385608581FFF755FD3B68A360BB883B
:10C8B000A38184F844502046BDE8F840FFF740BF0C
:10C8C00010B5044603F0DCFA236CC31AB3F57A7F83
:10C8D00014D34FF47A71B3FBF1F201FB1233C01A97
:10C8E000236B206451008B4234BF00239B1A2363C7
:10C8F000636B99428CBF00239B1A6363206BE0B982
:10C9000094F84430032B06D1042384F844302046A5
:10C91000FFF716FF0130636B73B994F84430032BB3
:10C9200000D04BB9002384F844302046FFF712FDB5
:10C930002046FFF705FF033010BD0020EBE74B68F2
:10C94000436000230381704770B5002401392346FA
:10C9500011F8010FB8B1A0F13005EEB2092E08D8D8
:10C9600003EB830305EB43039BB2FF2BF0D90020BD
:10C970000DE02E28FBD1032CF9D0601C1444237148
:10C98000C4B20023E4E7032C01D1D371012070BDB0
:10C9900007B5002300931A461946034802F02CFC01
:10C9A00003B05DF804FB00BF5C0700202DE9F743EE
:10C9B00005460E4603F064FA05F10C04288105F1E2
:10C9C0000801022202AD2046FEF7E7FB012325F80D
:10C9D000023D022229462046FEF7DFFB4FF480731A
:10C9E000022229462046ADF80630FEF7D6FB00238A
:10C9F000022229462046ADF80630FEF7CEFB022281
:10CA000029462046FEF7C9FB022229462046FEF7AA
:10CA1000C4FB37463378E3B13E46B04618F8013BD5
:10CA20000BB12E2B13D1A6EB0709B9F1000F0CDDCA
:10CA300001220DF1050120468DF80590FEF7ADFBB2
:10CA40004A4639462046FEF7A8FB4746E2E74646F7
:10CA5000E3E702A9012201F8033D2046FEF79DFB12
:10CA60004FF48076294602222046ADF80660FEF794
:10CA700094FB022229462046ADF80660FEF78DFBA6
:10CA8000012003B0BDE8F0832DE9F04387B00646EE
:10CA90000F46904603F0F4F906F10C0405462046D3
:10CAA000FEF7E2FB002808DC03F0EAF9401BB8427D
:10CAB00000F2C480F9F774FCF1E7726A73689A4275
:10CAC00040F0BF80338D352B40F0BB802046FEF711
:10CAD000E7FA0B2840F3B8800C220DEB0201204648
:10CAE000FEF77FFBBDF80E203189130A43EA0223CB
:10CAF000BDF80C201BB29DB29142ADF8065001D199
:10CB0000002B07DB2046FEF7D8FA4FF6FC7007B083
:10CB1000BDE8F08340F20F231D4005D02046FEF70C
:10CB2000CCFA4FF6FB70F2E7BDF812301F0A47EA65
:10CB30000327BFB22FB92046FEF7BFFA4FF6FA70AF
:10CB4000E5E7BDF810305BBAAAB29BB29A4216DA9A
:10CB500001220DF10A012046FEF743FB9DF80A2051
:10CB60001AB100212046FEF73CFB9DF80A1000296F
:10CB7000EED104222046FEF734FB0135E1E7002622
:10CB8000B14601220DF105012046FEF72AFB9DF872
:10CB9000052012F0C00134D112B12046FEF721FB6E
:10CBA0009DF80550002DECD1022202A92046FEF787
:10CBB00018FB02220DF10A012046FEF712FB0422A7
:10CBC00029462046FEF70DFB02220DF10601204604
:10CBD000FEF707FBBDF80830BDF80620B3F5807FEF
:10CBE00052BA92B21CD1BDF80A0040BA85B2012DEA
:10CBF00016D1042A0DD02046FEF75FFA4FF6F770E3
:10CC000085E7012200212046FEF7EBFA8DF805901A
:10CC1000C6E708F104012046FEF7E3FA284676E766
:10CC2000013600212046B6B2FEF7DBFAB742A8D1A2
:10CC30002046FEF742FA4FF6F67068E74FF6FF70AF
:10CC400065E74FF6FE7062E74FF6FD705FE70000A4
:10CC50002DE9F34705468A4691469846FFF774FE4C
:10CC60000446B8BB1E4B6A685B689A4234D003F036
:10CC700007F905F10C0600F00F0101F5806130465F
:10CC8000FEF728FA0128074620D1164B00933522DB
:10CC90006B68019369463046FEF770FA98B15146C9
:10CCA0002846FFF783FE70B13046FEF770FA50B1A8
:10CCB0004A4641462846FFF7E7FE0446F9F770FB6F
:10CCC000384603F011F93046FEF7F8F9204602B075
:10CCD000BDE8F0870124F9E76FF00104F6E700BF33
:10CCE0005C0700205489010007B5002300931A4611
:10CCF0001946034802F080FA03B05DF804FB00BF58
:10CD000064070020006903681B691847006903680D
:10CD10005B69184713B5006949680368034C0191C2
:10CD20009B6900946946984702B010BD5489010080
:10CD300000690368DB691847006903689B6A184744
:10CD40000069003018BF01207047006C7047016413
:10CD5000704710B590F83830044633B9206903683D
:10CD6000DB689847002808DA10BD03689B6898477D
:10CD70000028F3D14FF0FF30F6E794F82220A2F11B
:10CD80000803022BF0D8A36A002BC2BFE36A013369
:10CD9000E3620A2AE8D1E36B013BE363002BE3D1B2
:10CDA000092384F82230DFE710B5044600690368E0
:10CDB0001B6A984794F82230083B022B07D8A36AD5
:10CDC000002B04DD0028A2BFE36A1B18E36210BD3C
:10CDD00073B590F82230092B04460ED10026206945
:10CDE00003689B68984740B120690368DB689847EF
:10CDF000C5B20A2D1CD184F8225094F822300A2B97
:10CE000004D1E36B13B9092384F8223094F822305B
:10CE1000092B22D0206903689B68984794F8223038
:10CE20000A2B03D1E36B9842A8BF184602B070BD2D
:10CE30000D2DD4D0284605F0E6FA0028CFD0E06BBF
:10CE4000ADF8046010228DF804500021050101A8FE
:10CE500007F074FA2844E063C1E70020E6E7000029
:10CE600000234FF0FF32C0E90A23084A80F822303D
:10CE700012680263064A4362126880F83830C3635E
:10CE800047F2305342630364704700BF1000002034
:10CE90001400002038B504461D4600204FF47A7374
:10CEA000C4E901030B4B2360C4E9041204F1180028
:10CEB00002F09AF90123258484F8443084F845303F
:10CEC000054904F1480002F0B5FE2046FFF7C8FF0F
:10CED00038BD00BFF4870100AA88010010B50446E0
:10CEE000006903685B6A98472046BDE81040FFF779
:10CEF000B7BF012380F822307047000038B50446E0
:10CF00000069154602F0C9F90449206902F0C5F923
:10CF100029462069BDE8384002F0D6B9D16F01003A
:10CF200038B504460D460069114602F0B6F91D49B0
:10CF3000206902F0B2F92946206902F0AEF91A49D7
:10CF4000206902F0C1F994F84530F3B16369B3B1D7
:10CF50001649206902F0A1F9D4E9040102F09DF913
:10CF6000238C502B08D01249206902F096F90A222E
:10CF7000218C206902F0F1F9206902F095F90D4B3E
:10CF80000D491A682046FFF7B9FF94F8443023B1E1
:10CF90000A4A0B492046FFF7B1FF012384F82230EB
:10CFA000002038BDF8700100B9870100C387010077
:10CFB000E87101000C000020CA870100D58701003C
:10CFC000DB87010038B504460069154602F065F9B3
:10CFD0000549206902F061F9294620690A22BDE865
:10CFE000384002F0BCB900BFD16F010010B5044653
:10CFF000006902F059F9022384F8223010BD70B59F
:10D0000090F82230012B04460D46164601D8FFF752
:10D01000EDFF20690368324629465B68BDE8704031
:10D02000184770B590F82230012B04460D4601D800
:10D03000FFF7DCFF2069036829461B68BDE87040E4
:10D04000184710B50446206903689B68984720B1CB
:10D0500020690368DB689847F5E710BD2DE9F347C1
:10D06000994690F82230083B022B04460E46924621
:10D07000DDE90A7804D8FFF7E4FF2046FFF7F0FE69
:10D0800094F82250012D44D894F8443063B1D4E987
:10D090000401228C0368002934D121490091E169FF
:10D0A00001919B6969462EE0206903689B6A984755
:10D0B0000028ECD0314652462046FFF731FF0646A5
:10D0C000E0B9B9F1000F04D04A4616492046FFF7EF
:10D0D00015FF002F20DD3A4613492046FFF772FF67
:10D0E000B8F1000F18D001252046FFF77FFF2DB1C2
:10D0F00023683A465B68414620469847304602B06E
:10D10000BDE8F087DB6998470028D3D14FF0FF36A0
:10D11000F4E76FF00106F1E7002DEFD1E4E700BF7F
:10D120005489010093870100A087010090F8223004
:10D13000012B01D8FFF75ABF7047FFF7F7BF000078
:10D1400007B500234FF0FF32CDE90023024AFFF775
:10D1500085FF03B05DF804FBE68701002DE9F04789
:10D1600090F82230012B044651D9DFF8D8800025F1
:10D17000032700236362022384F8223002F080FE3A
:10D18000464682464FF00A090A2D46D002F078FE44
:10D19000236CA0EB0A00984245D2236820469B6886
:10D1A000984748B323682046DB689847431C0546E8
:10D1B000ECD094F82230022B05D0032B0FD002F0D4
:10D1C0005FFE8246E0E733782A2B01D083421AD1F2
:10D1D0007278731C0AB984F822701E46EFE7A0F13A
:10D1E0003002092A95BF636A042309FB032384F8EC
:10D1F000223098BF6362E2E74FF47A7002F074FE67
:10D20000C2E70A2D06D16FF00300BDE8F0876FF08A
:10D210000100FAE76FF00200F7E7636AC72B02DC50
:10D22000652B18BF002594F82230042BE9D1606AE1
:10D23000C72801DC65289CD10A2D18BF6FF00200B9
:10D24000E3E700BFAF87010038B501F148050446A8
:10D250003A21284602F0CEFD421C034605D106497C
:10D26000204602F0E7FC204638BD00222946204631
:10D2700002F0DEFDF7E700BFAA880100F8B501F172
:10D28000480605460F4630463A2102F0B3FD441CDD
:10D29000013005D10C49284602F0CCFC2846F8BDE7
:10D2A0003B6DA34209DD2146304602F087FD007840
:10D2B00005F0A0F808B10134F2E73B6D2246314693
:10D2C000284602F0B5FDE9E7AA88010010B5036819
:10D2D0000446DB68984794F82230A3F10802022A3A
:10D2E000C0B232D9052B31D0072B39D0042B54D101
:10D2F000226B137883420BD1531C2363537823B9D9
:10D30000C4E90A33052284F822200A281DD136E018
:10D31000636B197881420BD15A1C62635B78002BD6
:10D32000F3D1012384F83830062384F82230ECE767
:10D330001B4909688A42F7D11A4A12689342F3D10D
:10D340000D28F1D1072384F8223010BDA0F130025E
:10D35000092AE9D8A36A0A2101FB0323A362D4E7BF
:10D360000A28F2D194F838309BB1092384F822308E
:10D370000023E36394F82230083B022BE5D9042311
:10D3800084F82230064B1B682363064B1B686363DB
:10D39000DBE7082384F82230ECE70A28D5D1E9E757
:10D3A000100000201400002038B5044602F068FD8B
:10D3B000054694F82230083B022B13D902F060FD99
:10D3C000236C401B98420DD2236820469B689847E7
:10D3D00018B12046FFF77AFFE8E74FF47A7002F0C1
:10D3E00083FDE6E794F82230083B022B94BF00202F
:10D3F0006FF0020038BD10B590F82230083B022BC8
:10D40000044601D9FFF7D0FFA06A10BD38B590F8E7
:10D410002230083B022B054601D9002038BDFFF71A
:10D42000EAFF0130F9D02846EC6AFFF7E4FF8442B6
:10D43000B4BF00200120F1E7FFF7E8BFFFF7E6BF28
:10D4400038B500F1480504460E49284602F04FFC65
:10D4500094F82230083B022B09D92046FFF736FF0B
:10D460000D2801D00A2807D1236D002BF0D0206DA4
:10D47000003018BF012038BDC1B2284602F058FC68
:10D48000E6E700BFAA88010007B5002300931A460B
:10D490001946034801F0B0FE03B05DF804FB00BF7D
:10D4A0007C07002000B55DF804FB0020704700B544
:10D4B00001205DF804FB80687047C1607047036815
:10D4C00010B59B690C469847036821461B68BDE868
:10D4D000104018472DE9F84380460D46174601EBEA
:10D4E00002090C46A145A4EB050609D0D8F8003086
:10D4F0004046DB689847431C03D004F8010BF1E772
:10D500003E463046BDE8F883C368013310B5044693
:10D5100012D1236820469B69984703689B68984707
:10D5200058B123682046DB6898472028F1DD23683E
:10D53000C1B25B6920469847012010BD70B5044612
:10D54000C068431C18D102F09BFC00F5FA752368F3
:10D5500020469B69984703689B68984718B902F072
:10D560008FFC8542F3D8236820469B69984703685F
:10D57000BDE87040DB6818474FF0FF33E36070BDD3
:10D5800010B5182004F074FF044618B118220021C9
:10D5900004F0C3FF204610BD70B506460C46D4B15A
:10D5A000237C65681B0704D4E16811B13046FFF79E
:10D5B000F3FF237C03F00F03042B03D1606908B150
:10D5C00004F05EFF206808B104F05AFF204604F022
:10D5D00057FF2C46E3E770BD2DE9F04F036885B097
:10D5E000DB6805460E469847421C044604D14FF0BE
:10D5F000FF3005B0BDE8F08F2D2832D12B682846CA
:10D60000DB689847431C0446F1D04FF0FF3300938A
:10D61000A4F13003092B4FF000070DD84FF00A0892
:10D620002B682846DB689847A0F13003303C092B73
:10D6300008FB07470446F3D92E2C14D024F020030E
:10D64000452B10D0009B7B437361337C022262F335
:10D65000030333742B6828465B69E1B298470020C6
:10D66000C7E70123D3E7384604F0FEF82E2C8046A6
:10D67000894639D12B68DFF818B1DB68284698470E
:10D68000002704464FF0000A52465B464046494692
:10D6900004F054F980468946A4F1300004F0E4F81F
:10D6A00042464B4603F094FF2B688046DB682846D1
:10D6B00089469847A0F13003092B07F1FF3704464C
:10D6C000E2D924F02003452B2AD12B682846DB68B9
:10D6D00098472B28044609D12B682846DB689847D1
:10D6E00004464FF0010A0AE00027EAE72D28F8D1A6
:10D6F0002B682846DB6898474FF0FF0A04464FF036
:10D70000000B0A22A4F13003092B0DD802FB0B3BBE
:10D710002B680392DB6828469847039A0446F1E792
:10D720004FF0010A4FF0000B009804F09DF84246BC
:10D730004B4604F003F9CDE90001584604F094F893
:10D7400080465046894604F07FF802460B46404624
:10D75000494604F0F3F880463846894604F084F8D8
:10D7600002460B464046494603F032FF02460B464E
:10D770000020074902F04CFE02460B46DDE900019D
:10D7800004F0DCF804F0D2FB337C706103225EE726
:10D790000000244019B10A22496901F0BCBD0846C5
:10D7A0007047000000000000F8B506462DED028B22
:10D7B000D1B391ED058A18EE100A04F067F8B5EEC2
:10D7C000C08AF1EE10FA04460D4606D51A493046D5
:10D7D00001F063FD05F100431D462946204604F093
:10D7E00085FB0A2201460746304601F0C2FD134977
:10D7F000304601F052FD384604F026F802460B464A
:10D800002046294603F0E2FE09A3D3E9002303F0F2
:10D81000DFFE00220A4B04F091F804F067FB0A22B5
:10D820000146304601F0B4FDBDEC028B0020F8BD8E
:10D830009A9999999999A93FEB8D01009C800100D3
:10D8400000002440F8B50368DB6806460F46984799
:10D85000222803D04FF0FF342046F8BD3B7C042241
:10D8600062F303033B7400F0EFFA05460028F1D0A1
:10D8700033683046DB689847431C044611D0222C9D
:10D8800036D01F2C34DD5C2C04D02946E0B200F0E9
:10D89000F1FAEDE733683046DB689847421C0446EE
:10D8A00003D1284600F00EFBD6E7622817D007DC2C
:10D8B0002F2803D05C2801D02228D9D12946E6E7B9
:10D8C0006E280FD004DC6628D2D129460C20DEE772
:10D8D00072280AD07428CBD129460920D7E72946D7
:10D8E0000820D4E729460A20D1E729460D20CEE7B3
:10D8F000284600F0CBFA00247861ADE738B50D4634
:10D900001D49044601F0C9FC7DB3013D15F8011F16
:10D9100059B31F2907D9222905D05C2903D02046F5
:10D9200001F0BFFCF2E75C21204601F0BAFC297847
:10D930000C2914D007D8092915D00A2911D0082993
:10D94000E4D16221EBE72229E9D003D80D29DDD10A
:10D950007221E4E72F29E2D05C29E0D0D6E76621E6
:10D96000DDE76E21DBE77421D9E72221204601F0B3
:10D9700098FC002038BD00BFD46F01004969FFF753
:10D98000BDBF0368DB6810B504469847431C0AD046
:10D990002028236802DCDB682046F6E7C1B25B6919
:10D9A00020469847002010BD03682DE9F047DB684A
:10D9B00004460E46914698477B2803D04FF0FF302F
:10D9C000BDE8F087337C062262F3030333742046FC
:10D9D000FFF7D7FF23682046DB6898477D2844D0AF
:10D9E0002368C1B25B6920469847FF274FF0000AC1
:10D9F000FFF7C6FD05460028E0D08FB3F060204653
:10DA0000FFF7BFFF29462046FFF71CFF0130D5D0A6
:10DA10002046FFF7B6FF6B692B602368C5F814A09A
:10DA2000DB68204698473A28C8D12046FFF7A9FF6F
:10DA30004A462946204600F01BF80130BED0204659
:10DA4000FFF79FFF23682046DB6898472C28A846ED
:10DA50004FF00007CCD07D3818BF4FF0FF30AFE754
:10DA6000C8F80400C0F80880C9E70020A8E7000053
:10DA7000F7B504460D461746FFF783FF013002D184
:10DA80004FF0FF3011E023682046DB689847431CC5
:10DA90000646F5D02368C1B25B6920469847222E1E
:10DAA00005D129462046FFF7CDFE03B0F0BD2D2E4F
:10DAB00003D0A6F13003092B04D829462046FFF7EE
:10DAC0008BFDF2E75B2E05D13A462946204600F051
:10DAD00080F8EAE77B2E05D13A4629462046FFF733
:10DAE00063FFE2E76E2E17D102AE002346F8083D31
:10DAF000236804221B6931462046984704280246C1
:10DB0000BED12149304605F0CAFC0028B8D12B7C93
:10DB10006FF303032B74C8E7662E19D1002300931B
:10DB20008DF80430236805221B6969462046984712
:10DB30000528A5D105221549684605F0B0FC002846
:10DB40009ED12B7C2875012262F303032B74ACE772
:10DB5000742E95D102AE002346F8083D23680422B6
:10DB60001B693146204698470428024688D1084957
:10DB7000304605F094FC002882D12A7C012363F30F
:10DB800003022A742B7590E76E88010073880100E8
:10DB900079880100F8B5064617460D4611B90024EC
:10DBA0002046F8BDFFF7ECFC04460028F7D02846D5
:10DBB000FFF7E7FE3A4621462846FFF759FF0130B6
:10DBC000EED121463046FFF7E7FCE8E70022FFF7F9
:10DBD000E1BF2DE9F8430368DB6804460F46914630
:10DBE00098475B2803D04FF0FF30BDE8F8833B7CBB
:10DBF000052262F303033B742046FFF7C2FE23684D
:10DC00002046DB6898475D282BD02368C1B25B694A
:10DC100020469847FF26FFF7B3FC05460028E2D0D0
:10DC2000D6B1F8602046FFF7ACFE4A4629462046AA
:10DC3000FFF71EFF06460028D5D12046FFF7A1FEBC
:10DC400023682046DB6898472C28A846E3D05D3837
:10DC500018BF4FF0FF30C8E7C8F80400C0F80880CC
:10DC6000E0E70020C1E738B5054651B3CC687B2119
:10DC700001F017FB013002D14FF0FF3038BDB4B1D5
:10DC800021682846FFF73AFE0130F5D03A212846B0
:10DC900001F007FB0130EFD02146284600F014F8D0
:10DCA0000130E9D0646814B12C212846E0E77D21D9
:10DCB000284601F0F6FA01304FF0FF3018BF00207F
:10DCC000DCE70846DAE70000E9B10B7C03F00F035C
:10DCD000062B18D8DFE803F004070D0F1113150009
:10DCE0000A4901F0DABA0B7D0BB10949F9E7094994
:10DCF000F7E7FFF74FBDFFF757BDFFF73FBE00F057
:10DD00000EB8FFF7B0BF0020704700BF6E8801005B
:10DD100079880100738801001046FFF7D5BF38B538
:10DD20000546F1B1CC685B2101F0BBFA013002D1AC
:10DD30004FF0FF3038BD54B121462846FFF7C4FFED
:10DD40000130F5D0646814B12C212846ECE75D2140
:10DD5000284601F0A6FA01304FF0FF3018BF00202E
:10DD6000E8E70846E6E7CB680022D0B201320BB103
:10DD70005B68FAE77047C86820B11AB1013AD2B2BD
:10DD80004068F9E7704738B5CC68154634B1294684
:10DD9000206805F000FB08B16468F7E7204638BD4D
:10DDA0004AB1CB6813B9CA6070470B46596800295D
:10DDB000FBD15A6093607047F8B505460E4617468A
:10DDC0001C4673B1186808B104F05AFB384605F0D8
:10DDD0002FFB2246206031462846BDE8F840FFF779
:10DDE000DFBFF8BD08B5FFF7CBFB18B1037C6FF3BD
:10DDF0000303037408BD10B50C46FFF7C1FB28B13F
:10DE0000037C4461022262F30303037410BD70B506
:10DE10000D46194604461646FFF7EDFF3246034607
:10DE200029462046BDE87040FFF7C6BF07B500236E
:10DE300000931A461946034801F0DEF903B05DF875
:10DE400004FB00BF8407002038B50C2004F010FB51
:10DE5000044650B1064820604FF480752A460021E0
:10DE600004F05BFB00236560A360204638BD00BF63
:10DE70008C080020D1E90123934204D20A68D054CF
:10DE80008B6801338B60002070470000826838B5D2
:10DE9000044622B10368134413F8013C1BB1214628
:10DEA0000020FFF7E7FFA06804F0E2FA054628B17A
:10DEB000034905F0B4FA204604F0E2FA284638BDDA
:10DEC0008C08002008B104F0DBBA704710B5054C8F
:10DED000204601F0E9F920460349BDE8104001F071
:10DEE000D3B900BFE8070020A4880100F0B504788A
:10DEF0009FB005464CB31A4B1A4F1B68986804F044
:10DF000067F92846174906F037F91EAD012445F890
:10DF1000780D3946002006F02FF91E2C264645F8CC
:10DF2000240002D001340028F3D10F4B009F1C685D
:10DF300084B12168384605F068FA48B96368294613
:10DF4000304698470446FFF7C1FF20461FB0F0BD9A
:10DF5000A468EDE70549064801F0ACF9F3E700BF16
:10DF600038000020F8700100D0070020AB880100C5
:10DF7000E8070020F8B505460C200F4604F078FAB3
:10DF80000C4B04461860284605F06DFA013004F089
:10DF90006FFA2946064605F042FA284605F063FA6C
:10DFA00000233354044B1A68A260C4E900671C6064
:10DFB000F8BD00BFD00700209007002070B51648BC
:10DFC000164D01F0BFFCC4B20A2C0CD00D2C0AD0A7
:10DFD000082C15D12146104801F063F92B7873B154
:10DFE000013B2B700BE02B780D4E0E490A480024A4
:10DFF000F45401F052F93046FFF778FF2C7070BDF1
:10E000002146054801F04DF92B783A2B9FBF5A1C49
:10E010002A70034AD454F2E7E8070020D40700200E
:10E0200094070020A888010010B5044C204601F098
:10E0300083FC10B1FFF7C2FFF8E710BDE80700202E
:10E04000054A00231370054A0146136010B10448C5
:10E0500001F032BC704700BFD407002090070020B9
:10E06000E807002070B504460D4601F009FFA061E5
:10E07000A068036829461B68BDE87040184770B562
:10E0800004460D46164601F0FBFEA061A068036839
:10E09000324629465B68BDE87040184710B5044613
:10E0A000C06804F0EDF9204610BD2DE9F0410546A9
:10E0B0000E4601F0E5FE4FF47A778046A8680368C3
:10E0C0009B689847044658B901F030FF01F0D8FE2C
:10E0D000AB8AA0EB08007B439842EFD3204605E0D3
:10E0E000A8680368DB68984730700120BDE8F081BC
:10E0F00038B5148821441546FFF7D7FF08B101341D
:10E100002C8038BD2DE9F74F02AD002625F8026DB1
:10E110008A462A46C1680446FFF7EAFF18B900207C
:10E1200003B0BDE8F08FE3680DF1080993F80080B3
:10E1300009F8036D0127BDF80630052B07D14FF014
:10E14000FF33A068E36303685B6A9847E7E74946E3
:10E150002046FFF7AAFF0028E1D0BDF80630E268AC
:10E16000591CADF806109DF80510D1549DF80530E6
:10E1700003F07F0207FB02661A064FEAC717DAD4DC
:10E180009DF8063008F0F008013BB8F1300F8AF82E
:10E1900000301DD12A46E1682046FFF7A9FF00287C
:10E1A000BDD02A46E1682046FFF7A2FF0028B6D07E
:10E1B000E2689AF80030134459789D78137805EB9B
:10E1C00001259B07ADB201D50235ADB2022701E0B2
:10E1D00000273D46BDF806B0A7EB0B0707EB0B0287
:10E1E00096422AD949462046FFF75FFF002896D07D
:10E1F000A06B88B1B8F1300F0ED19AF80020C2F1AF
:10E20000FF2202F57F02FE325A44AA4204D9026874
:10E210009DF8051012689047BDF80620218A9142AA
:10E2200008D9E1689DF805008854BDF80620013240
:10E23000ADF806200BF1010BD0E7A26B22B9218AC1
:10E24000594538BFADF80620BDF8060068E7012043
:10E25000704773B50025DC1103F07F06A3B20CB143
:10E2600046F080060DF1080C681C6544C0B205F844
:10E27000046C0546002CEED1C0F10405515501ADEA
:10E28000A04205DD231A1344615D59710134F7E79B
:10E29000013002B070BDF8B5064617461C46FFF7C0
:10E2A000D8FFB368C0B21A680444C0F105015568CC
:10E2B000394422461846A847054601F0E1FDB06101
:10E2C000A8B2031B58425841F8BD10B5C368E022FC
:10E2D0001A70C36800225A7004468068E1680368B7
:10E2E00002225B689847A0684FF0FF33E36303683E
:10E2F0005B699847A06803685B6A984701F0C0FDB6
:10E30000C4E9060010BD023330B598B20C46631A5A
:10E3100014F8015B9BB21DB1431C155498B2F6E78B
:10E32000C11A0A44191202F8021C02F8013C30BD5D
:10E3300038B50546806808B9002038BD03689B6A77
:10E340009847EC6B68B9002CF6D1A8686FF002030F
:10E35000EB6303685B699847A86803685B6A984742
:10E36000EAE7B4FA84F04009E7E700002DE9FF4747
:10E370000C9D9DF840A00446894617461E46FFF7AF
:10E38000D7FF8046002840F0DF80A06803689B6AC2
:10E390009847002840D00123E3826E4B029345F258
:10E3A0005443ADF80C3004238DF80E30052302A938
:10E3B0001944E26811F8051CD15401330C2BF6D135
:10E3C000002D3DD09DF838309DF834205B0143F09E
:10E3D000040343EAC203DBB2BAF1000F01D043F0F9
:10E3E00002031FB1002E2DD143F08003E2681373A6
:10E3F000638AE2681B125373E368628A9A73218A04
:10E40000484605F073F8238A113098421DD9A06858
:10E4100003685B6A984797E0A068216B0368A28E47
:10E4200039B1DB6998470128B5D06FF00103E36388
:10E430008AE049499B690291E16A039102A9F1E7E7
:10E440002B46C9E743F0C003D0E749460F23E268F3
:10E450002046FFF758FF814605B3218A284605F07C
:10E4600045F809F102031844238A9842CFD84B4655
:10E470002946E2682046FFF746FF218A05460F98A5
:10E4800005F034F8238A023028449842BFD82B463E
:10E49000E2680F992046FFF736FF814617B3218ABD
:10E4A000384605F023F809F102031844238A9842FC
:10E4B000ADD84B46E26839462046FFF724FF814637
:10E4C00086B1218A304605F011F809F1020318449B
:10E4D000238A98429BD84B46E26831462046FFF794
:10E4E00012FF8146A9F105039BB2E2681021204684
:10E4F000FFF7D1FE01F0C4FCC4E906004FF47A75C1
:10E50000A06803689B68984758B901F0B9FCE369B3
:10E51000C01AA38A6B439842F2D36FF00303E363FC
:10E5200075E70DF107012046FFF7ECFD04287FF4A5
:10E530006EAFE368DD785DB901F0A2FC4FF0010831
:10E54000E06184F82050E563404604B0BDE8F08700
:10E55000E5635CE700044D515489010010B586B0B5
:10E56000012404940B9C03949DF8284002949DF888
:10E5700024400194089C0094FFF7F8FE06B010BDFB
:10E580002DE9F3470446FFF7D3FE8046D0B101F0F2
:10E5900077FC628A4FF47A735343E269821A9A4293
:10E5A000074603D8A269821A93421FD294F82030FA
:10E5B00063B16FF00303A068E36303685B6A984785
:10E5C0004FF00008404602B0BDE8F087E268C02185
:10E5D0001170E2685370A068E168036802225B680A
:10E5E0009847C4E90677012384F82030A0680368BF
:10E5F0009B6898470028E5D00DF107012046FFF7FA
:10E6000081FD83B20646002B73D0E368E7611A7878
:10E6100002F0F002302A57D1626A002AD2D09DF867
:10E6200007209918901C49781D5C05EB0125ADB2B7
:10E63000D11C19442A46184403F056FFE3689DF89C
:10E6400007202B44134400229A70E1689DF807C00C
:10E6500091F8009009F00609B2B20CF10200B9F18C
:10E66000020F0844666A0CF10303A2EB0C0225D1E9
:10E670002B440CF1050C11F803E00B44521B93F8EA
:10E6800001A06544053A29440AEB0E2AB047E36825
:10E6900040221A70E36883F80190E3681FFA8AFA4F
:10E6A0004FEA2A229A70E36883F803A0A068E16821
:10E6B000036804225B689847A76183E72B44033A09
:10E6C000521B1944B0477DE7C02A0BD1D0221A70E3
:10E6D000E36800225A70A068E168036802225B6860
:10E6E00098476FE7D02A7FF46DAF002384F820307D
:10E6F00068E72046FFF71CFE002808BF4FF000081F
:10E7000060E770B590B005460E46FFF711FEE0B128
:10E71000304604F0A8FE3123C4B28DF80030A31CAB
:10E720008DF801303B220023314601A88DF80230DC
:10E730008DF8034004F0C5FE2B68221D5B68694616
:10E7400028469847003018BF012010B070BD2DE951
:10E75000F0470446884617461D469DF82060FFF79F
:10E76000E7FD50B3B4F810904046494604F0BEFEB1
:10E77000EB1D1844814520D341460523E26820461D
:10E78000FFF7C1FD00211FFA81FC4318AC459BB285
:10E79000E26801F1010104D217F80CC002F803C0CD
:10E7A000F1E7002EA3F1050320469BB214BF3121EF
:10E7B0003021BDE8F047FFF76EBD0020BDE8F087CF
:10E7C00073B505460E4614466AB1018A104604F038
:10E7D0008DFE034600220092314622462846FFF76E
:10E7E000B6FF02B070BD1346F4E7F7B505460E4616
:10E7F0001F46144662B1018A104604F077FE0346B4
:10E800000097224631462846FFF7A1FF03B0F0BD2E
:10E810001046F4E72DE9F0470446884692461E4626
:10E82000FFF786FD002843D0218A404604F05EFEB3
:10E830009DF82030002BE3680CBF3022312287B2D4
:10E840001A70B21C3A44012002F07F01E568D20937
:10E8500018BF41F08001431C29545FFA80F9D2B9F6
:10E8600041469BB2E2682046FFF74DFDA368E16890
:10E870001A68D2F8048002461846C04755468046BA
:10E88000B244AA4509D0A06815F8011B03681B68AB
:10E8900098478044F5E71846D6E701F0F1FAA06101
:10E8A00009F1030038443044A0EB080358425841B2
:10E8B000BDE8F087F7B505460E461F46144662B11F
:10E8C000018A104604F012FE0346009722463146A4
:10E8D0002846FFF79FFF03B0F0BD1046F4E7F8B5F8
:10E8E00005460E4614461F46FFF722FD28B3314663
:10E8F0000523EA682846FFF706FD631F002F03443F
:10E900000CBF3021312106469BB2EA682846FFF74A
:10E91000A0FC0146A868EC680368053E0E44C1F1FE
:10E9200005015B68214432469847044601F0A8FA85
:10E93000A861A0B2831B58425841F8BD70B50D467E
:10E940000446018A2846164604F0D0FD45B3012E40
:10E9500026D8238A0930834222D32046FFF7E8FCD9
:10E96000F0B1E38A01339BB2C3B1E382E38AE26888
:10E970001B125371E368E28A9A71E2682946072301
:10E980002046FFF7C0FCE3681E54031FE2682046E0
:10E990009BB28221BDE87040FFF77DBC0123E4E714
:10E9A000002070BD0022FFF7C9BF70B50D460446B8
:10E9B000018A284604F09AFD25B3238A0930834250
:10E9C00020D32046FFF7B4FCE0B1E38A01339BB2C9
:10E9D000B3B1E382E38AE2681B125371E368E28A0F
:10E9E0009A71E268294607232046FFF78CFC431FF3
:10E9F000E26820469BB2A221BDE87040FFF74BBC05
:10EA00000123E6E7002070BD016382867047416202
:10EA10007047C06B704738B504460D4609B90020F1
:10EA200038BD038A4BB9084603F022FDE060E06878
:10EA30002582003018BF0120F2E7C06804F0F0FB27
:10EA40000028F3D1EBE7000070B50C4B002504461D
:10EA5000456040F8283B0E4600F0C6FB4FF0FF3300
:10EA6000E363A660A56325824FF480712046FFF71B
:10EA7000D2FF0F236382A382204670BDC4880100A9
:10EA800007B5002300931A461946034800F0B4FB6B
:10EA900003B05DF804FB00BFD80700208271054A6F
:10EAA000417112680449B2FBF1F14FF47A724A43A2
:10EAB000C26070471800002040420F0038B504467D
:10EAC0000D464079022101F0A1FB01F0D9F9A0F532
:10EAD000FA60A060657438BD70B505460E46002426
:10EAE000687901F0CDFBB042A3B206D1EA689A4240
:10EAF00004F10104F4D84FF0FF33184670BD30B56F
:10EB00000D46D1B0044601F0BBF93DB9A368C31A64
:10EB1000B3F5FA6F02D2207C51B030BD002502213E
:10EB2000A06025606079257101F070FB012001F083
:10EB3000DBF90121607901F069FB2946607901F078
:10EB40008DFBA379153B012B00F28C8040F24C40E9
:10EB5000013800BF00BF00BF00BF00BF00BF00BF43
:10EB600000BF00BF00BF00BF00BF00BF00BF00BFAD
:10EB700000BF00BF00BF00BF00BF00BF00BF00BF9D
:10EB800000BF00BF00BF00BF00BF00BF00BF00BF8D
:10EB900000BF00BF00BF00BF00BF00BF00BF00BF7D
:10EBA00000BF00BF00BF00BF00BF00BF00BF00BF6D
:10EBB00000BF00BF00BF00BF00BF00BF00BF00BF5D
:10EBC00000BF00BF00BFC3D16079022101F01EFB6E
:10EBD000607C00283BD0013800BF00BF00BF00BFF1
:10EBE00000BF00BF00BF00BF00BF00BF00BF00BF2D
:10EBF00000BF00BF00BF00BF00BF00BF00BF00BF1D
:10EC000000BF00BF00BF00BF00BF00BF00BF00BF0C
:10EC100000BF00BF00BF00BF00BF00BF00BF00BFFC
:10EC200000BF00BF00BF00BF00BF00BF00BF00BFEC
:10EC300000BF00BF00BF00BF00BF00BF00BF00BFDC
:10EC400000BF00BF00BF00BF00BF00BFC3D172B68E
:10EC500000212046FFF740FF013007D1002020743B
:10EC600062B659E7142001F03FF9ADE701212046D3
:10EC7000FFF732FF0130F1D0002500212046FFF7D9
:10EC80002BFF01214DF805002046FFF725FF0DEB76
:10EC900005030835B5F5A07F5860EED162B60022B5
:10ECA0005DF832500DEBC203691C586801D0431C5B
:10ECB00002D1002020742FE7D1108542635C4FEA17
:10ECC0004303DBB202F1010238BF43F00103282AFB
:10ECD0006354E5D16178237822790B44A1780B4401
:10ECE000E1780B44DBB29A42E3D10120E2E7000075
:10ECF0002DE9F8430D462DED028B11460446FFF732
:10ED0000FEFE00287ED0A3790B3B0B2B7AD8DFE8E0
:10ED100003F0063F79797979797979796565A3780E
:10ED2000E07808EE103A0106B8EE488A48BFFFEED8
:10ED3000007A00F00F0048BF37EEC88A02F094FD59
:10ED400031A3D3E9002302F0F9FD064618EE100ABC
:10ED50000F4602F09BFD0B4602463946304602F054
:10ED600037FC03F0E3F803466DB102F08FFD2AA3F0
:10ED7000D3E9002302F0E2FD254B002202F028FC3B
:10ED800003F0D4F80346BDEC028B1846BDE8F883C7
:10ED9000E078A67800F00F0002F066FD1AA3D3E930
:10EDA000002302F0CBFD07EE906AF8EE677A80460A
:10EDB00017EE900A894602F069FD02460B4640466E
:10EDC000494602F005FC03F0B1F83206034648BF9D
:10EDD00080F00043002DD6D01846C6E7A678E37829
:10EDE000300200F4FE40184307EE900AF8EEE77A8E
:10EDF00017EE900A02F04AFD03A3D3E9002302F0C4
:10EE00009DFDE0E7034BBEE79A9999999999B93F1F
:10EE1000000040400000C07FCDCCCCCCCCCCFC3F2F
:10EE2000D0B50446FFF76BFE90B3A3790B3B0B2BD9
:10EE30002ED8DFE803F006062D2D2D2D2D2D2D2D9E
:10EE40001C1C607802F010FD14A3D3E9002302F02B
:10EE500075FD064620780F4602F006FD02460B4679
:10EE60003046394602F0B4FB03F060F8D0BD20888C
:10EE700040BA80B207EE900AF8EEE77A17EE900AF1
:10EE800002F004FD05A3D3E9002302F057FDEBE7F0
:10EE90000148EBE7AFF300800000C07F9A99999991
:10EEA0009999B93F10B50446C06803F0E9FAB4F97E
:10EEB0000600002802DB002101F0A8F9204610BD61
:10EEC00070B50546C0680E4603F0DAFAEC7C2A7C81
:10EED00094420CBF0324042414FB06F4A4B2AC80B7
:10EEE000204603F0C5FAE86028B12246002103F06D
:10EEF00014FB6E8070BDA8806880FBE7F0B4FF292A
:10EF0000C1F38107C1F38112C1F30115477401F008
:10EF100003078CBF002101210170C168C47C067CFD
:10EF2000C2740574877461B1A41B6142A2EB05052C
:10EF300061416A426A41914203D04188F0BCFFF7C7
:10EF4000BFBFF0BC704738B5437804460D4633B1B7
:10EF5000B0F90600002802DB002101F057F96378C0
:10EF6000E5804BB12846012101F050F928460021E7
:10EF7000BDE8384001F072B938BD70B50E460021C9
:10EF8000044641700172C160416119461546FFF7A0
:10EF9000B5FF31462046FFF793FF20462946FFF78D
:10EFA000D2FF204670BD70B540F2FA5404FB00F366
:10EFB00003F500431B14B3F5FF7F98B222DAFE2B52
:10EFC000D8B242DDC0F1FE00C5B20023FF204E1CC6
:10EFD000C943C9B27043013201EB2020504300F411
:10EFE0007F4406FB03F006FB05F301EB202001EB59
:10EFF000232150434A43120244EA102002F47F02C4
:10F00000104370BDB3F57F7F0DDAB0F53F7FDBB203
:10F010008BBFC3F1FC030233D8B2DBB294BFFF2035
:10F02000FF230025D3E7A04211D040F2FA44A042CA
:10F03000DBB204D80433DDB20020FF23C7E7C3F1FD
:10F04000FA03DBB20020FF25C1E70023FBE7002322
:10F050001846F8E770B50446083015460E4600F02D
:10F06000C3F8FF23064A84F8223000232660257166
:10F070002361A382C4E906222384204670BD00BF19
:10F08000EB8D01000161828270470000024B002974
:10F0900008BF194681617047EB8D0100024B0029C2
:10F0A00008BF1946C1617047EB8D010001847047AC
:10F0B00073B50D4601690446164639B92B4BC26833
:10F0C0005B689A4202D1002002B070BDA28A002A79
:10F0D000F9D094F8223005F007000341DB0738D55A
:10F0E00015F47E7F08BF238C206804BF03F47E7371
:10F0F0001D43036800292ED05B6A98470128E2D19E
:10F100003C21206800F0CDF80A222946206800F052
:10F1100024F9237933BB1649206800F0B5F8A169BA
:10F12000206800F0BAF82021206800F0BAF8E16900
:10F13000206800F0B2F82379B3B90E49206800F0D6
:10F14000A3F83146206800F0A8F8206803689B6A9D
:10F1500098470120B8E708490091E16801911B6ACE
:10F160006946CAE70549D7E70549E7E7E007002010
:10F17000CC880100D2880100548901005770010039
:10F18000DD88010008B5FFF793FF08BD07B5002330
:10F1900000931A461946034800F02EF803B05DF8B4
:10F1A00004FB00BFE00700202DE9F84306460D46AA
:10F1B000071D00F10709002417F8011B0A22284641
:10F1C00000F0E4F82E218046284600F06AF84F450A
:10F1D00040440444F0D10A22F179284600F0D6F8E0
:10F1E0002044BDE8F8830000024A02600022426029
:10F1F000704700BF5489010030B58371034D9DF8FD
:10F200000C30056001714271C37130BD5489010039
:10F21000014AC0E90021704754890100024A026096
:10F220000A684260704700BF548901000B68436060
:10F230007047416070472DE9F04106460D4601EBED
:10F2400002080C464445A4EB050707D0336814F8C0
:10F25000011B1B68304698470028F3D13846BDE8AB
:10F26000F08170B5044608460D4604F0FCF82368AA
:10F270000246294620465B68BDE87040184709B140
:10F28000FFF7EFBF0846704708B5FFF7F8FF08BD66
:10F2900003688A685B680968184708B5FFF7EFFFDD
:10F2A00008BD03681B6818470149FFF7DABF00BFB4
:10F2B000A888010038B50546FFF7E1FF0446284657
:10F2C000FFF7F2FF204438BD38B50546FFF7D7FFFA
:10F2D00004462846FFF7E8FF204438BD70B58AB0E1
:10F2E0000D460AA9002301F8043D012A98BF0A220D
:10F2F000B5FBF2F402FB1456F3B2092E94BF30337F
:10F300003733DBB2254601F8013D002CF0D1FFF781
:10F31000B6FF0AB070BD2DE9F04107460E4615460E
:10F320002AB90368C9B21B68BDE8F04118470A2A28
:10F3300005D1002905DBBDE8F041FFF7CFBFD2B210
:10F34000F9E72D21FFF7ADFF2A4604467142384602
:10F35000FFF7C4FF2044BDE8F081FFF7DCBF38B5FC
:10F360000546FFF7D8FF04462846FFF79DFF2044D7
:10F3700038BD10B42AB903685DF8044B1B68C9B2E4
:10F380001847D2B25DF8044BFFF7A8BFFFF7F1BFF3
:10F39000FFF7EFBF2DE9F84F194606461046144611
:10F3A0001D469DF8287002F063FD28B14C49304697
:10F3B000BDE8F84FFFF755BF25F000494FF0FF3289
:10F3C000484B2046494602F053FD48B94FF0FF3202
:10F3D000444B2046494602F02DFD08B94249E6E774
:10F3E0004FF06042414B2046294602F037FD08B1FC
:10F3F0003F49DCE74FF060423E4B2046294602F091
:10F400000FFD0028F4D1002200232046294602F0F7
:10F4100007FDD0B12D213046FFF743FF05F1004332
:10F4200082461D463449DFF8D8904FF0000B00208B
:10F430004FF000085FFA8BF39F4208D942464B46D3
:10F4400002F0A6FB0BF1010BF4E78246EAE7224645
:10F450002B4602F0BDF80D46044602F047FD0A2295
:10F46000014680463046FFF739FF8244A7B3404645
:10F4700002F0EAF902460B462046294602F0A6F8B9
:10F4800004460D4630461D49DFF87490FFF7E9FE4B
:10F490004FF000088244013FFFB2FF2F1CD04B46C3
:10F4A00042462046294602F049FA0D46044602F03B
:10F4B000F5FC0A22014683463046FFF72CFF8244C2
:10F4C000584602F0D1F902460B462046294602F082
:10F4D0007DF804460D46DEE75046BDE8F88F00BFD4
:10F4E00058890100FFFFEF7F5C890100FFFFEF41BA
:10F4F00060890100FFFFEFC10000E03F9C80010038
:10F50000000024409DF800100091FFF743BF08B5AC
:10F510004022002103F001F80022C0E9102208BDBA
:10F52000026C10B5531C446C03F03F039C421CBF9B
:10F530008154036410BD0023C0E910337047D0E943
:10F54000102393421FBFC25C013303F03F034364A7
:10F5500014BF10464FF0FF307047D0E91030181A32
:10F5600048BF40307047D0E91023934214BFC05CBD
:10F570004FF0FF307047036C406C013303F03F03E2
:10F580001B1A5842584170470649074A074B9B1AB5
:10F5900003DD043BC858D050FBDC00F037F8F0F72F
:10F5A0004FFE0000FC8D010000000020A40200209E
:10F5B000FEE7FEE7FEE7FEE7FEE7FEE7FEE7FEE723
:10F5C000FEE7FEE7044B1868421C04BF034B1878A3
:10F5D000831F58425841704730010010E00F00F07F
:10F5E000074B1B78062B09D1064B1B68C3F303138B
:10F5F000033B032B02D8044AD05C704700207047BD
:10F60000E00F00F0E80F00F06889010008B5FFF78F
:10F61000D9FF28B1654B664A1B68C3F30423136006
:10F62000FFF7DEFF10B1634B634A1A60FFF7CAFFB2
:10F6300028B1624B624A1B68C3F342331360FFF781
:10F64000CFFF20B15F4AD36823F08073D360FFF708
:10F65000B9FF40B14FF080430022C3F80C21C3F83A
:10F660001021C3F83825FFF7BBFF10B1564B03221A
:10F670001A60FFF7B5FF40B1544B05221A60012212
:10F680009A6700229A603F225A60514B1A68511CB7
:10F690000BBF504B504B1A781B6802BF08331B68D6
:10F6A000C3F30313062A4DD1033B032B03D84B4A64
:10F6B000D35C002B46D04FF08052494BD2F8041453
:10F6C000C3F82015D2F80814C3F82415D2F80C1486
:10F6D000C3F82815D2F81014C3F82C15D2F8141456
:10F6E000C3F83015D2F81814C3F83415D2F81C1426
:10F6F000C3F84015D2F82014C3F84415D2F82414E6
:10F70000C3F84815D2F82814C3F84C15D2F82C14B5
:10F71000C3F85015D2F83014C3F85415D2F8341485
:10F72000C3F86015D2F83814C3F86415D2F83C1445
:10F73000C3F86815D2F84014C3F86C15D2F8442405
:10F74000C3F87025FFF73EFF28B1264B264A1B68F9
:10F7500003F04F031360FFF735FF48B14FF08043CC
:10F76000D3F80024D20744BF6FF00102C3F800248D
:10F77000174B1B68062B09D1174B1B68033B022B49
:10F7800081BF1A4A136843F480631360184AD2F8A1
:10F79000883043F47003C2F88830BFF34F8FBFF353
:10F7A0006F8F144B144A1A6008BD00BF2403001069
:10F7B0004035014074C007400DF0ADBA440200105E
:10F7C0003C050040F0ED00E0A00500401056004070
:10F7D00030010010E00F00F03401001064890100D6
:10F7E00000C0004058020010E40E00403C170040EA
:10F7F00000ED00E0180000200090D00310B5044692
:10F8000000F03EFBE06023682046DB689847002854
:10F8100008DA00F035FBE368C01AA3689842F2D317
:10F820004FF0FF3010BD2DE9F04180460D468F1896
:10F830000C46BC42A4EB050607D04046FFF7DEFFAE
:10F84000002802DB04F8010BF3E73046BDE8F08145
:10F850002DE9F8438046894616461C467BB1D718E9
:10F860001546BD42A5EB060409D04046FFF7C6FF8A
:10F87000002804DB814502D005F8010BF1E72046A2
:10F88000BDE8F88370B50D4609490446164600F0F8
:10F89000D1F92846FFF7B2FF002806DB864204D0E4
:10F8A000C1B2204600F044FAF3E7204670BD00BF25
:10F8B000AA8801000120704703681322DB691847FA
:10F8C00070470369C3F81C150369D3F81C21002A8B
:10F8D000FBD00022C3F81C210120704710B490F91E
:10F8E0005C30144C59090122203103F01F0302FA45
:10F8F00003F344F8213003695DF8044B0421C3F895
:10F90000081303695A600369DA6003690022C3F8C7
:10F91000002502694FF0FF33C2F80C350269C2F8C6
:10F9200014350269C2F8083502691430C2F810357E
:10F93000FFF701BE00E100E01430FFF70EBE143007
:10F94000FFF711BE1430FFF7FABD0000036990F80D
:10F950005E2010B5C3F80C25036990F85D20C3F84C
:10F96000142590F861200369012A01BF90F85F40D7
:10F97000C3F81045036990F8604006BFC3F8084516
:10F9800003690022B1F5966FC3F86C2569D9B1F50A
:10F99000166F69D9B1F5965F69D9B1F5165F68D967
:10F9A000B1F5615F67D9B1F5964F66D9B1F5E14F11
:10F9B00065D9B1F5164F64D9B1F5614F64D9B1F588
:10F9C000963F64D9B1F5E13F63D9B1F5613F63D9A1
:10F9D000364B994263D9B1F5E12F63D9B1F5612F67
:10F9E00094BF4FF070634FF080530269C2F8243522
:10F9F00003690422C3F8002501690023C1F8083116
:10FA00000169C1F81C31016901230B6001698B6038
:10FA10000169C1F8042390F95C20510902F01F022A
:10FA200093406031224A42F8213090F95C30002B3B
:10FA3000BDBF03F00F0302F6FC32D2189B18B5BF0E
:10FA400060236022137683F8002390F95C30012252
:10FA5000590903F01F0302FA03F3154A42F8213053
:10FA600010BD4FF49E23C0E74FF41D23BDE7114B9B
:10FA7000BBE7114BB9E7114BB7E7114BB5E7114B9A
:10FA8000B3E74FF41D03B0E74FF46B03ADE70E4B44
:10FA9000ABE74FF0EB73A8E74FF06C73A5E74FF0BF
:10FAA0008063A2E74FF0E8639FE700BF90D00300B8
:10FAB00000E100E000B013000050270000F03A0021
:10FAC00000A04E0000C0750000903A012DE9F04101
:10FAD0001E4600254FF47A73C0E901530D4B0446CE
:10FAE00040F8143B17468846FFF711FD0A4AC4F850
:10FAF000108084F85C7052F8263084F85D309DF8F0
:10FB0000183052F8233084F85E3084F86150204673
:10FB1000BDE8F08174890100E488010010B5036933
:10FB2000D3F8082104464AB1D3F818151430C9B2E5
:10FB3000FFF7F6FC23690022C3F8082110BD00007E
:10FB40000148FFF7EBBF00BFE807002007B5192306
:10FB500000930222182303490348FFF7B7FF03B0BD
:10FB60005DF804FB00200040E807002010B50446C3
:10FB700028B103F021FB90FBF4F303FB14042046AF
:10FB800010BD884210B5044603DA081AFFF7EEFFED
:10FB90000444204610BD10B5029C401AE41A60438C
:10FBA000521A90FBF2F0184410BD10B504460068DC
:10FBB00002F066FC204610BD10B50446006808B18E
:10FBC00002F05EFC00232360C4E9013310BD38B5A8
:10FBD00004460D460068013103F022FB10B1C4E970
:10FBE0000005012038BD036810B5044623B1436801
:10FBF0008B4201D3012010BD2046FFF7E8FF00280B
:10FC0000F9D0A368002BF5D122681370F2E770B524
:10FC10000E46114604461546FFF7E5FF20B920467B
:10FC2000FFF7CAFF204670BDA5603146206803F08B
:10FC3000F6FBF7E738B500230446C0E900338360DC
:10FC40000D4639B1084603F00EFC2946024620460F
:10FC5000FFF7DDFF204638BD38B5054608460C469F
:10FC600003F001FC214602462846BDE83840FFF774
:10FC7000CEBF38B5054600680C4668B16A688B6827
:10FC80009A4207D3096803F0CAFBA368AB6000235C
:10FC9000A36038BD02F0F4FB23682B6063686B60DF
:10FCA000A368AB600023C4E90033F1E7884210B5D4
:10FCB0000B46044604D0096821B19A68FFF7A7FFF4
:10FCC000204610BDFFF778FFFAE710B50023044681
:10FCD000C0E900338360FFF7E9FF204610BD88428A
:10FCE00010B5044601D0FFF7C4FF204610BD10B583
:10FCF000044619B1FFF7B0FF204610BDFFF75CFFC7
:10FD0000FAE770B505460E4609B9002070BD6AB124
:10FD1000846814442146FFF766FF0028F5D0286860
:10FD2000AB683146184403F07AFBAC600120EDE784
:10FD300007B500238DF80410012201A98DF80530C4
:10FD4000FFF7DFFF03B05DF804FB10B58A680968B0
:10FD50000446FFF7D6FF10B92046FFF72DFF2046D7
:10FD600010BD826808B53AB921B10878B0FA80F0C0
:10FD7000400900E0012008BD006809B90078F5E7F6
:10FD800003F043FBF2E7884270B515D083688A68B8
:10FD900093420FD183B104680D68013C14F8010F40
:10FDA00050B104F075FB064615F8010B04F070FB2A
:10FDB0008642F3D0002070BD0120FCE783688B42AF
:10FDC00001D9006818B9034800230370704708443C
:10FDD000704700BF4C0800208368934210B506D9D5
:10FDE0000468A01803F004FB08B1001B10BD4FF01D
:10FDF000FF30FBE70022FFF7EFBFF8B583689342BF
:10FE0000054602D84FF0FF30F8BD0368541C0022AD
:10FE10001F5D1A550668304603F074FB37550028FD
:10FE2000F0D02B68C01AEFE78268013AFFF7E5BF10
:10FE30002DE9F0419A420E461F460F4988BF1346EE
:10FE40001546804684BF3D461F46FFF7F3FEB46863
:10FE5000AC420DD9BC4228BF3C46336800221F5D2E
:10FE60001A55316840462944FFF741FF33681F5552
:10FE70004046BDE8F08100BFAA880100FEE700000F
:10FE80000A4B19680A4B30B5D3F804050C060D0A65
:10FE900044EA00024FF47A712B46A2FB014501FBB4
:10FEA0000355E00B40EA454030BD00BF500800203C
:10FEB00000100140094B1968094B30B5D3F804050F
:10FEC0000D0A0C06074944EA00022B46A2FB014535
:10FED00001FB0355E00B40EA454030BD50080020CF
:10FEE0000010014040420F0038B5044648B1FFF70A
:10FEF000C7FF054600F01AF8FFF7C2FF401BA042FB
:10FF0000F8D338BD074B0022C3F8042182B0D3F8E0
:10FF10000431054A0193019B13680133DBB213607E
:10FF200002B0704700100140500800207047704731
:10FF300008B500F017F8FFF7FAFF0120FFF7D4FF2C
:10FF4000F5F7B4F9034CF5F7B3F9002CFBD0AFF398
:10FF50000080F8E70000000002F08ABA02F088BAD8
:10FF600002F08EBA2A4BE02283F811234FF40032BC
:10FF7000C3F880211A604FF080430122C3F818258E
:10FF80009A6003F588330021C3F808150221C3F8ED
:10FF90000413C3F844131A604FF01023D3F800225F
:10FFA000002A03DBD3F80432002B2FDA194B01228D
:10FFB000C3F80425D3F80024002AFBD04FF0102208
:10FFC0001521C2F80012D3F80024002AFBD04FF00C
:10FFD00010231522C3F804220E4B1A46D3F800143E
:10FFE0000029FBD00021C3F80415D2F80034002BFF
:10FFF000FBD0BFF34F8F0849084BCA6802F4E06298
:020000021000EC
:100000001343CB60BFF34F8F00BFFDE7704700BFC6
:1000100000E100E000E0014000ED00E00400FA052E
:10002000192837B50CD84B4B53F82030052B00F06E
:10003000828007D8032B12D07BD8022B00F081805E
:10004000002074E01D2B78D003D81C2BF8D105229A
:1000500006E01E2B73D01F2BF2D1082200E00222F3
:100060003D4B196808296EDD0A296FDD0D29B5BFE2
:100070000C240E24022303233848C0F8F035012352
:10008000C0F8003500200546030103F1804303F565
:10009000E04301300828C3F81455C3F81055F3D1D4
:1000A0002F4B18682F4B1B6800021B0303F480536F
:1000B00000F4E0601843294BC3F81805C3F8142571
:1000C000C3F810250DF10602C3F82C260122C3F84F
:1000D00030261A60D3F80021002AFBD00022C3F892
:1000E000002101225A601D4B1A46D3F80401002852
:1000F000FBD00020C3F8040101209860D2F814312D
:10010000002BFBD00023C2F81431BDF906209A421F
:10011000124AB8BFADF80630A142C2F80035BDF9A9
:10012000060004D035BF611A091BC840884003B0DF
:1001300030BD032294E7042292E7062290E70722CB
:100140008EE701228CE70824002395E70A24012387
:1001500092E700BFE4880100280000200070004002
:100160002C0000205C080020192830B53CD8224B18
:1001700053F82000214B00221D4653F82240B4F1D1
:10018000FF3F32D11E4C45F822006FEA41411D4D20
:100190001D4B246853F822306FEA514125F81210A4
:1001A000012101FA04F4C3F86005013CC3F86405B9
:1001B00005EB4202C3F86805C3F86C050020C3F8DC
:1001C0000015C3F80C05C3F80405C3F80845C3F8C7
:1001D0001405C3F81005C3F82025C3F82415C3F887
:1001E0002815C3F82C05996030BD8442CAD001326D
:1001F000032AC2D1F8E700BFE48801001C000020F8
:1002000030000020540800209C89010019280FD8D4
:10021000114B53F8203003290AD8DFE801F0021609
:100220000A1003F5E0734FF0A042002142F82310BA
:10023000704703F5E0734FF0A0420C21F6E703F599
:10024000E0734FF0A0420421F0E703F5E0734FF0B4
:10025000A0420321EAE700BFE488010019280CD876
:10026000064B53F82020012393404FF0A04211B9D0
:10027000C2F80C357047C2F808357047E4880100B1
:1002800019289FBF4FF0A043054AD3F8103552F804
:1002900020009ABF23FA00F000F001000020704710
:1002A000E488010038B50025057329B90B4B0C4AC9
:1002B0000C48252101F08AFE01600B4951F82220EB
:1002C000027151F8233083719DF8103051F82330BA
:1002D00043710223C371856038BD00BFA889010046
:1002E0000B8A0100B6890100E4880100037B23B971
:1002F00043738373036101230373704784B00DF16B
:10030000100C0CE90E009DF808100268002301296A
:10031000C2F80035039B12D00BD303290CD0C2F8CE
:100320005435019BC2F824350123C2F8003504B0CE
:10033000704743F00203F2E743F00403EFE743F0B2
:100340000603ECE710B5FFF7D1FF03688279C3F825
:1003500008254279C3F80C250279C3F81025034B10
:10036000BDE810400ECBFFF7C9BF00BF74080020E6
:1003700010B485B001AC84E80E0094E80E0005B01E
:100380005DF8044BFFF7BABF70470368C3F81C154C
:10039000D3F80821002AFBD0D3F818050022C3F8AF
:1003A0000821C0B27047000007B5094B09490A4847
:1003B0004FF080421A6000229A6002221A710B23C9
:1003C00000930C220D23FFF76DFF03B05DF804FBD3
:1003D0007408002000300240600800200B460146EF
:1003E000184601F01DBE0000C0F3C7537F3B162B1B
:1003F000024605DC002B04DB0348184122EA00001A
:10040000704700F000407047FFFF7F0000000000D1
:100410002DE9F04FDFF82C938DB006460F461446B9
:100420001D4600F095F999F90080B8F1FF3FCDE93C
:10043000000136D022462B462046294601F018FD01
:10044000834670BB32463B463046394601F010FDCC
:100450008246002840F0A280304639460022002320
:1004600001F0D4FC10B3002200232046294601F0FD
:10047000CDFC8346002867D09FEDA77B0122AC4BC3
:10048000CDF828A00292CDE90467CDE906458DEDAF
:10049000087B0393B8F1000F41D09FEDA17B8DED58
:1004A000007BDDE900010DB0BDE8F08FDDE9000162
:1004B00000F066FF8046002800F08D804FF0000AB3
:1004C0004FF0000BDDE9000152465B4601F09EFC57
:1004D0000028E6D03046394600F052FF0028E0D030
:1004E0002046294600F04CFF0028DAD099F9003068
:1004F0008F4A039204210022022BCDE90467CDE943
:100500000645CDE908AB02910A9203D002A800F09B
:100510003DFF50B901F092FD2223036005E002A8DF
:1005200000F034FF002800F09B800A9B1BB101F013
:1005300085FD0A9B03609DED087B8DED007BDDE969
:1005400000010DB0BDE8F08F2046294600F018FFED
:100550000028A6D0002200232046294601F060FC96
:1005600000289ED0724A99F90030CDF828B00121B8
:10057000CDE90467CDE90645CDE90212002B74D020
:100580006C490020022BCDE9080172D101F056FD23
:10059000212303600A9B002BCDD0C8E70022002353
:1005A0002046294601F032FC00283FF47AAF624B26
:1005B0005F49CDF828B000220120B8F1020FCDE943
:1005C00004670290CDE90645CDE908230391A6D141
:1005D000CDE9002365E73046394600F0D1FE00281A
:1005E0003FF46CAF2046294600F0CAFE00283FF4D5
:1005F00065AFDDE900231046194601F039FC99F991
:1006000000A000286BD10323DFF824C10A902946FB
:10061000204602930022494BCDF80CC0CDE9064597
:10062000CDE9046701F08AF904460D46BAF1000FDE
:1006300025D1DFF814B14FF0604A00220023304684
:100640003946CDE908AB01F0EBFB38BB02A800F05E
:100650009DFE00289ED101F0F1FC2223036099E762
:1006600001F0ECFC212303605FE79FED2B7B8DED18
:10067000087B02A800F08AFE00288BD186E79FED58
:100680002A7B00220023304639468DED087B01F09D
:10069000C7FBA0B9BAF1020FDDD0D7E72046294643
:1006A00000F07CFE22462B4601F0B0FBA0B9244BA3
:1006B00099F900A04FF06042CDE90823EAE720460F
:1006C000294600F06BFE22462B4601F09FFB18B92D
:1006D000184B0022CDE9082399F900A0DAE701229E
:1006E000134BCDF828800292CDE90467CDE9064589
:1006F0000393BAF1000FB8D0002200231046194628
:1007000001F046FABAF1020FCDE908013FF43EAF1D
:10071000AFE700BFAFF30080000000000000000062
:10072000000000000000F03F000000000000F07F2B
:10073000488A01000000F0FF0000F03F0000E03FA9
:10074000FFFFEFC734000020FFFFEF47000000006D
:100750002DE9F04F23F0004555EA020493B00DD087
:100760006B4E21F00044B4420F4682460BDD04F18B
:10077000404404F5801454EA0A0350D1654900202E
:1007800013B0BDE8F08F9B46944647D0B542EEDCEF
:100790005F4EB5425DD0002F80468946CDE90023EB
:1007A0005BDB0026BCF1000F0ED1594B9D423FD0C0
:1007B000584B9D4200F08880BBF1804F00F09C8038
:1007C000554B9B4500F0B8834046494600F0D4FDA8
:1007D000BAF1000F06D1002C59D04E4B27F0404201
:1007E0009A4254D0FF0F013F56EA070373D04B4B98
:1007F0009D4240F39B8003F104739D4240F33E848D
:10080000474B9C4272DDBBF1000F72DD3EA3D3E982
:1008100000231046194601F091F8B1E728B141488C
:1008200013B0BDE8F04F00F0B3BDA542F7DCAFE771
:1008300004F1404303F5801353EA0A039ED0384B7A
:100840009C4240F38383BBF1000F52DBDDE90001E2
:1008500096E7BCF1000F9ED089E7334B9D4231DC17
:10086000A3F154739D429CDD2B15A3F2FF33142B8F
:1008700040F3A583C3F134032CFA03F202FA03F325
:1008800063458ED102F00102C2F102068AE7BBF194
:10089000000F05DA02460B4600201E4901F078F9E8
:1008A000002FBFF66DAF04F1404404F5801454EA04
:1008B000060300F03F84012E7FF462AF01F1004394
:1008C00019465DE702266DE7BBF1000FC0F24883D1
:1008D0004046494654E742464B461046194600F00A
:1008E00075FE02460B4601F053F949E7BBF1000FD4
:1008F0008CDB0020002143E742464B4640464946F8
:1009000001F01CF83CE700BF9C7500883CE4377E92
:100910000000F07F0000F03F0000E03F0000E041F9
:10092000FFFFEF3F4C8A0100FFFF3F43B4F5801FFC
:1009300080F261830022D24B01F000F86FF0340C9A
:100940000C462315CF4DC4F31302A3F2FF3342F03C
:100950007F546344AA420B9344F4401440F33F8312
:10096000C94B9A4240F304849FEDAF7B8DED087B29
:100970008DED107B9FEDAE7B0B9B8DED067B0133E8
:100980000B93A4F580140025DDE906232146824659
:1009900000F01CFEA346DDE906238046894650464A
:1009A0002146CDE90CAB00F013FE02460B460020B9
:1009B000B64901F0EDF80A460146CDE90E1213469C
:1009C00049460246404600F0B9FF631043F0005329
:1009D00082468B4603F500238C46CDE904AB5919BA
:1009E000D3460023CDE902BC0293DDE902AB00202F
:1009F00004460D4602460B465046594600F09EFFFF
:100A000002460B464046494600F0E0FDDDE906237C
:100A1000804689462046294600F0D8FD02460B460E
:100A2000DDE90C0100F0D2FD52465B4600F086FF86
:100A300002460B464046494600F0C8FDDDE90E235C
:100A400000F07CFFDDE90445CDE9060122462B4696
:100A50002046294600F072FF77A3D3E9002304461D
:100A60000D4600F06BFF76A3D3E9002300F0B0FD44
:100A700022462B4600F062FF73A3D3E9002300F067
:100A8000A7FD22462B4600F059FF71A3D3E90023AE
:100A900000F09EFD22462B4600F050FF6EA3D3E9E6
:100AA000002300F095FD22462B4600F047FF6CA383
:100AB000D3E9002300F08CFD2246804689462B4670
:100AC0002046294600F03AFF02460B46404649467A
:100AD00000F034FF524604460D465B46DDE9040152
:100AE00000F076FDDDE9062300F028FF22462B46C4
:100AF00000F06EFD5246804689465B465046594698
:100B000000F01CFF0022624BCDE90C0100F060FDFB
:100B100042464B4600F05CFD02980D4604462246D4
:100B20002B465046594600F009FF002282468B466C
:100B3000574B2046294600F049FDDDE90C2300F023
:100B400045FD02460B464046494600F03FFDDDE9C3
:100B5000042300F0F3FE2246804689462B46DDE959
:100B6000060100F0EBFE02460B464046494600F007
:100B70002FFD8046894602460B465046594600F0F6
:100B800027FD029838A3D3E9002304460D4600F060
:100B9000D5FE5246CDE904015B462046294600F0C9
:100BA00015FD02460B464046494600F00FFD30A3B6
:100BB000D3E9002300F0C2FE2FA3D3E9002380462F
:100BC00089462046294600F0B9FE02460B464046BB
:100BD000494600F0FDFCDDE9102300F0F9FC8046F9
:100BE0000B98894600F040FE424682468B464B46B3
:100BF000DDE9040100F0ECFCDDE9082300F0E8FC8D
:100C000052465B4600F0E4FC029852465B460446BE
:100C10000D4600F0DBFCDDE9082300F0D7FCDDE940
:100C2000042337E0AFF30080000000000000000064
:100C3000000000000000F03FEF4E454A287ECA3F0A
:100C400065DBC9934A86CD3F01411DA96074D13F40
:100C50004D268F515555D53FFFAB6FDBB66DDB3F52
:100C6000033333333333E33F000000E009C7EE3F83
:100C7000FD033ADC09C7EE3FF5015B14E02F3EBEF1
:100C8000000040438E98030079B60B000000F03F4F
:100C90000000084000F09AFC0B46024649464046D8
:100CA00000F094FC013E56EA070382468B4600F0B2
:100CB0005E819FEDD37B8DED047BDDE90012002387
:100CC0000E461746CDE902670293DDE90267084642
:100CD0003B461146324600F079FC22462B4600F096
:100CE0002DFEDDE90023804689465046594600F036
:100CF00025FE02460B464046494600F069FC324656
:100D0000804689463B4620462946CDE9008900F0C9
:100D100015FE0B46024606460F464046494600F081
:100D200057FCD14B994204460D468A4640F3248134
:100D300001F13F4303F5E003034340F0FF81B2A319
:100D4000D3E90023DDE9000100F042FC3246804691
:100D500089463B462046294600F038FC02460B46B1
:100D60004046494601F07AF8002840F0E781A8465D
:100D70004FEA2853A3F2FE324FF480131341534439
:100D8000C3F30A52B94DA2F2FF321541C3F3130463
:100D900023EA05010020C2F1140B44F48014BAF1D7
:100DA000000F02460B4644FA0BFB30463946B8BFEB
:100DB000CBF1000B00F00AFC06460F463246DDE997
:100DC00000013B4600F004FC4FEA0B5A0D4600249C
:100DD0008FA3D3E900232046294600F0AFFD324619
:100DE000804689463B462046294600F0EFFB0246F6
:100DF0000B46DDE9000100F0E9FB87A3D3E90023FE
:100E000000F09CFD86A3D3E9002306460F4620464A
:100E1000294600F093FD02460B463046394600F065
:100E2000D7FB06460F4602460B464046494600F0B1
:100E3000CFFB42464B4604460D4600F0C7FB024638
:100E40000B463046394600F0C1FB224680468946B3
:100E50002B462046294600F071FD73A3D3E90023F9
:100E600006460F4600F06AFD71A3D3E9002300F0A7
:100E7000ADFB32463B4600F061FD6FA3D3E9002392
:100E800000F0A6FB32463B4600F058FD6CA3D3E9C8
:100E9000002300F09BFB32463B4600F04FFD6AA367
:100EA000D3E9002300F094FB32463B4600F046FDB8
:100EB00002460B462046294600F088FB06460F46B0
:100EC00002460B462046294600F038FD0022CDE9B7
:100ED00000014FF080433046394600F077FB024670
:100EE0000B46DDE9000100F053FE424606460F4680
:100EF0004B462046294600F021FD42464B4600F075
:100F000067FB02460B463046394600F05FFB22463F
:100F10002B4600F05BFB02460B460020544900F0D4
:100F200055FB8A44BAF5801FC0F232815146DDE993
:100F3000042300F003FD23E4002FFFF645AC4046F8
:100F4000494613B0BDE8F04F00F056B9BBF1000FB1
:100F5000BFF6CFACDDE90034184604F100410FE4E0
:100F600042464B460020424900F012FE08E49FED45
:100F7000387B8DED047BA0E63E4B21F00048984580
:100F800040F3EA803C4B0B4403430AD132463B46D4
:100F900000F01CFBDDE9002300F056FF00283FF4C1
:100FA000E7AEDDE904012CA3D3E9002300F0C6FC81
:100FB00029A3D3E9002300F0C1FCFFF7E1BBBCF19A
:100FC000000F40F0D280C3F1140345FA03F202FA95
:100FD00003F3AB4200F0E0806646FFF7E9BB9FED0C
:100FE000207B8DED087B8DED107B9FED057B002533
:100FF0008DED067BC8E44FF0000CA2E4AFF3008057
:10100000000000000000F03FFE822B654715973C72
:1010100000000000432EE63FEF39FAFE422EE63F85
:10102000396CA80C615C20BED0A4BE726937663EE4
:10103000F16BD2C541BDBB3E2CDE25AF6A56113FD8
:1010400093BDBE166CC1663F3E5555555555C53FBF
:10105000000000000000F0BF59F3F8C21F6EA501A8
:101060000000000000000000FFFF8F40FFFF0F00A6
:101070000000F03FFFCB904000346F3F5A4B9C4242
:101080007FF734AC594B9C423FF7BDAB0022574B26
:1010900000F09CFA44A3D3E9002304460D4600F077
:1010A0004DFC43A3D3E9002382468B4620462946C4
:1010B00000F044FC0022CDE902014D4B20462946B8
:1010C00000F03CFC02460B463BA1D1E9000100F0D8
:1010D0007DFA22462B4600F031FC02460B460020EA
:1010E000444900F073FA2246804689462B46204642
:1010F000294600F023FC02460B464046494600F0D4
:101100001DFC2FA3D3E9002300F018FC02460B4678
:10111000DDE9020100F05AFA02460B468046894694
:101120005046594600F054FA002004460D465246F7
:101130005B46AFE502460B46FFF7CFBBDDE9040196
:1011400021A3D3E9002300F0F9FB1FA3D3E9002377
:1011500000F0F4FBFFF714BB264B98453FF708AEB1
:10116000DDE902239246934631E60026FFF72CBBC9
:101170009FED177B8DED087B9FED177B8DED107B31
:101180009FED177B4FF480258DED067BFFF7FCBBB1
:101190005A4600F091F9CAE602F00102C2F10206D5
:1011A000FFF706BBAFF30080000000604715F73F74
:1011B00044DF5DF80BAE543E555555555555D53F5A
:1011C000FE822B654715F73F9C7500883CE4377E0F
:1011D0000000004003B8E23F06D0CF43EBFD4C3E99
:1011E000000000000000F83FFEFFEF3F0000F03F6E
:1011F0000000D03F0000E03F5E4A8A432DE9F04105
:1012000004460D4600F0958000290B4606468446AC
:1012100056DD0F1500F0A580C3F31303A7F2FF37C7
:1012200043F480134FEADC72F80702EB43034FEA02
:101230004C0504D5ED0F05EB43034FEA8C05002662
:101240007F10B44616224FF400110CEB01009842B7
:101250004FEAD5744FEA450503DC1B1A00EB010C7D
:101260000E44013A04EB43034FEA5101EDD110461D
:10127000964620244FF0004209E051D05B00013C2B
:1012800003EBD5734FEA52024FEA450537D0634569
:1012900002EB0E01F1DD002901EB020E0ADBE04654
:1012A000A3EB0C03A94288BF03F1FF336D1A10446E
:1012B000C446E3E7BEF1000FF1DB0CF10108EFE7F4
:1012C00021F00042024329D0002942D10146CA0A36
:1012D000153B4905002AFAD012F4801001D044E0F1
:1012E00060465200D40200F1010CF9D5CCF1200483
:1012F00001FA0CFCE1401F1A41EA02038CE72B4380
:1013000021D14408731003F17F53F20703F5001352
:1013100048BF44F0004403EB07512046BDE8F0818C
:10132000A942ABD8002901EB020EC3DB984600238B
:10133000BCE702460B4600F001FB22462B4600F0BC
:1013400047F9BDE8F081411C16BF421C0136540824
:10135000D8E7024600F03AF902460B4600F018FCC6
:10136000DCE71A4631463B46B6E78C4620244FF070
:10137000FF30BFE70000F07F21F0004319467047BF
:1013800041F0004101F58010C00F70470020704708
:1013900000200149704700BF0000F87F2DE9F041AF
:1013A000C1F30A57A7F2FF35132D82B002460B4650
:1013B0000C464FEAD178064633DC002D4EDB3C4923
:1013C000294103EA0100104326D049080B4052EAA4
:1013D00003060CD04FF48023132D24EA010143FAB5
:1013E00005F444EA01040CBF4FF0004600263149E1
:1013F00001EBC8082346D8E9004532462046294675
:1014000000F0E6F8CDE9000122462B46DDE90001B7
:1014100000F0DCF802460B461046194602B0BDE863
:10142000F081332D07DDB5F5806FF5D100F0D0F8F0
:1014300002460B46F0E7A7F213474FF0FF31F940A1
:101440000842E9D049080842D1D04FF0804320EA51
:10145000010143FA07F741EA0706C8E721F0004116
:101460000143D9D0C3F3130101434E420E43114D42
:101470005C0C360B640406F4002305EBC80243EA57
:101480000401D2E900450B4602462946204600F0F9
:101490009FF8CDE9000122462B46DDE9000100F06E
:1014A00095F821F00041024641EAC873B4E700BF55
:1014B000FFFF0F00508A0100F8B5C1F30A5304463C
:1014C0000D460E4617460BBB21F00046034633433C
:1014D0001BD0354B002200F031FA344B9F420446BA
:1014E0000D4635DBC1F30A530E46363B3B4440F212
:1014F000FE72934232DC002B11DD26F0FF4626F40B
:10150000E00646EA035520462946F8BD40F2FF7240
:101510009342EBD102460B4600F05AF8F8BD13F1A6
:10152000350F28DA4CF250339F4222462B460ADD13
:1015300019A1D1E9000100F03DF817A3D3E9002378
:1015400000F0FCF9F8BD16A1D1E9000100F032F875
:1015500013A3D3E9002300F0F1F9F8BD22462B468E
:101560000DA1D1E9000100F025F80BA3D3E9002378
:1015700000F0E4F9F8BD26F0FF4626F4E006363325
:1015800046EA0355204629460022094B00F0D6F9C9
:10159000F8BD00BFAFF300809C7500883CE4377E47
:1015A00059F3F8C21F6EA50100005043B03CFFFF85
:1015B0000000903C03F0004321F0004242EA0301A6
:1015C000704700BF81F0004102E000BF83F000439C
:1015D00030B54FEA41044FEA430594EA050F08BFCE
:1015E00090EA020F1FBF54EA000C55EA020C7FEA92
:1015F000645C7FEA655C00F0E2804FEA5454D4EB0F
:101600005555B8BF6D420CDD2C4480EA020281EAD8
:10161000030382EA000083EA010180EA020281EA10
:101620000303362D88BF30BD11F0004F4FEA013162
:101630004FF4801C4CEA113102D0404261EB410171
:1016400013F0004F4FEA03334CEA133302D05242F7
:1016500063EB430394EA050F00F0A780A4F10104B3
:10166000D5F1200E0DDB02FA0EFC22FA05F28018ED
:1016700041F1000103FA0EF2801843FA05F35941D3
:101680000EE0A5F120050EF1200E012A03FA0EFC52
:1016900028BF4CF0020C43FA05F3C01851EBE3717C
:1016A00001F0004507D54FF0000EDCF1000C7EEB99
:1016B00000006EEB0101B1F5801F1BD3B1F5001FD7
:1016C0000CD349085FEA30004FEA3C0C04F10104F6
:1016D0004FEA445212F5800F80F09A80BCF1004F1F
:1016E00008BF5FEA500C50F1000041EB045141EAA1
:1016F000050130BD5FEA4C0C404141EB010111F4A2
:10170000801FA4F10104E9D191F0000F04BF01464C
:101710000020B1FA81F308BF2033A3F10B03B3F12A
:1017200020020CDA0C3208DD02F1140CC2F10C02BA
:1017300001FA0CF021FA02F10CE002F11402D8BF18
:10174000C2F1200C01FA02F120FA0CFCDCBF41EAE4
:101750000C019040E41AA2BF01EB0451294330BDB3
:101760006FEA04041F3C1CDA0C340EDC04F1140490
:10177000C4F1200220FA04F001FA02F340EA030067
:1017800021FA04F345EA030130BDC4F10C04C4F1AD
:10179000200220FA02F001FA04F340EA030029468D
:1017A00030BD21FA04F0294630BD94F0000F83F4D7
:1017B000801306BF81F480110134013D4EE77FEABA
:1017C000645C18BF7FEA655C29D094EA050F08BF06
:1017D00090EA020F05D054EA000C04BF19461046E7
:1017E00030BD91EA030F1EBF0021002030BD5FEA2B
:1017F000545C05D14000494128BF41F0004130BD53
:1018000014F580043CBF01F5801130BD01F00045A6
:1018100045F0FE4141F470014FF0000030BD7FEA19
:10182000645C1ABF194610467FEA655C1CBF0B4614
:10183000024650EA013406BF52EA033591EA030F2B
:1018400041F4002130BD00BF90F0000F04BF002123
:10185000704730B54FF4806404F132044FF0000556
:101860004FF0000150E700BF90F0000F04BF0021CF
:10187000704730B54FF4806404F1320410F0004535
:1018800048BF40424FF000013EE700BF42004FEA30
:10189000E2014FEA31014FEA02701FBF12F07F43AD
:1018A00093F07F4F81F06051704732F07F4208BF64
:1018B000704793F07F4F04BF41F40021704730B56B
:1018C0004FF4607401F0004521F000411CE700BFB7
:1018D00050EA010208BF704730B54FF000050AE03A
:1018E00050EA010208BF704730B511F0004502D53B
:1018F000404261EB41014FF4806404F132045FEA3D
:10190000915C3FF4D8AE4FF003025FEADC0C18BFE5
:1019100003325FEADC0C18BF033202EBDC02C2F1D7
:10192000200300FA03FC20FA02F001FA03FE40EA69
:101930000E0021FA02F11444BDE600BF70B54FF06D
:10194000FF0C4CF4E06C1CEA11541DBF1CEA13554B
:1019500094EA0C0F95EA0C0F00F0DEF82C4481EAB3
:10196000030621EA4C5123EA4C5350EA013518BFD3
:1019700052EA033541F4801143F4801338D0A0FBC0
:1019800002CE4FF00005E1FB02E506F00042E0FB6D
:1019900003E54FF00006E1FB03569CF0000F18BF73
:1019A0004EF0010EA4F1FF04B6F5007F64F540741B
:1019B00004D25FEA4E0E6D4146EB060642EAC621AE
:1019C00041EA55514FEAC52040EA5E504FEACE2E1B
:1019D000B4F1FD0C88BFBCF5E06F1ED8BEF1004F1E
:1019E00008BF5FEA500E50F1000041EB045170BD9A
:1019F00006F0004646EA010140EA020081EA0301DE
:101A0000B4EB5C04C2BFD4EB0C0541EA045170BDD9
:101A100041F480114FF0000E013C00F3AB8014F153
:101A2000360FDEBF002001F0004170BDC4F100049C
:101A3000203C35DA0C341BDC04F11404C4F120051D
:101A400000FA05F320FA04F001FA05F240EA020078
:101A500001F0004221F0004110EBD37021FA04F6AE
:101A600042EB06015EEA430E08BF20EAD37070BD68
:101A7000C4F10C04C4F1200500FA04F320FA05F0C7
:101A800001FA04F240EA020001F0004110EBD370C9
:101A900041F100015EEA430E08BF20EAD37070BD39
:101AA000C4F1200500FA05F24EEA020E20FA04F312
:101AB00001FA05F243EA020321FA04F001F00041C1
:101AC00021FA04F220EA020000EBD3705EEA430E32
:101AD00008BF20EAD37070BD94F0000F0FD101F061
:101AE0000046400041EB010111F4801F08BF013C9A
:101AF000F7D041EA060195F0000F18BF704703F0D8
:101B00000046520043EB030313F4801F08BF013D5E
:101B1000F7D043EA0603704794EA0C0F0CEA13551A
:101B200018BF95EA0C0F0CD050EA410618BF52EAD4
:101B30004306D1D181EA030101F000414FF00000DA
:101B400070BD50EA410606BF1046194652EA4306E8
:101B500019D094EA0C0F02D150EA013613D195EA5C
:101B60000C0F05D152EA03361CBF104619460AD1A4
:101B700081EA030101F0004141F0FE4141F47001AE
:101B80004FF0000070BD41F0FE4141F4780170BD9E
:101B900070B54FF0FF0C4CF4E06C1CEA11541DBF03
:101BA0001CEA135594EA0C0F95EA0C0F00F0A7F805
:101BB000A4EB050481EA030E52EA03354FEA013132
:101BC00000F088804FEA03334FF0805545EA131345
:101BD00043EA12634FEA022245EA111545EA10650D
:101BE0004FEA00260EF000419D4208BF964244F1A4
:101BF000FD0404F5407402D25B084FEA3202B61AC3
:101C000065EB03055B084FEA32024FF480104FF496
